:100000000C94CE100C94D1AD0C94A6AD0C947BAD99
:100010000C9450AD0C9425AD0C94FAAC0C94CFAC70
:100020000C944FA50C94FF100C94FF100C94FF102F
:100030000C94FF100C94FD9B0C94FF100C94FF107B
:100040000C94FF100C94FD9D0C94FF100C94FF1069
:100050000C94FF100C94FF100C949C9C0C94FCAD21
:100060000C94FF100C9490A40C94FF100C94FF10AF
:100070000C94FF100C94FF100C94FF100C94FF10C4
:100080000C94FF100C94FF100C94FF100C94FF10B4
:100090000C94FF100C94FF100C94FF100C94FF10A4
:1000A0000C94FF100C94FF100C94FF100C94FF1094
:1000B0000C94FF100C94FF100C94FF100C94FF1084
:1000C0000C94FF100C94FF100C94FF100C94FF1074
:1000D0000C94FF100C94FF100C94FF100C94FF1064
:1000E0000C94FF10E42AE72AD62ADA2AE02A1E2BEB
:1000F000EB2AEF2AF52AF92AFD2A032B072B0B2BD3
:100100001E2B112B152B192B434B484B4D4B574B8B
:10011000614BDA4B6B4B734B7B4B854B8F4B994B46
:10012000A84BB24BDA4BBC4BC64BD04B14511451BD
:100130001B511B511B512251225122512F51295128
:1001400029512951C4A4CAA4DBA4E6A4EEA403A5A2
:10015000F2A403A5F6A4FAA403A500A5084AD73B78
:100160003BCE016E84BCBFFDC12F3D6C74319ABD86
:1001700056833DDA3D00C77F11BED9E4BB4C3E91AA
:100180006BAAAABE000000803F05A84CCDB2D44E99
:10019000B93836A9020C50B9918688083CA6AAAA9B
:1001A0002ABE000000803F00434F4D4D554E49434D
:1001B0004154494F4E0044525952554E00455252F7
:1001C0004F525300494E464F004543484F0020745C
:1001D0006F6F206C6F6E6720657874727573696FCE
:1001E0006E2070726576656E7465640A0020636FB8
:1001F0006C6420657874727573696F6E20707265B7
:1002000076656E7465640A0047322F473320626159
:100210006420706172616D65746572730A00205AA2
:100220003A200020593A200042656420583A2000C4
:100230005072696E742074696D653A200000012562
:10024000311D28FF24301CFF45232F1B0A17FFFFF9
:10025000040806FF06222B1AFFFF043803FF36FFAF
:10026000FFFFFFFFFF50726F746563746564205079
:10027000696E0A00C901C401BD01B601A8016F661B
:10028000660044454255473A006F6B0020573A00DC
:1002900020573A004361703A454D455247454E4319
:1002A000595F5041525345523A310A004361703A06
:1002B000434153455F4C494748545F425249474880
:1002C000544E4553533A300A004361703A544F47F5
:1002D000474C455F4C49474854533A300A00436104
:1002E000703A534F4654574152455F504F5745520D
:1002F0003A300A004361703A4C4556454C494E47E6
:100300005F444154413A310A004361703A5A5F50A8
:10031000524F42453A310A004361703A4155544FB9
:100320004C4556454C3A310A004361703A505249A7
:100330004E545F4A4F423A310A004361703A50527C
:100340004F47524553533A300A004361703A415582
:10035000544F5245504F52545F54454D503A310A14
:10036000004361703A454550524F4D3A310A0046BC
:1003700049524D574152455F4E414D453A4D61728C
:100380006C696E20204649524D574152455F564593
:100390005253494F4E3A312E312E352E34342045AA
:1003A000585452554445525F545950453A4165722C
:1003B0006F7374727564657220534F555243455F75
:1003C000434F44455F55524C3A68747470733A2FEA
:1003D0002F636F64652E616C6570686F626A656318
:1003E00074732E636F6D2F646966667573696F6EC3
:1003F0002F4D41524C494E2050524F544F434F4C79
:100400005F56455253494F4E3A312E30204D4143AD
:1004100048494E455F545950453A4C756C7A426F85
:1004200074204D696E692032204558545255444518
:10043000525F434F554E543A3120555549443A6521
:10044000353530323431312D643436642D34323127
:10045000642D626133612D61323031323664373957
:100460003330660A002F2F200053657474696E675D
:100470002054726176656C20416363656C657261BE
:1004800074696F6E3A200053657474696E67205208
:1004900065747261637420416363656C6572617435
:1004A000696F6E3A200053657474696E67205072EC
:1004B000696E7420416363656C65726174696F6E07
:1004C0003A200053657474696E67205072696E74C7
:1004D00020616E642054726176656C2041636365AF
:1004E0006C65726174696F6E3A200020643A002076
:1004F000693A0020703A0043290A0061626C656421
:1005000020286D696E2074656D702000436F6C64E7
:100510002065787472756465732061726520004B84
:1005200064200023646566696E6520204445464169
:10053000554C545F004B69200023646566696E6505
:10054000202044454641554C545F004B7020002309
:10055000646566696E65202044454641554C545F8C
:1005600000504944204175746F74756E652066694A
:100570006E69736865642120507574207468652005
:100580006C617374204B702C204B6920616E642069
:100590004B6420636F6E7374616E74732066726F48
:1005A0006D2062656C6F7720696E746F20436F6E8B
:1005B00066696775726174696F6E2E680A005049CA
:1005C00044204175746F74756E65206661696C6551
:1005D00064212074696D656F75740A005049442068
:1005E0004175746F74756E65206661696C65642110
:1005F0002054656D706572617475726520746F6FDB
:1006000020686967680A00204B643A2000204B6923
:100610003A2000204B703A20000A20436C6173732B
:10062000696320504944200A002054753A20002074
:100630004B753A2000206D61783A2000206D696E7C
:100640003A200020643A200020626961733A200059
:10065000426564204C6576656C696E672000466172
:10066000696C656420746F20656E61626C65204200
:100670006564204C6576656C696E670A0042656446
:10068000204C6576656C20436F7272656374696F88
:100690006E204D61747269783A000000000000001D
:1006A0003F4300003743546F6F20666172206672CB
:1006B0006F6D207265666572656E636520706F6927
:1006C0006E740A003A20007A5F6D696E3A20202D20
:1006D00032207A5F6D61783A202035005A204F66CB
:1006E000667365742000416374697665204578748B
:1006F00072756465723A2000556E6B6E6F776E206E
:10070000636F6D6D616E643A2022001000C90210A3
:10071000012C014001220170011801B0010E01F00D
:100720000104015002FA00B002F0003003E600D0EC
:1007300003DC009004D2007005C800A006BE0000D3
:1007400008B400B009AA00D00BA000600E960060AB
:10075000118C000015820020197800C01D6E00A0C9
:10076000226400B0275A00902C500000314600E06F
:10077000343C0010383200903A2800603C1E00A043
:100780003D1400803E0A00203F00000000200023AE
:1007900000260029002C002F003200000100000379
:1007A0000106010901000000000000C0C0000000B7
:1007B000000000254300003F43000037434E6F20F8
:1007C00063617365206C696768740A0020706F73D9
:1007D0006974696F6E206F7574206F662072616E28
:1007E00067652E0A003F50726F626520001000ADF1
:1007F0000330016A0150022B0170030A019004F5D5
:1008000000B005E500D006D800F007CE001009C5FD
:1008100000300ABE00500BB700700CB100900DAB59
:1008200000B00EA600D00FA200F0109D001012998B
:1008300000301395005014920070158E0090168BA6
:1008400000B0178700D0188400F0198100101B7EBB
:1008500000301C7B00501D7900701E7600901F73C5
:1008600000B0207000D0216E00F0226B00102469CF
:100870000030256600502663007027610090285ED6
:1008800000B0295C00D02A5900F02B5600102D54DE
:1008900000302E5100502F4E0070304B00903148E8
:1008A00000B0324500D0334200F0343E0010363BF9
:1008B00000303737005038330070392E00903A2915
:1008C00000B03B2300D03C1B00F03D1100103F0165
:1008D00000F03F0000206673616374697665002054
:1008E0006F7400206F74707700207332676100208E
:1008F0007332676200206F6C6100206F6C620020B1
:1009000073740020656E002074737465705F617687
:10091000673A002063736163743A00206176675F11
:1009200073673A00207367743A0020737465616CD2
:10093000746800207673656E3A002F002069687233
:100940003A002045303A0020667361637469766529
:1009500000206F7400206F7470770020733267611D
:1009600000207332676200206F6C6100206F6C6240
:10097000002073740020656E002074737465705FCE
:100980006176673A002063736163743A0020617690
:10099000675F73673A00207367743A002073746569
:1009A000616C746800207673656E3A002F002069D0
:1009B00068723A00205A3A0020667361637469765F
:1009C0006500206F7400206F7470770020733267A9
:1009D0006100207332676200206F6C6100206F6CD1
:1009E00062002073740020656E002074737465705B
:1009F0005F6176673A002063736163743A00206137
:100A000076675F73673A00207367743A00207374E7
:100A100065616C746800207673656E3A002F002063
:100A20006968723A0020593A0020667361637469FC
:100A3000766500206F7400206F7470770020733229
:100A4000676100207332676200206F6C6100206F65
:100A50006C62002073740020656E002074737465EE
:100A6000705F6176673A002063736163743A0020B7
:100A70006176675F73673A00207367743A0020738A
:100A80007465616C746800207673656E3A002F009F
:100A9000206968723A0020583A00544D433231338D
:100AA00030205374617475733A0A007A5F6D61780F
:100AB0003A20007A5F6D696E3A2000795F6D617847
:100AC0003A2000785F6D696E3A20005265706F724F
:100AD00074696E6720656E6473746F7020737461DF
:100AE0007475730A004572726F723A002020506C60
:100AF000616E6E6572427566666572427974657381
:100B00003A20002046726565204D656D6F72793A16
:100B10002000436F6D70696C65643A204E6F7620DB
:100B2000323120323031370A00207C204175746820
:100B30006F723A2028416C657068204F626A656365
:100B4000747320496E632E2C204C756C7A426F743E
:100B500020476974205265706F7369746F727929C8
:100B60000A004E6F76203231203230313731333A3D
:100B700033303A323900204C61737420557064610F
:100B80007465643A2000312E312E350A004D6172B1
:100B90006C696E0020536F667477617265205265D0
:100BA0007365740A00205761746368646F6720522C
:100BB000657365740A002042726F776E206F7574DA
:100BC0002052657365740A002045787465726E6101
:100BD0006C2052657365740A00506F7765725570AA
:100BE0000A0073746172740A00290A002F33322CD0
:100BF000207673656E73653D00206D412028697213
:100C0000756E3D0045302063757272656E74207399
:100C1000657420746F2000290A002F33322C20764F
:100C200073656E73653D00206D4120286972756E95
:100C30003D005A2063757272656E7420736574206E
:100C4000746F2000290A002F33322C207673656ED2
:100C500073653D00206D4120286972756E3D005915
:100C60002063757272656E742073657420746F20D2
:100C700000290A002F33322C207673656E73653D90
:100C800000206D4120286972756E3D005820637503
:100C90007272656E742073657420746F2000205A20
:100CA0003A0020593A0020583A00656E6473746F18
:100CB0007073206869743A20006563686F3A007445
:100CC0007275650066616C736500206178697320D8
:100CD00074656D7065726174757265207072657788
:100CE00061726E207472696767657265643A20008C
:100CF000207072657761726E20666C616720636C2C
:100D000065617265640A004572726F72207772695C
:100D100074696E6720746F20454550524F4D210A0B
:100D2000002066697273740A005A0059005800481E
:100D30006F6D652000656E7175657565696E6720FC
:100D4000220000002200250028002B002E00310088
:100D5000340002010000050108010B010000210020
:100D6000240027002A002D0030003300010100007C
:100D7000040107010A010102102020080810204088
:100D8000102040800201020108040201010204084F
:100D900010204080804020100804020180040201DD
:100DA0008040201008040201080402010102040826
:100DB0001020408001020408102040800505050530
:100DC000070508080808020202020A0A08080404C3
:100DD00004040101010101010101030303030303F1
:100DE0000303040707070C0C0C0C0C0C0C0C020280
:100DF000020206060606060606060B0B0B0B0B0B7D
:100E00000B0B25753A2530327500253032753A25A1
:100E10003032750025756420253032753A25303220
:100E2000750020647269766572206F7665727465EC
:100E30006D7065726174757265207761726E696E2E
:100E400067210A003A200000000A0B02090C0D0E6F
:100E5000080703040100000000000000000000007B
:100E60000000000000000000000000000000000082
:100E7000000000121110000000000000000000003F
:100E800000000000000000000000000000202863B7
:100E9000616C63756C6174656429210A0020213DD1
:100EA0002000454550524F4D20435243206D6973F9
:100EB0006D61746368202D202873746F72656429D6
:100EC0002000290A002062797465733B20637263F5
:100ED00020002073746F7265642073657474696E8A
:100EE00067732072657472696576656420280020D6
:100EF0004D61726C696E3D563430290A00284545B3
:100F000050524F4D3D00454550524F4D2076657231
:100F100073696F6E206D69736D6174636820005032
:100F2000726F62696E67206661696C656400505219
:100F30004F4245204641494C20434C45414E204EAE
:100F40004F5A5A4C450A005265776970696E670AB4
:100F50000050726F62696E67206661696C6564003B
:100F600050524F4245204641494C20434C45414E4A
:100F7000204E4F5A5A4C450A005265776970696E87
:100F8000670A0050726F62696E67206661696C65FE
:100F9000640A00205A3A200020593A200042656431
:100FA00020583A200020746F6F206C6F6E672065A8
:100FB0007874727573696F6E2070726576656E7481
:100FC00065640A0020636F6C6420657874727573C1
:100FD000696F6E2070726576656E7465640A00488C
:100FE000617264636F6465642044656661756C74E6
:100FF0002053657474696E6773204C6F6164656417
:101000000A00282300002823000064000000E803F1
:1010100000000000964300009643000000410000DD
:10102000C8410000C9420000C942A5C2DF44000017
:10103000D243202F002042403A0020403A004E6F19
:10104000204C696E65204E756D62657220776974FB
:101050006820636865636B73756D2C204C617374D5
:10106000204C696E653A20005072696E746572207A
:1010700073746F707065642064756520746F20658B
:1010800072726F72732E20466978207468652065CD
:1010900072726F7220616E6420757365204D3939EC
:1010A0003920746F20726573746172742E20285415
:1010B000656D706572617475726520697320726503
:1010C0007365742E2053657420697420616674659D
:1010D000722072657374617274696E67290A004EBA
:1010E0006F20436865636B73756D20776974682042
:1010F0006C696E65206E756D6265722C204C617333
:1011000074204C696E653A2000636865636B737583
:101110006D206D69736D617463682C204C6173740C
:10112000204C696E653A20004C696E65204E756DE5
:10113000626572206973206E6F74204C6173742035
:101140004C696E65204E756D6265722B312C204C9A
:10115000617374204C696E653A20004D3131300066
:101160004B494C4C45442E20004B494C4C2063616C
:101170007573656420627920746F6F206D75636884
:1011800020696E6163746976652074696D65202DD0
:101190002063757272656E7420636F6D6D616E642D
:1011A0003A20002064726976657220686F6D696EFE
:1011B000672073656E7369746976697479207365E5
:1011C0007420746F2000205A3A0020593A002043BE
:1011D0006F756E7420583A0020453A00205A3A0044
:1011E00020593A00583A00290A0020627974657340
:1011F0003B20637263200053657474696E677320CB
:1012000053746F726564202800205A0020590058DA
:101210000020204D61783A2000205A0020590058C3
:101220000020204D696E3A20004F6E20004F666608
:1012300000536F667420656E6473746F70733A2028
:101240000020643A0020693A0020703A00204500EE
:10125000205A0020204D39303720580053746570D3
:10126000706572206D6F746F722063757272656E37
:1012700074733A0A0020453000205A00205900209B
:101280005800537465707065722064726976657277
:101290002063757272656E743A0A0020204D3835ED
:1012A00031205A005A2D50726F6265204F66667366
:1012B000657420286D6D293A0A00204400204900F9
:1012C00020204D333034205000204400204900209D
:1012D000204D3330312050005049442073657474E0
:1012E000696E67733A0A0020204D34323020530073
:1012F0004175746F20426564204C6576656C696E3B
:10130000673A0A00205A0020590020204D3230361A
:10131000205800486F6D65206F66667365743A0AE1
:1013200000204500205A002059002058002042008B
:1013300020540020204D3230352053004164766126
:101340006E6365643A20533C6D696E5F66656564E3
:10135000726174653E20543C6D696E5F7472617693
:10136000656C5F66656564726174653E20423C6DC4
:10137000696E5F7365676D656E745F74696D655FD7
:101380006D733E20583C6D61785F78795F6A657255
:101390006B3E205A3C6D61785F7A5F6A65726B3E86
:1013A00020453C6D61785F655F6A65726B3E0A003F
:1013B00020540020520020204D3230342050004173
:1013C0006363656C65726174696F6E2028756E6900
:1013D00074732F7332293A20503C7072696E745FB7
:1013E000616363656C3E20523C7265747261637424
:1013F0005F616363656C3E20543C74726176656C1A
:101400005F616363656C3E0A00204500205A00203E
:10141000590020204D3230312058004D6178696DDF
:10142000756D20416363656C65726174696F6E20D0
:1014300028756E6974732F7332293A0A00204500AB
:10144000205A0020590020204D3230332058004DC2
:101450006178696D756D2066656564726174657328
:101460002028756E6974732F73293A0A002045008D
:10147000205A0020590020204D3932205800537442
:101480006570732070657220756E69743A0A002069
:10149000204D3230302044300A0020204D32303090
:1014A0002044002044697361626C65640A004669E7
:1014B0006C616D656E742073657474696E67733AE0
:1014C000002020473231202020203B20556E6974B7
:1014D0007320696E206D6D0A002061786973206445
:1014E00072697665722063757272656E743A200057
:1014F00020496E76616C69642065787472756465E4
:101500007220002569730025696D20256973002507
:1015100069682025696D2025697300256964202587
:1015200069682025696D2025697300256979202562
:101530006964202569682025696D20256973000A82
:101540000A426564204C6576656C20436F72726553
:101550006374696F6E204D61747269783A00202B54
:10156000000A436F7272656374656420426564208B
:101570004865696768742076732E2042656420543C
:101580006F706F6C6F67793A0A00202B000A426512
:10159000642048656967687420546F706F67726172
:1015A0007068793A0A2020202B2D2D2D20424143AE
:1015B0004B202D2D2B0A2020207C20202020202095
:1015C00020202020207C0A204C207C202020202845
:1015D0002B29202020207C20520A2045207C2020FE
:1015E0002020202020202020207C20490A20462066
:1015F0007C20282D29204E20282B29207C20470ABA
:101600002054207C20202020202020202020207CEE
:1016100020480A2020207C20202020282D2920203E
:1016200020207C20540A2020207C202020202020E4
:1016300020202020207C0A2020204F2D2D204652C3
:101640004F4E54202D2D2B0A2028302C30290A00F3
:101650004D65616E206F662073616D706C656420EE
:10166000706F696E74733A200020643A2000206223
:101670003A200045716E20636F656666696369652F
:101680006E74733A20613A200052756E6E696E670F
:1016900020696E204452592D52554E206D6F64655D
:1016A0000A00473239204175746F20426564204C2E
:1016B0006576656C696E670A0028422961636B0074
:1016C000284629726F6E7400285229696768740071
:1016D000284C29656674003F4E756D626572206FF7
:1016E000662070726F626520706F696E7473206916
:1016F0007320696D706C61757369626C6520283246
:10170000206D696E696D756D292E0A003F28562976
:101710006572626F7365206C6576656C20697320F5
:10172000696D706C61757369626C652028302D3449
:10173000292E0A000000F0410000F04100000041A5
:10174000000000005761726E696E673A20486F6D45
:10175000696E672042756D702044697669736F7297
:10176000203C20310A0002020400000000000000BA
:101770000000000040000025430000454300003702
:1017800043FF01014B494C4C45442E200024F4D426
:101790003050C38E20C2A24017828B7011127A91F2
:1017A0000D816CD90AA861E108C7586607615143E9
:1017B000061E4B5D05C145A7041A411104093D9859
:1017C00003713931034036DB0265339102D4305462
:1017D00002802E1D02632CEE01752AC501B028A0DF
:1017E00001102781018F2564012B244B01E0223455
:1017F00001AC211F018D200D01801FFC00841EED16
:1018000000971DDF00B81CD200E61BC600201BBCE1
:1018100000641AB200B219A8000A19A0006A189947
:1018200000D117910040178B00B516840031167E49
:1018300000B31579003A157300C7146F0058146A85
:1018400000EE1366008813630025135E00C7125B69
:10185000006C12570015125400C111510070114F45
:101860000021114B00D61049008D1047004610444E
:101870000002104200C00F4000800F3E00420F3CAB
:1018800000060F3B00CB0E3800930E37005C0E3580
:1018900000270E3400F30D3200C10D3100900D30E1
:1018A00000600D2E00320D2D00050D2C00D90C2BE3
:1018B00000AE0C2900850C29005C0C2700350C2794
:1018C000000E0C2600E80B2400C40B2400A00B2300
:1018D000007D0B23005A0B2100390B2100180B202F
:1018E00000F80A1F00D90A1E00BB0A1E009D0A1D2F
:1018F00000800A1D00630A1C00470A1B002C0A1BFB
:1019000000110A1A00F7091A00DD091900C40919A3
:1019100000AB091900920917007B09180063091729
:10192000004C09160036091600200916000A091590
:1019300000F5081500E0081400CC081400B80814DD
:1019400000A4081400900813007D0812006B08130F
:10195000005808120046081200340811002308112C
:10196000001208110001081100F0071000E0071034
:1019700000D0071000C0071000B0070F00A107102B
:101980000091070E0083070F0074070F0065070E14
:101990000057070E0049070E003B070D002E070EEB
:1019A0000020070D0013070D0006070D00F9060CB7
:1019B00000ED060D00E0060C00D4060C00C8060C75
:1019C00000BC060C00B0060C00A4060B0099060C27
:1019D000008D060B0082060B0077060B006C060BD1
:1019E0000061060A0057060B004C060A0042060A70
:1019F0000038060A002E060A0024060A001A060A03
:101A0000001006090007060A00FD050900F4050993
:101A100000EB050900E2050900D9050900D0050918
:101A200000C7050900BE050900B5050800AD050899
:101A300000A50509009C050800940508008C050810
:101A400000840508007C050800740508006C050783
:101A500000650508005D050700560508004E0507EE
:101A60000047050700400508003805070031050755
:101A7000002A050700230507001C050600160507B8
:101A8000000F0507000805060002050700FB040615
:101A900000F5040700EE040600E8040600E204076F
:101AA00000DB040600D5040600CF040600C90406C6
:101AB00000C3040600BD040600B7040600B1040517
:101AC00000AC040600A6040600A00405009B040662
:101AD0000095040500900406008A040500850405AD
:101AE00000800406007A04050075040500700405F2
:101AF000006B04050066040500610405005C040534
:101B00000057040500520405004D04050048040573
:101B100000430405003E0404003A040500350405B2
:101B200000300404002C04050027040400230405ED
:101B3000001E0404001A0404001604050011040425
:101B4000000D04040009040500040404000004045A
:101B500000FC030400F8030400F4030400F0030491
:101B600000EC030400E8030400E4030400E00304C1
:101B700000DC030400D8030400D4030400D00304F1
:101B800000CC030400C8030300C503030024F404CD
:101B9000D9201BC40C5C0E9804C4095F0265077150
:101BA00001F405F900FB04B30048048700C1036990
:101BB000005803550003034500BE023A0084023179
:101BC0000053022A002902250004022000E4011C1F
:101BD00000C8011900AF0117009801140084011317
:101BE00000710110006101100051010E0043010D50
:101BF0000036010B002B010B0020010B0015010921
:101C0000000C01090003010800FB000800F30008B4
:101C100000EB000700E4000600DE000600D8000626
:101C200000D2000600CC000500C7000500C2000578
:101C300000BD000400B9000400B5000400B10004B8
:101C400000AD000400A9000400A5000300A20003E9
:101C5000009F0004009B0003009800030095000211
:101C60000093000300900003008D0002008B00032E
:101C70000088000200860002008400030081000248
:101C8000007F0002007D0002007B0002007900025C
:101C9000007700010076000200740002007200016B
:101CA00000710002006F0002006D0001006C000274
:101CB000006A00010069000200670001006600017F
:101CC0000065000100640002006200010061000183
:101CD00000600001005F0002005D0001005C000187
:101CE000005B0001005A000100590001005800018A
:101CF000005700010056000100550001005400018A
:101D00000053000000530001005200010051000187
:101D100000500001004F0001004E0000004E000185
:101D2000004D0001004C0001004B0000004B000181
:101D3000004A00010049000100480000004800017D
:101D40000047000100460000004600010045000079
:101D50000045000100440001004300000043000171
:101D6000004200000042000100410000004100016B
:101D700000400001003F0000003F0001003E000065
:101D8000003E0001003D0000003D0001003C00005D
:101D9000003C0000003C0001003B0000003B000153
:101DA000003A0000003A000100390000003900014B
:101DB0000038000000380000003800010037000043
:101DC0000037000100360000003600000036000138
:101DD000003500000035000000350001003400002F
:101DE0000034000000340001003300000033000024
:101DF0000033000100320000003200000032000118
:101E0000003100000031000000310001003000000E
:101E10000030000000300001002F0000002F000003
:101E2000002F0000002F0001002E0000002E0000F7
:101E3000002E0001002D0000002D0000002D0000EC
:101E4000002D0001002C0000002C0000002C0000E0
:101E5000002C0001002B0000002B0000002B0000D4
:101E6000002B0001002A0000002A0000002A0000C8
:101E7000002A0001002900000029000000290000BC
:101E800000290000002900010028000000280000AF
:101E900000280000002800000028000100270000A2
:101EA0000027000000270000002700000027000195
:101EB000002600000026000000260000002600008A
:101EC000002600010025000000250000002500007C
:101ED000002500000025000000250001002400006E
:101EE0000024000000240000002400000024000161
:101EF0000023000000230000002300000023000056
:101F00000023000000230000002300010022000045
:101F10000022000000220000002200000022000039
:101F2000002200010021000000210000002100002B
:101F3000002100000021000000210000002100011C
:101F40000020000000200000002000000020000011
:101F50000020000000200000002000000020000100
:101F6000001F0000001F0000001F0000001F0000F5
:101F7000001F0000001F0000001F0001001E0000E5
:101F8000001E0000001E0000001E000000457272CE
:101F90003A204D494E54454D5020424544004D494C
:101FA0004E54454D502074726967676572656400D0
:101FB0004572723A204D494E54454D5020453100EE
:101FC0004572723A204D494E54454D5020453000DF
:101FD0004572723A204D415854454D502042454477
:101FE000004D415854454D502074726967676572C1
:101FF0006564004572723A204D415854454D502059
:102000004531004572723A204D415854454D50209B
:10201000453000026D0046696C616D656E74207517
:102020007365643A200053746174733A20002C2065
:102030004C6F6E67657374206A6F623A2000546F4C
:1020400074616C2074696D653A2000537461747317
:102050003A20002C204661696C65643A20002C20EF
:1020600046696E69736865643A20005072696E74DF
:10207000733A200053746174733A200020420020A8
:1020800050006F6B00526573656E643A20005072A9
:10209000696E7465722068616C7465642E206B696A
:1020A0006C6C28292063616C6C6564210A00626590
:1020B000640A002C2073797374656D2073746F70DB
:1020C00070656421204865617465725F49443A20F7
:1020D00000544845524D414C2052554E41574159AC
:1020E0002042454400546865726D616C2052756EE3
:1020F0006177617900544845524D414C2052554E0C
:102100004157415920453100544845524D414C20DA
:1021100052554E4157415920453000486561746918
:102120006E67206661696C656420424544004865BD
:102130006174696E67206661696C656400486561F9
:1021400074696E67206661696C65640048656174D6
:10215000696E67206661696C6564204530004E4198
:102160004E494E495459494E46CDCCCC3D0AD72311
:102170003C17B7D13877CC2B329595E6241FB14F59
:102180000A000020410000C84200401C4620BCBE9E
:102190004CCA1B0E5AAEC59D740002AC11241FBE62
:1021A000CFEFD1E2DEBFCDBF00E00CBF13E0A0E077
:1021B000B2E0ECEFF7E701E00BBF02C007900D9231
:1021C000A832B107D9F72FE0A8E2B3E001C01D9211
:1021D000A636B207E1F711E2CCE9D1E200E006C091
:1021E00022970109FE010BBF0E94E7BACA39D10745
:1021F00080E00807A9F70E940D430C94FCBB0C94E7
:1022000000002F923F924F925F926F927F928F9237
:102210009F92AF92BF92CF92DF92EF92FF920F9375
:102220001F93CF93DF93CDB7DEB7C955D1090FB652
:10223000F894DEBF0FBECDBF0091580620E6029F86
:1022400080011124095D1B4F8091260480FF1AC074
:10225000E9EBFCE084917F013FEFE31AF30A81117F
:1022600002C0780104C00E94FD34F701F3CFD7010A
:102270008D917D01882319F00E94FD34F8CF8AE00A
:102280000E94FD3410929A03109299038FE3809379
:1022900025041092240410922304109242031092F9
:1022A00043031092440310924503F80180810F5FAD
:1022B0001F4F8032D1F38E34B1F4818190ED980FAD
:1022C0009A3020F08D3211F08B3269F43296DF01B2
:1022D00031962C9120532A30D0F3CD01FC01019688
:1022E00020812032D9F3F0931D04E0931C047F0178
:1022F000BFEFEB1AFB0A10816AE270E0C7010E948F
:10230000DCBB009739F0DC0111978C918032E1F34E
:1023100011961C921D3429F0143519F0173409F068
:10232000CDC0F7014E2F9F2F81918032D9F380537A
:102330008A3008F0C3C01093250420912304309103
:102340002404E42FF92F6AE0AF014F5F5F4F629FD3
:10235000C001639F900D1124208130E0205331098A
:10236000820F931F218120532A3030F09093240450
:10237000809323049A0103C09C01FA01E5CFD9019F
:102380002F5F3F4F4C914032D1F31D3449F0B09054
:102390001C044091990350919A0361E070E050C091
:1023A0008E31910591F03CF48731910571F08C31BB
:1023B000910569F70AC0853791054CF38737910578
:1023C00024F0803AE3E09E0711F7B0939A03A093BC
:1023D000990374C02132F1F10FEB020F0A3108F0BA
:1023E0005AC09F01F901A0812F5F3F4FA032D1F366
:1023F00020ED2A0F2A3008F042C09F01E02EF12C78
:10240000D701B595A795B595A795B595A795AE5B59
:10241000BC4F07706B01002E01C0CC0C0A94EAF788
:10242000DC90DC28DC922115310599F12B19D701BC
:10243000A85DBC4F2C93208121542A3188F5DF01FF
:10244000FD0131962C912111C5CF50939A034093F1
:10245000990334C01D3409F0BFCF8032910509F0D3
:10246000BBCFF0939A03E093990363E270E0CF014E
:102470000E94DCBB009711F1DC011C921FC023ED10
:102480002A0F223008F4B9CFAB3211F00C94022697
:10249000B4CF20E0CCCF4115510569F6AD01CBCFCB
:1024A0009F013196D9010C9100530A30C8F3F9010C
:1024B0002F5F3F4FA081A032D1F3C1CF809125047F
:1024C0008D3409F45FC5843511F40C94A425873448
:1024D00011F00C94E52580912304909124048A3115
:1024E000910509F436C3A4F48430910544F4823094
:1024F00091050CF01CC197FF28C00C94FF25843077
:10250000910509F4A9C20C9709F4E1C20C94FF25C6
:102510008E31910509F45FC43CF48C31910509F4C6
:102520009FC30CF41BC34AC48B35910509F4F0C456
:102530008C35910509F4F1C48A35910511F00C949C
:10254000FF25109222040C94FF25809126028823F7
:1025500011F40C94FF250E94675086E493E00E94DA
:1025600079360E94A4398091260483FD8FC0C090E3
:102570005203D0905303E0905403F0905503209100
:102580000606309107064091080650910906C701DA
:10259000B6010E948EB3882309F478C08091CD03E0
:1025A000811138C06091140270911502882777FD5F
:1025B0008095982F0E9494B39B01AC016091E60333
:1025C0007091E7038091E8039091E9030E948EB334
:1025D00087FF20C0C0920606D0920706E092080648
:1025E000F0920906E9EBFCE084918F010F5F1F4F29
:1025F000882321F00E94FD34F801F6CFEDEEF1E0E2
:1026000084918F010F5F1F4F882321F00E94FD34BA
:10261000F801F6CFC0905203D0905303E0905403DA
:10262000F090550320910606309107064091080668
:1026300050910906C701B6010E94EBB720E030E0D7
:1026400048E453E40E9412BA181604F5C092060634
:10265000D0920706E0920806F0920906E9EBFCE04A
:1026600084918F010F5F1F4F882321F00E94FD345A
:10267000F801F6CFEEECF1E084918F010F5F1F4F70
:10268000882321F00E94FD34F801F6CF2091460303
:102690003091470340914803509149036091FA05F6
:1026A0007091FB058091FC059091FD050E948EB311
:1026B00081111DC020914A0330914B0340914C037E
:1026C00050914D036091FE057091FF0580910006C9
:1026D000909101060E948EB3811109C060910A0297
:1026E00070910B0280910C0290910D021AC06091C2
:1026F000120270911302882777FD8095982F0E940F
:1027000094B320910A0230910B0240910C02509137
:102710000D020E94F3B32AE037ED43E25CE30E942E
:10272000F3B30E94E86F0E94CE360C94FF252091EF
:102730002602222311F40C94FF2511E0029709F0E0
:1027400010E00E94675019821A821B821C821D822F
:102750001E821F82188682E50E94CC37882309F4E6
:102760002CC10E9403366B017C012091FA05309147
:10277000FB054091FC055091FD052F8F38A349A31F
:102780005AA38090FE059090FF05A0900006B0909F
:1027900001068091460390914703A0914803B091B0
:1027A00049038BA39CA3ADA3BEA320914A03309100
:1027B0004B0340914C0350914D032FA338A749A7D9
:1027C0005AA720E030E0A901C701B6010E948EB3EC
:1027D000882309F408C12F8D38A149A15AA16BA102
:1027E0007CA18DA19EA10E948EB381110BC0A50179
:1027F00094016FA178A589A59AA50E948EB388231C
:1028000009F4F1C020E030E0A901C701B6010E943F
:102810008EB3881F8827881F181749F080E090E042
:10282000A0E8BFEB8FAB98AFA9AFBAAF08C020E06C
:1028300030E040E85FE32FAB38AF49AF5AAF2F8DA0
:1028400038A149A15AA16BA17CA18DA19EA10E9492
:10285000EBB76FA778AB89AB9AABA50194016FA1D9
:1028600078A589A59AA50E94EBB76BAB7CAB8DAB25
:102870009EAB2FA538A949A95AA9CA01B9010E943E
:10288000F3B32B013C012BA93CA94DA95EA9CA01B8
:10289000B9010E94F3B39B01AC01C301B2010E94D4
:1028A000ECB70E9457BA6BA77CA78DA79EA720E024
:1028B00030E040E05FE30E94F3B32B013C01A7014D
:1028C0009601C701B6010E94F3B36B017C01A3011D
:1028D0009201C301B2010E94F3B39B01AC01C70195
:1028E000B6010E94EBB70E9457BA9B01AC016FA9D9
:1028F00078AD89AD9AAD0E94F3B36B017C012BA139
:102900003CA14DA15EA16F8D78A189A19AA10E94E1
:10291000ECB720E030E040E05FE30E94F3B32B012E
:102920003C016BA97CA98DA99EA990582BA53CA51B
:102930004DA55EA50E94C8B89B01AC01C701B601B8
:102940000E94F3B39B01AC01C301B2010E94ECB73A
:102950002F8D38A149A15AA10E94EBB769837A83D0
:102960008B839C832FA138A549A55AA5C501B40125
:102970000E94ECB720E030E040E05FE30E94F3B358
:102980002B013C012BA53CA54DA55EA56FA578A903
:1029900089A99AA90E94C8B89B01AC01C701B601D8
:1029A0000E94F3B39B01AC01C301B2010E94ECB7DA
:1029B000A50194010E94EBB712C089E40E94CC37B4
:1029C000882331F00E94033669837A838B839C834A
:1029D0008AE40E94CC37882331F00E9403366D834D
:1029E0007E838F83988720E030E0A90169817A8116
:1029F0008B819C810E948EB381110BC020E030E05E
:102A0000A9016D817E818F8198850E948EB3882374
:102A100049F0612FCE0101960E9460880E94A4397E
:102A20000C94FF25E5EEFAE084918F010F5F1F4FB4
:102A3000882321F00E94FD34F801F6CFE8E0F2E0AF
:102A400084918F010F5F1F4F882311F40C94FF2591
:102A50000E94FD34F801F4CF80E50E94CC37882332
:102A600029F00E94C3354B015C0103C0812C912CDD
:102A7000540183E50E94CC37882361F00E9403361D
:102A800020E030E04AE754E40E94F3B30E9435B9F5
:102A90004B015C010E94345E0E94A439C090560331
:102AA000D0905703E0905803F0905903C80CD91CFC
:102AB000EA1CFB1C0E94DB386C197D098E099F09FA
:102AC00097FD02C00C94FF250E940872F3CF0E946C
:102AD000FF4F81110C94FF2580E50E94CC3788239D
:102AE00019F00E94D33501C060E06E8F83E50E942B
:102AF000CC37882319F00E94D33501C06CE06A8F6F
:102B000084E50E94CC37882319F00E94D33501C098
:102B100063E06E8B82E50E94CC37882319F00E9417
:102B2000033604C060E070E080ED90E469837A834E
:102B30008B839C839E012A5E3F4FAE014F5F5F4FA8
:102B4000BE01665E7F4FCE014E960E9416530C94D6
:102B5000FF2581E0809326020C94FF250E94FF4F01
:102B600081110C94FF2580E50E94CC37882321F049
:102B70000E94D335462F01C040E06091020670915B
:102B80000306809104069091050600E010E020E223
:102B900031E409831A832B833C8300E010E025E3B2
:102BA00033E40D831E832F83388700E010E020EA92
:102BB00031E409871A872B873C8700E010E020EC7E
:102BC0003FE70D871E872F87388B413071F14230E8
:102BD00021F51E8A1F8A188E198E20E030E040EA07
:102BE00051E40E94ECB77B018C0120E030E047E328
:102BF00053E40E9412BA181624F4E12CF12C07E3D6
:102C000013E4A701B8014A8F5B8F6C8F7D8FBE01E3
:102C10006A5E7F4FCE014A9611C020E030E040EA64
:102C200051E40E948EB387FF0BC01E8A1F8A188E44
:102C3000198EBE016A5E7F4FCE0109960E940F5326
:102C40001E8A1F8A188E198EAE014A5E5F4FBE0122
:102C50006B5F7F4FCE0101960E940B530C94FF25B2
:102C60000E94345E1091EF0380E00E9473A60E94E0
:102C7000C73981E08093E90588E50E944237E82E54
:102C800089E50E944237F82E8AE50E944237D82E05
:102C9000E11005C0F11007C001E0082705C0FF20C2
:102CA00011F0082F01C000E080E1EAEFF5E0A6E4B2
:102CB000B3E001900D928A95E1F7011105C0D110A2
:102CC00003C0E11006C00AC082E00E94428C0023CB
:102CD000C1F380E00E94428C011102C0FF2019F074
:102CE00081E00E94428C0E941B611E8A1F8A188EFE
:102CF000198E01110BC0D11009C0409102065091EC
:102D00000306609104067091050604C040E050E09F
:102D100062E373E449835A836B837C83BE016A5EFA
:102D20007F4FCE0101960E940F5340E050E060EAD1
:102D300070E44A8F5B8F6C8F7D8F01110BC0F11097
:102D400009C04091FE055091FF0560910006709109
:102D5000010604C040E050E06AE373E44E8B5F8BF1
:102D6000688F798F01110BC0E11009C04091FA05FD
:102D70005091FB056091FC057091FD0504C040E099
:102D800050E060EA70E449835A836B837C83AE0130
:102D9000465E5F4FBE016A5E7F4FCE0101960E9484
:102DA0000B5380919B038093E905812F0E9473A6AA
:102DB0000E94AE390E9466780C94FF2581E08093D2
:102DC000ED0524982C9A0E945E8D1092ED05249AB0
:102DD0002C980C94FF2520E030E0A9016091FA05C1
:102DE0007091FB058091FC059091FD050E94ECB768
:102DF000182F88E568966FAF689769967FAF6997D7
:102E00006A969FAF6A970E94CC3768966FAD6897B5
:102E100069967FAD69976A969FAD6A97882321F07E
:102E20000E9403369B0102C09B01812FA901BC01B6
:102E30004E8B5F8B688F798F20E030E0A901609125
:102E4000FE057091FF0580910006909101060E9499
:102E5000ECB75B018C0189E50E94CC37882321F017
:102E60000E9403365B018C01A501B80149835A8396
:102E70006B837C834090F4035090F5036090F603DD
:102E80007090F7032091F0033091F1034091F20329
:102E90005091F3036E897F89888D998D0E94EBB7DD
:102EA0006B017C012FE632E143E85AEB0E9412BA33
:102EB00087FF02C00C94FF2522E430E045E253E492
:102EC000C701B6010E948EB3181614F40C94FF25A6
:102ED000A3019201B501C8010E94EBB76B017C010F
:102EE00021E338E040EC50EC0E9412BA87FF02C0A8
:102EF0000C94FF2522E430E04FE353E4C701B60110
:102F00000E948EB3181614F40C94FF250C940C2612
:102F100081E0809322040C94FF2585E40E94CC3745
:102F2000C82E811102C00E94345EFCEEEF2EF2E04A
:102F3000FF2E0AEF15E0B12CD12CD7018D917D0128
:102F40000E94CC37882361F00E940336F801608329
:102F5000718382839383F3E0DF1611F0BB24B39473
:102F6000D3940C5F1F4F24E0D212E7CFBB2019F09F
:102F70000E941B6103C0C1100E94C14F0E9466786D
:102F80000C94FF2580912304909124048E3B91059D
:102F900009F4DCC30CF0B3C08C35910509F48EC480
:102FA0000CF063C08C34910509F453C2ACF5823146
:102FB000910509F431C494F497FF02C00C94FF25E5
:102FC000823091050CF451C1419711F00C94FF250A
:102FD00017981698159814980C94FF258A32910525
:102FE00009F4DEC18B34910509F42FC24F9711F01B
:102FF0000C94FF258FE29FE00E94E7386E8B7F8B59
:10300000888F998FBE016F5F7F4FCE0146960E94D9
:10301000037FE9EBFCE0AEC18235910509F4F3C30F
:10302000C4F48E34910509F42DC20CF427C2813505
:10303000910511F00C94FF250E9401A60E94345EB8
:103040000E94AFA7109264031092630300E010E0A7
:10305000C3C38435910509F4DFC30CF4D8C38535A7
:10306000910509F410C40C94FF258237910509F4E9
:10307000ABC4FCF48B36910509F49CC364F4893627
:10308000910509F404C30CF076C38836910509F460
:10309000FDC10C94FF258E36910509F426C28F36AA
:1030A000910509F435C28D36910511F00C94FF2578
:1030B00031C38837910509F461C574F486379105E9
:1030C00009F418C50CF04DC58337910511F00C9427
:1030D000FF25EFE6F3E07EC48C38910509F4B9C210
:1030E0008B39910509F4EDC28937910511F00C94E3
:1030F000FF251092E90510929B030C94FF2580395F
:1031000031E0930711F40C94F5220CF04FC08C3D84
:10311000910509F430C614F58C3C910509F4BBC542
:1031200074F4893C910509F479C58B3C910509F447
:1031300096C5883C910511F00C94FF2526C58E3C60
:10314000910509F415C60CF410C6833D910511F0E4
:103150000C94FF250E9427820C94FF258E3251E0AB
:10316000950709F4D8C694F4823E910509F410C677
:103170008D32B1E09B0709F44EC68D3D910511F0EB
:103180000C94FF250E94CB810C94FF258033E1E055
:103190009E0709F443C60CF414C78336914011F01E
:1031A0000C94FF250E9460350C94FF25873F31E089
:1031B000930711F40C940E244CF58C3A51E09507CA
:1031C00011F40C94552384F48239B1E09B0711F477
:1031D0000C94FC2214F40C94F822843A914011F4DB
:1031E0000C9400230C94FF25853F21E0920711F4F5
:1031F0000C94082414F00C940B24843F914011F09B
:103200000C94FF250E9437790C94FF258F3853E0EA
:10321000950711F40C94CB24ACF48A38B3E09B07E7
:1032200011F40C9450248B38E3E09E0711F40C94B5
:1032300092248335934011F00C94FF25E9EBFCE0D8
:103240000C941C24823923E0920711F40C945D2520
:10325000873E33E0930711F40C9494258039934012
:1032600011F00C94FF250C941425009199031091F2
:103270009A0380E50E94CC37882369F00E94C33509
:103280006B017C01BB24B394611571058105910527
:1032900031F4B12C04C0B12CC12CD12C760183E5C2
:1032A0000E94CC37882311F40C9462260E940336C6
:1032B00020E030E04AE754E40E94F3B30E9435B9BD
:1032C0006B017C01B11024C0611571058105910568
:1032D000F9F401151105E1F0D8018C918823C1F0B2
:1032E000E9EBFCE084915F01BFEFAB1ABB0A8823D6
:1032F00021F00E94FD34F501F5CFF80181918F0195
:10330000882319F00E94FD34F8CF8AE00E94FD3432
:1033100081E0809340070E94345E0E94A439C1146A
:10332000D104E104F104F9F0809056039090570322
:10333000A0905803B09059038C0C9D1CAE1CBF1C70
:103340000E94DB38681979098A099B0997FD04C036
:10335000109240070C94FF25809140078823C1F309
:103360000E940872EDCF80914007882389F30E9464
:103370000872F9CF84918F010F5F1F4F882321F0CE
:103380000E94FD34F801F6CFBE016F5F7F4F80E3EE
:1033900092E00E9404358AE00E94FD340C94FF25DF
:1033A00083E50E94CC37882311F40C94FF250E94FA
:1033B000E335E82E80E50E94CC37811110C081E012
:1033C000E11001C080E08093ED05882321F024986E
:1033D0002C9A0C94FF25249A2C980C94FF2580E5B8
:1033E0000E94CC37882341F00E94D33577FF02C07A
:1033F0000C94FF258B0102C00DE010E0802FEDE35F
:10340000F2E09491891739F0319622E0E536F2071F
:10341000C1F70C946726E5EEFAE084918F010F5F07
:103420001F4F882321F00E94FD34F801F6CFE5E616
:10343000F2E084918F010F5F1F4F882311F40C94E9
:10344000FF250E94FD34F801F4CF0E94B07E0C9459
:10345000FF2580912F0F813011F00C94FF2582E021
:1034600080932F0F0E94DB386093380F7093390FD1
:1034700080933A0F90933B0F0C94FF250E947AA5FE
:103480000C94FF250E94DBAA0C94FF2588E690E0AF
:103490000E948B8181110C94FF258091260483FF6B
:1034A00002C00C94FF2583E50E94CC37882311F4D9
:1034B0000C94FF250E9403360E9430B97093D40CFF
:1034C0006093D30C80E00E945B390E94033620E0B9
:1034D00030E040E752E40E948EB3181614F00E94C8
:1034E0007AA50E9403360C94FF258EE40E94CC3707
:1034F000882311F40C94FF250E94D33560935A035E
:1035000070935B0380935C0390935D030C94FF25A1
:1035100083E50E94CC37882321F00E94E335C82E32
:1035200001C0C12CC0922604E9EBFCE084918F011C
:103530000F5F1F4F882321F00E94FD34F801F6CF62
:10354000E2E8F2E084918F010F5F1F4F882321F0A2
:103550000E94FD34F801F6CFCC20A1F1E4E7EE2E75
:10356000E2E0FE2E00E010E020E0D12CC601002EAB
:1035700002C0959587950A94E2F780FF17C09924B9
:103580009394920E222319F08CE20E94FD34F701ED
:1035900025913491F90184915901FFEFAF1ABF0AC7
:1035A000882329F00E94FD349501F4CF922E0F5FFD
:1035B0001F4F22E0E20EF11C0530110509F444C052
:1035C000292DD4CFEEE7F2E084918F010F5F1F4FDA
:1035D0008823D1F10E94FD34F801F6CF8AE50E94DC
:1035E0004237882311F40C9442240E9403366B0165
:1035F0007C0120E030E040E050EC0E9412BA87FFEE
:1036000002C00C94342420E030E040EA50E4C701CA
:10361000B6010E948EB3181614F40C943424C09290
:103620000B04D0920C04E0920D04F0920E04C092B0
:103630002202D0922302E0922402F092250242E07C
:10364000C701B6010E94B3778AE00E94FD340C9452
:10365000FF258091260483FF02C00C94FF2583E59B
:103660000E94CC37882311F40C94FF250E94033666
:103670000E9430B96739710514F066E970E0709303
:10368000D00C6093CF0C0E9412390C94FF2589E670
:1036900090E00E948B8181110C94702AE9E8F2E09D
:1036A00084918F010F5F1F4F882321F00E94FD340A
:1036B000F801F6CF0E9480718AE00E94FD340C94DC
:1036C000702A83E50E94CC37882311F40C94FF25DF
:1036D0000E94E335809362038D3318F08CE380936E
:1036E00062030E94DB386B017C012091620330E0B1
:1036F000A8EEB3E00E94DCB7C60ED71EE81EF91E86
:10370000C0925E03D0925F03E0926003F092610387
:103710000C94FF258DE690E00E948B8181110C9422
:10372000FF258091260483FF02C00C94FF2583E5CA
:103730000E94CC378FA381110C947C2682E50E94D5
:10374000CC3781110C947C260C94FF2580912604A3
:1037500083FF02C00C94FF2583E50E94CC378FA322
:1037600081110C94A92782E50E94CC3781110C9419
:10377000A9270C94FF2583E50E94CC37882339F0D4
:103780000E94D3358B016F3F710519F010F00FEFD8
:1037900010E080E50E94CC37811106C010936403CD
:1037A000009363030C94FF250E94E33581110C9470
:1037B000FF25F4CF80E50E94CC37811106C010921E
:1037C0006403109263030C94FF250E94D335672B8A
:1037D00011F00C94FF25F3CF62E370E080E090E0FD
:1037E0000E9444380E9470A90F5F1F4F03311105DA
:1037F00099F762E370E080E090E00E9444380E9414
:1038000070A90C94FF25109221040C94FF2581E0EF
:10381000809321040C94FF2583E50E94CC378823F4
:10382000A1F00E94033620E030E04AE754E40E9411
:10383000F3B30E9435B960930E0270930F02809328
:103840001002909311020C94FF2588E50E944237E4
:1038500081110C94DA2889E50E94423781110C9479
:10386000DA288AE50E94423781110C94DA2885E42F
:103870000E94423781110C94DA280E94345E0E9423
:10388000AFA70C94FF2583E50E944237882311F4EB
:103890000C94FF250E94033620E030E04AE754E410
:1038A0000E94F3B30E9435B9609365037093660379
:1038B00080936703909368030C94FF253CEEA32E3E
:1038C00032E0B32E09E813E0912CD5018D915D0112
:1038D0000E944237882309F46DC0B3E09B1263C095
:1038E0000E9403366B017C0120E030E040EA51E4A5
:1038F0000E948EB387FF4EC0A70196016091950389
:103900007091960380919703909198030E94C8B894
:103910002B013C019B01AC016091850370918603F2
:1039200080918703909188030E94F3B3609385038D
:10393000709386038093870390938803A301920179
:103940006091BD037091BE038091BF039091C0034D
:103950000E94F3B36093BD037093BE038093BF03D3
:103960009093C00360917503709176038091770303
:10397000909178030E9492B3A30192010E94F3B345
:103980000E9435B960937503709376038093770333
:1039900090937803C0929503D0929603E092970398
:1039A000F092980307C00E940336F8016083718388
:1039B0008283938393940C5F1F4FF4E09F1285CF13
:1039C0000E94115F0C94FF250E94345E0E9466786D
:1039D0000C94FF2584918F010F5F1F4F882321F0E6
:1039E0000E94FD34F801F6CFE1E6F3E084918F0107
:1039F0000F5F1F4F882321F00E94FD34F801F6CF9E
:103A0000EAE4F3E084918F010F5F1F4F882321F0D8
:103A10000E94FD34F801F6CFEAE3F3E084918F01D0
:103A20000F5F1F4F882321F00E94FD34F801F6CF6D
:103A3000E9E2F3E084918F010F5F1F4F882321F0AB
:103A40000E94FD34F801F6CFE8E1F3E084918F01A4
:103A50000F5F1F4F882321F00E94FD34F801F6CF3D
:103A6000E9E0F3E084918F010F5F1F4F882321F07D
:103A70000E94FD34F801F6CFE4EFF2E084918F016B
:103A80000F5F1F4F882321F00E94FD34F801F6CF0D
:103A9000EEEDF2E084918F010F5F1F4F882321F03C
:103AA0000E94FD34F801F6CFE9ECF2E084918F0139
:103AB0000F5F1F4F882321F00E94FD34F801F6CFDD
:103AC000ECEAF2E084918F010F5F1F4F882321F011
:103AD0000E94FD34F801F6CFE4E9F2E084918F0111
:103AE0000F5F1F4F882311F40C94FF250E94FD34B3
:103AF000F801F4CF85E40E944237882381F00E94C8
:103B0000F435882361F0E9EBFCE084918F010F5FCD
:103B10001F4F882321F00E94FD34F801F6CF81E485
:103B20000E944237882381F00E94F435882361F097
:103B3000E5E6F4E084918F010F5F1F4F882321F0A9
:103B40000E94FD34F801F6CF0091990310919A0379
:103B5000D8018D918D01882309F476CD0E94FD3422
:103B6000F7CF81E08093ED0524982C9A0E94E639E6
:103B70001092ED05249A2C980C94FF2581E08093F7
:103B8000E90580939B030C94FF2588EC90E00E944C
:103B90008B8181110C94FF2584E40E944237882395
:103BA000D1F10E94033611E020E030E0A9010E942B
:103BB0008EB3811101C010E01093A003112359F1BD
:103BC0000091EE0310E00E940336F801EE0FFF1F94
:103BD000EE0FFF1FE456FC4F608371838283938353
:103BE00020E030E0A90160919C0370919D038091D9
:103BF0009E0390919F030E948EB381110CC080E0C0
:103C000090E0A0E4B0E480939C0390939D03A09384
:103C10009E03B0939F030E943436F1C70CEE12E06E
:103C200091EAE92E93E0F92EF80181918F010E942B
:103C30004237882351F00E9403360E9435B9D701DC
:103C40006D937D938D939C931397B4E0EB0EF11CD1
:103C5000E2E0003F1E0741F70E949334D0C70CEE0C
:103C600012E081EBE82E83E0F82ED8018D918D01D2
:103C70000E944237882339F00E940336F70160839F
:103C8000718382839383F4E0EF0EF11C22E0003F06
:103C9000120759F7B4C783E50E9442378823D9F049
:103CA0000E940336AB01BC014093C9035093CA0381
:103CB0006093CB037093CC034093C5035093C6032A
:103CC0006093C7037093C80383EC94E00E940A8258
:103CD0008AE00E94FD3480E50E944237882399F0F3
:103CE0000E940336AB01BC014093C9035093CA0341
:103CF0006093CB037093CC0386EA94E00E940A821F
:103D00008AE00E94FD3482E50E944237882399F0C0
:103D10000E940336AB01BC014093C1035093C20320
:103D20006093C3037093C40387E894E00E940A82FF
:103D30008AE00E94FD3484E50E944237882309F41A
:103D40005EC70E940336AB01BC014093C50350938C
:103D5000C6036093C7037093C80389E694E00E948A
:103D60000A828AE00E94FD344AC70E94703747C722
:103D70000E946B6144C783E50E94CC37882309F415
:103D80003EC70E94D335709313026093120237C767
:103D900080E50E944237882309F431C70E94D33559
:103DA000F62E062F172F83E50E94CC37882321F0AB
:103DB0000E94D3356B0103C0CC24CA94DC2C96013D
:103DC0002F5F3F4F2330310508F019C717FD17C784
:103DD0000E94345E3FEFC316D30631F0CA94CD285B
:103DE00071F000E010E00DC08F2D0E947C3831E0B2
:103DF00020E0892B09F030E0032F122F02C001E0F0
:103E000010E08F2D0E947C388017910709F4F7C6C7
:103E10000E940872F6CF0E941187F1C680E50E94C9
:103E20004237882351F00E9403366093E203709377
:103E3000E3038093E4039093E50389E40E9442370F
:103E4000882381F00E9403362CEA35EC47E25EE3DA
:103E50000E94F3B36093DE037093DF038093E0036B
:103E60009093E10384E40E944237882381F00E940A
:103E700003362CEA35EC47E25EE30E94C8B8609353
:103E8000DA037093DB038093DC039093DD03E9EBAB
:103E9000FCE084918F010F5F1F4F882321F00E9467
:103EA000FD34F801F6CF4091E2035091E3036091B5
:103EB000E4037091E50383EF94E00E940A822CEA08
:103EC00035EC47E25EE36091DE037091DF038091A1
:103ED000E0039091E1030E94C8B8AB01BC018FEEF2
:103EE00094E00E94B7822CEA35EC47E25EE36091F1
:103EF000DA037091DB038091DC039091DD030E9473
:103F0000F3B3AB01BC018BEE94E00E94B7828AE070
:103F10000E94FD3474C683E50E944237182F88231F
:103F200071F00E9403360E9430B9709315026093BD
:103F3000140221E0672B09F020E02093CD0380E5F7
:103F40000E944237882369F08091140290911502F3
:103F5000892B19F00E94F43501C081E08093CD03D4
:103F60004EC611114CC6E9EBFCE084918F010F5F46
:103F70001F4F882321F00E94FD34F801F6CF809175
:103F8000CD03882319F062EF72E002C06FE872E09F
:103F90008CE095E00E940435609114027091150246
:103FA0008BEF94E00E941E79E7EFF4E084918F019B
:103FB0000F5F1F4F882309F422C60E94FD34F801C9
:103FC000F5CF85E40E94CC37882321F00E94D335B9
:103FD0001B0102C0212C312C83E40E94CC378823A2
:103FE00039F00E94D33562967FAF6EAF629706C0FC
:103FF00085E090E062969FAF8EAF629785E50E9464
:104000004237882331F00E94F43563968FAF63976F
:1040100003C063961FAE6397E12CF12C37FE03C0FB
:104020000CE812E402C006E113E483E50E94CC37F9
:10403000882321F00E9403367B018C012114310476
:1040400011F41092EE030E94DB382B013C01C101F8
:104050000196029728F4AFE9CA2EA2E0DA2E0BC02F
:1040600002EB12E0D8018D918D01882309F4ECCA8E
:104070000E94FD34F7CFF60181916F01882319F07A
:104080000E94FD34F8CF8AE00E94FD340E9401A610
:104090008FE7FFEF2F163F0619F48093E70C02C05D
:1040A0008093E90CB701C8010E9430B9882777FDD9
:1040B0008095982F0E9494B36BAF7CAF8DAF9EAF6D
:1040C00081E0809347022C964CAE5DAE6EAE7FAE23
:1040D0002C9767964CAE5DAE6EAE7FAE67971FAE07
:1040E00020E421962FAF21973CE122963FAF229703
:1040F00046E423964FAF239724961FAE2497259628
:104100001FAE259726961FAE269727961FAE279798
:104110001FAA18AE19AE1AAE1BAA1CAA1DAA1EAA67
:10412000C12CD12C7601FFE78F2E912CA12CB12C24
:104130008FE790E0A0E0B0E08BA79CA7ADA7BEA75B
:1041400060961CAE1DAE1EAE1FAE609791E0289625
:104150009FAF289718AA1FA610E01F8E1BA200E091
:1041600080914702882309F439C20E94DB386FA38B
:1041700078A789A79AA78091D70C882309F40EC144
:104180000E94E8A7AFEF2A163A0659F41091EA0305
:10419000B091EB03BF8FE091EC03EBA30091ED0333
:1041A0000AC01091E603F091E703FF8F2091E80326
:1041B0002BA30091E903212F3F8D4BA1502F249673
:1041C0006FAD249725967FAD259726968FAD2697C0
:1041D00027969FAD27970E948EB387FF0EC0249627
:1041E0001FAF24973F8D25963FAF25974BA126966D
:1041F0004FAF269727960FAF2797212F3F8D4BA1C3
:10420000502F6FAD21967FAD219722968FAD2297CB
:1042100023969FAD23970E9412BA181664F41FAF1D
:104220005F8D21965FAF21978BA122968FAF22974A
:1042300023960FAF239728969FAD2897992309F4CB
:1042400052C02BAD3CAD4DAD5EAD612F7F8D8BA1CE
:10425000902F0E9412BA18160CF0A0C08FA198A53A
:10426000A9A5BAA584199509A609B709AC01BD018C
:10427000485853416109710977FD90C04BA55CA571
:104280006DA57EA5481959096A097B097595679539
:1042900057954795EFEF2E163E0619F44093E70C1D
:1042A00002C04093E90C60968CAF9DAFAEAFBFAF3C
:1042B0006097FBAD2496FFAF24972CAD25962FAFCA
:1042C00025973DAD26963FAF26974EAD27964FAF2B
:1042D00027978FA198A5A9A5BAA52C968CAF9DAFBD
:1042E000AEAFBFAF2C972BAD3CAD4DAD5EAD612FEA
:1042F0007F8D8BA1902F0E948EB387FD02C00C94FE
:104300005D2A8FA198A5A9A5BAA52C962CAD3DAD87
:104310004EAD5FAD2C97821B930BA40BB50BAC017C
:10432000BD01485853416109710977FF02C00C94DF
:104330005D2A4FA558A9452B09F05EC78BA59CA502
:10434000ADA5BEA5880D991DAA1DBB1DB595A79548
:1043500097958795EFEF2E163E0611F00C94592A8B
:104360008093E70C2FA538A92F5F3F4F38AB2FA7BD
:104370003BAD3FAF4CAD21964FAF21975DAD22963F
:104380005FAF22978EAD23968FAF23974FA058A48F
:1043900069A47AA491E028969FAF289720E030E0A6
:1043A00040EA51E46BAD7CAD8DAD9EAD0E94ECB7A3
:1043B0009B01AC01612F7F8D8BA1902F0E9412BABF
:1043C00018166CF4ECEDF5E084918F010F5F1F4F30
:1043D000882309F414C40E94FD34F801F5CF80E36A
:1043E00098EFAFEFBFEF67962CAD3DAD4EAD5FAD33
:1043F0006797821B930BA40BB50B2FA138A549A57A
:104400005AA5820F931FA41FB51FB7FD0FC00E94AE
:1044100080718AE00E94FD348FA198A5A9A5BAA554
:1044200067968CAF9DAFAEAFBFAF67978FA198A5D2
:10443000A9A5BAA5880F991FAA1FBB1F84199509A2
:10444000A609B7092C962CAD3DAD4EAD5FAD2C97AE
:10445000821B930BA40BB50B81389F44A241B1057D
:1044600068F0EEEBF5E084918F010F5F1F4F88231A
:1044700009F4C5C30E94FD34F801F5CF4FA558A932
:1044800062968EAD9FAD6297841795070CF068CE4B
:10449000E1E6F5E084918F010F5F1F4F882321F043
:1044A0000E94FD34F801F6CF9FEF2916390619F462
:1044B00003E912E002C006E213E0B8018FE495E0E0
:1044C0000E940435B701A6018BE495E00E940A82A0
:1044D0008AE00E94FD34B80189E395E00E9404352A
:1044E0004BA95CA96DA97EA985E395E00E940A828B
:1044F0008AE00E94FD34B80183E295E00E94043511
:104500004FA958AD69AD7AAD8FE195E00E940A825E
:104510008AE00E94FD346396AFAD6397AA2309F445
:104520006EC32320209469F5C092E203D092E30386
:10453000E092E403F092E5032CEA35EC47E25EE317
:104540006BA97CA98DA99EA90E94F3B36093DE0399
:104550007093DF038093E0039093E1032CEA35EC42
:1045600047E25EE36FA978AD89AD9AAD0E94C8B805
:104570006093DA037093DB038093DC039093DD0395
:104580003EC3C092D603D092D703E092D803F092F4
:10459000D9032CEA35EC47E25EE36BA97CA98DA92F
:1045A0009EA90E94F3B36093D2037093D3038093C8
:1045B000D4039093D5032CEA35EC47E25EE36FA970
:1045C00078AD89AD9AAD0E94C8B86093CE03709360
:1045D000CF038093D0039093D10311C380914702FE
:1045E00081110DC30E9401A60AC30E94345E07C355
:1045F00081E00E94215503C380E00E942155FFC243
:1046000086E50E944237882321F08DE796E00E94DC
:10461000277883E50E944237882321F00E94F435F1
:10462000182F01C010E083E50E944237882319F05B
:10463000812F0E9473A6F090EF03111103C0E9EBE4
:10464000FCE01AC0F110FBCFE5EEFAE084918F0197
:104650000F5F1F4F882321F00E94FD34F801F6CF31
:10466000EEE5F6E084918F010F5F1F4F882339F349
:104670000E94FD34F801F6CF84918F010F5F1F4F28
:10468000882321F00E94FD34F801F6CFFF2019F0B5
:1046900067E972E002C06BE972E080E596E00E9493
:1046A00004358AE00E94FD34AAC28EEE882E85E091
:1046B000982E9AEFA92E95E0B92E28E0222E24E01C
:1046C000322E00E010E0E22DE095EF8FD1018D91C8
:1046D0001D01882309F48BC0F50140805180628060
:1046E0007380F801EA5EFD4F208131814281538160
:1046F000F801E450FC4F60817181828193810E94B6
:10470000ECB720E030E040E05FE30E94F3B39B01B0
:10471000AC01C301B2010E9412BA181644F4F801A8
:10472000E656F94FC590D590E590F49003C0C12CA2
:10473000D12C7601F801E051FC4F2081318142817A
:104740005381C301B2010E94EBB79B01AC01C701C9
:10475000B6010E94EBB76B017C0120E030E040EA3B
:1047600051EC0E9412BA87FD29C020E030E040EAF7
:1047700051E4C701B6010E948EB31816FCF0D401B3
:104780002D913D914D915C91C701B6010E94EBB70F
:104790009B01AC01C301B2010E94ECB7F50160833B
:1047A000718382839383D401CD92DD92ED92FC924A
:1047B00013978F8D820D0E94D83619C0E5EEFAE06E
:1047C00084918F010F5F1F4F882321F00E94FD34D9
:1047D000F801F6CFE6EAF6E084918F010F5F1F4FF4
:1047E000882309F40CC20E94FD34F801F5CFB4E02F
:1047F0008B0E911C0C5F1F4FE4E0AE0EB11C0C3011
:10480000110509F063CF0E941B610E946678F7C111
:104810000E949B58F4C10E94A35FF1C183E50E94EE
:104820004237882319F00E94F43501C081E091E0FD
:1048300089270E94D482E3C184918F010F5F1F4FAB
:10484000882321F00E94FD34F801F6CFECEDF6E06C
:1048500084918F010F5F1F4F882311F40C94EE1A7F
:104860000E94FD34F801F4CFE7ECF6E084918F016B
:104870000F5F1F4F882311F40C94241B0E94FD34FA
:10488000F801F4CF40910B0450910C0460910D0499
:1048900070910E0484EC96E00E940A820C94241B12
:1048A0000CEE12E09E012F5F3F4F7901D8018D91F0
:1048B0008D010E94CC37882319F00E94D33502C0A5
:1048C00060E070E0F701619371937F01F2E0003FD7
:1048D0001F0761F749815A8168E580E79EE041152D
:1048E000510519F00E94B37502C00E94E6814B8108
:1048F0005C8169E58BEF9DE04115510519F00E943F
:10490000B37502C00E94E6814D815E816AE586E84A
:104910009DE04115510519F00E94B37570C10E94C8
:10492000E6816DC188E50E9442378823F1F00E943C
:10493000D3358B01222717FD2095322F00930F04CA
:10494000109310042093110430931204DB012FEF15
:1049500030E00E94E1BA20ED37E040E050E00E94F4
:10496000B6B7B9018EE20E941F4B8AE50E9442371A
:10497000882329F00E94D33581E00E9421A685E496
:104980000E944237882309F43AC10E94D33582E05D
:104990000E9421A634C188E50E944237182F89E57C
:1049A0000E944237E82E8AE50E944237F82E85E4BD
:1049B0000E944237082F111108C0E11018C0F110F1
:1049C00022C0811185C511E007C0EE2021F0FF2033
:1049D00011F0182F01C010E068E580E79EE00E940A
:1049E000ED51E11005C0112309F46CC501C010E0C0
:1049F00069E58BEF9DE00E94ED51F11005C0112398
:104A000009F466C501C010E06AE586E89DE00E94F1
:104A1000ED51002331F065E481E19DE00E94ED510C
:104A2000EEC01111F8CFEBC088E50E944237182F75
:104A300089E50E944237E82E8AE50E944237F82E27
:104A400085E40E944237082F111108C0E11018C0F8
:104A5000F11022C0811140C511E007C0EE2021F005
:104A6000FF2011F0182F01C010E068E580E79EE0FC
:104A70000E94D851E11005C0112309F426C501C0D8
:104A800010E069E58BEF9DE00E94D851F11005C060
:104A9000112309F421C501C010E06AE586E89DE014
:104AA0000E94D851002331F065E481E19DE00E942D
:104AB000D851A5C01111F8CFA2C088E50E94423795
:104AC000882331F00E94D33580E79EE00E949C4D00
:104AD00068E580E79EE00E948D7E89E50E9442376E
:104AE000882331F00E94D3358BEF9DE00E949C4DCE
:104AF00069E58BEF9DE00E948D7E85E40E94423740
:104B0000882361F00E94D33581E19DE00E949C4D95
:104B100065E481E19DE00E948D7E71C065E481E1E4
:104B20009DE00E948D7E6BC081E08093260283E52C
:104B30000E944237811103C00E9445A760C00E94B5
:104B4000F43581115CC0F8CFF0902304FF2029F1E7
:104B5000E9EBFCE084918F010F5F1F4F882321F068
:104B60000E94FD34F801F6CF84E50E94FD346F2DDC
:104B700070E080E090E04AE00E94007780E20E94CE
:104B8000FD340BED12E0D8018D918D01882311F4D5
:104B90000C94241B0E94FD34F6CF10921B04E9EB09
:104BA000FCE084918F010F5F1F4F882321F00E944A
:104BB000FD34F801F6CF60E070E086EE96E00E94EA
:104BC0001E798AE00E94FD341AC0E9EBFCE0849172
:104BD0008F010F5F1F4F882321F00E94FD34F801E1
:104BE000F6CF60911C0470911D0488EF96E00E943E
:104BF000043582E20E94FD348AE00E94FD340E9466
:104C0000D7A66EC44115510519F4AF0141505109A1
:104C100020E030E00C94FE1180E00E9473A60E9418
:104C2000C73983E50E944237882309F449C00E94AE
:104C3000F43521E0482FBE016F5F7F4FCE014696CD
:104C40000E94FD556B017C019B01AC010E9498BA4A
:104C5000811131C02CEA35EC47E257E36E897F8938
:104C6000888D998D0E94ECB7AB01BC0188E292E07F
:104C70000E94B7822CEA35EC47E257E369817A81DA
:104C80008B819C810E94ECB7AB01BC0183E292E076
:104C90000E94B7822CEA35EC47E257E3C701B60120
:104CA0000E94ECB7AB01BC018EE192E00E94B7829A
:104CB0008AE00E94FD340E94AE390E9466789FCF40
:104CC00081E0B7CFB1100C9488190C946919802F2A
:104CD0000E94004B6E2D802F0E94A538F12CB70149
:104CE000802F0E941F4B0830110509F088CFF092E9
:104CF0006403E092630383CF0E9403360E9430B9BD
:104D00007093D40C6093D30C80E00E945B390E94B6
:104D1000033620E030E040E752E40E948EB31816DC
:104D20001CF00E947AA502C00E94B07E81E08093B0
:104D300047021BA21CA21DA21EA21BA61CA61DA6EA
:104D40001EA61F8E1FA63CE33BAB4CE14FAB56E4C7
:104D50005BAFC12CD12C60E8E62E7FEBF72E812CC7
:104D6000912C54016091D30C7091D40C882777FD5D
:104D70008095982F0E9494B3162F072F782E692EB6
:104D8000262F372F482F592FB601C7010E948EB307
:104D90008823D9F02091E6033091E7034091E8039E
:104DA0005091E903612F702F872D962D0E948EB3AD
:104DB000881F8827881F8F8F8FA1882351F09F8D90
:104DC000992339F0809147021ACF1C2D0D2D7E2C8E
:104DD0006F2C0E94DB386B017C01DC01CB012BA521
:104DE0003CA54DA55EA5821B930BA40BB50BB7FD8F
:104DF00039C0D701C60188519C4FAF4FBF4F8BA719
:104E00009CA7ADA7BEA70E948071ECE8F2E0849158
:104E10002F019FEF491A590A882321F00E94FD347F
:104E2000F201F5CF81149104A104B104A9F0C501E8
:104E3000B40168517C4F8F4F9F4F6C197D098E09CB
:104E40009F0928EE33E040E050E00E9494B7CA0189
:104E5000B9010E948D7703C08FE30E94FD348AE080
:104E60000E94FD340E9408720E94A4392090E6033B
:104E70003090E7034090E8035090E9039101A201CC
:104E8000612F702F872D962D0E94EBB79F7720E022
:104E900030E040E251E481149104A104B10429F40A
:104EA0000E948EB387FD05C006C00E9412BA181674
:104EB00014F446015701AF8DAA2379F12BA13CA12F
:104EC0004DA15EA1211531054105510541F0D701E4
:104ED000C601821B930BA40BB50BB7FD1EC091013D
:104EE000A2016FA57BA98FA99BAD0E94EBB720E023
:104EF00030E040EC5FE30E948EB387FD63CFD701C3
:104F0000C601805A9541AF4FBF4F8BA39CA3ADA361
:104F1000BEA32FA63BAA4FAA5BAE8091470288236F
:104F200009F450CF81149104A104B10429F4C12ED5
:104F3000D02EE72CF62C16CF98EEC91A93E0D90A9A
:104F4000E108F108C818D908EA08FB08F7FE3ACFCB
:104F5000EECF0E9403360E9430B96739710514F014
:104F600066E970E07093D00C6093CF0C0E94123908
:104F70000E94033620E030E040EA50E40E9412BA7A
:104F8000181614F40E94B07E81E08093470280914D
:104F90001B048093EE031BA21CA21DA21EA21BA633
:104FA0001CA61DA61EA61F8E1FA6ACE3ABABBCE1C4
:104FB000BFABE6E4EBAFC12CD12C40E8E42E5FEBB5
:104FC000F52E812C912C54016091CF0C7091D00C56
:104FD000882777FD8095982F0E9494B3162F072F6E
:104FE000782E692E262F372F482F592FB601C7014B
:104FF0000E948EB38823D1F02091EA033091EB0315
:105000004091EC035091ED03612F702F872D962D69
:105010000E948EB3881F8827881F8F8FFFA1FF23D0
:1050200049F0882339F080914702E9CD1C2D0D2DE0
:105030007E2C6F2C0E94DB386B017C01DC01CB01E4
:105040002BA53CA54DA55EA5821B930BA40BB50B10
:10505000B7FD39C0D701C60188519C4FAF4FBF4F34
:105060008BA79CA7ADA7BEA70E948071E0E9F2E0E4
:1050700084912F019FEF491A590A882321F00E9439
:10508000FD34F201F5CF81149104A104B104A9F01B
:10509000C501B40168517C4F8F4F9F4F6C197D093A
:1050A0008E099F0928EE33E040E050E00E9494B75B
:1050B000CA01B9010E948D7703C08FE30E94FD34BD
:1050C0008AE00E94FD340E9408720E94A439209058
:1050D000EA033090EB034090EC035090ED03910114
:1050E000A201612F702F872D962D0E94EBB79F771D
:1050F00020E030E040EA50E481149104A104B104BE
:1051000029F40E948EB387FD05C006C00E9412BA22
:10511000181614F446015701AF8DAA2379F12BA17B
:105120003CA14DA15EA1211531054105510541F07C
:10513000D701C601821B930BA40BB50BB7FD1EC094
:105140009101A2016FA57BA98FA99BAD0E94EBB72E
:1051500020E030E040EC5FE30E948EB387FD63CF38
:10516000D701C601805A9541AF4FBF4F8BA39CA377
:10517000ADA3BEA32FA63BAA4FAA5BAE8091470268
:10518000882309F450CF81149104A104B10429F4B7
:10519000C12ED02EE72CF62C17CF98EEC91A93E02B
:1051A000D90AE108F108C818D908EA08FB08F7FE8F
:1051B0003ACFEECF0E94345E88E50E9442378823C2
:1051C00019F0179A1092EA0589E50E944237882360
:1051D00019F0169A1092EB058AE50E94423788234F
:1051E00019F0159A1092EC0585E40E944237882345
:1051F00009F405CD149A03CD60964CAC5DAC6EAC51
:105200007FAC6097480E591E6A1E7B1E60962CADBF
:105210003DAD4EAD5FAD6097281B390B4A0B5B0B64
:10522000CA01B901A50194010E9485B7A3019201A9
:105230000E94B6B749015A018BA59CA5ADA5BEA594
:10524000880E991EAA1EBB1E94E189169104A10422
:10525000B1040CF1ACEE8A169104A104B1043CF443
:10526000B0E88B169104A104B1041CF105C06BEEEB
:10527000862E912CA12CB12C8BA69CA6ADA6BEA6E9
:105280002EEF30E040E050E0281939094A095B0967
:1052900049015A0112C084E190E0A0E0B0E08BA780
:1052A0009CA7ADA7BEA754E1852E912CA12CB12CB3
:1052B00004C08BA69CA6ADA6BEA6E8E4F6E0849149
:1052C0009F012F5F3F4F882381F068962FAF68972B
:1052D00069963FAF69970E94FD3468962FAD689735
:1052E00069963FAD6997F901EACF6BA57CA58DA5BD
:1052F0009EA50E948D77E3E4F6E084919F012F5FE5
:105300003F4F882381F068962FAF689769963FAF2B
:1053100069970E94FD3468962FAD689769963FADF6
:105320006997F901EACFC501B4010E948D774FADAD
:1053300021965FAD219722966FAD229723967FAD80
:1053400023978CE396E00E940A8224964FAD24971F
:1053500025965FAD259726966FAD269727967FAD4C
:10536000279785E396E00E940A82AFA5B8A9139714
:1053700014F40C949E21C501B4010E9494B320E062
:1053800030E040E850E40E94F3B36B017C012FADA4
:1053900021963FAD219722964FAD229723965FAD80
:1053A000239724966FAD249725967FAD2597269653
:1053B0008FAD269727969FAD27970E94EBB72BEDD1
:1053C0003FE049E450E40E94F3B320E030E040E0E5
:1053D0005FE30E94F3B39B01AC01C701B6010E94D9
:1053E000C8B86B017C01C301B2010E9494B32FE6DF
:1053F00032E143E85AE30E94F3B32B013C01B701C9
:10540000A6018FE296E00E940A82B301A20189E21E
:1054100096E00E940A822AE939E949E15FE3C7017F
:10542000B6010E94F3B36B017C019B01AC010E94A9
:10543000ECB7A30192010E94C8B86BAB7CAB8DABFB
:105440009EABA3019201C701B6010E94F3B320E015
:1054500030E040E05EE30E94F3B36FAB78AF89AF1A
:105460009AAFE9E1F6E084913F01BFEF6B1A7B0A46
:10547000882321F00E94FD34F301F5CFB701A60186
:1054800083E196E00E940A824BA95CA96DA97EA9DE
:105490008DE096E00E940A824FA958AD69AD7AADC1
:1054A00087E096E00E940A828AE00E94FD340C9414
:1054B0009E218093E90C0C94B22128961FAE289768
:1054C0000C94CE21FF2021F09FCAFF2029F0E5CACD
:1054D000002309F494CB9FCA002309F490CBE4CABB
:1054E000C75ADF4F0FB6F894DEBF0FBECDBFDF91B6
:1054F000CF911F910F91FF90EF90DF90CF90BF90D1
:10550000AF909F908F907F906F905F904F903F9063
:105510002F90089524E08202C0011124FC01EC5672
:10552000F34F4081518162817381FC01E55BF94F4A
:105530004083518362837383E091C70CF091C80C60
:1055400082899389A489B5898093A40C9093A50C32
:10555000A093A60CB093A70C0895CF93DF932FB719
:10556000F89494E08902E0011124FE01EC56F34F17
:1055700060817181828193812FBF0E9494B3C55C49
:10558000D94F288139814A815B810E94F3B3DF9131
:10559000CF910895089590E0FC013197E231F10533
:1055A00008F04CC0EE58FF4F0C94DBBA809180009D
:1055B0008F7703C0809180008F7D80938000089555
:1055C00080918000877FF9CF84B58F7702C084B542
:1055D0008F7D84BD08958091B0008F7703C0809146
:1055E000B0008F7D8093B0000895809190008F77F8
:1055F00007C0809190008F7D03C080919000877FCD
:105600008093900008958091A0008F7707C08091CB
:10561000A0008F7D03C08091A000877F8093A000B1
:105620000895809120018F7707C0809120018F7DA0
:1056300003C080912001877F8093200108953FB7A8
:10564000F8948091570F9091580FA091590FB091F5
:105650005A0F26B5A89B05C02F3F19F00196A11D32
:10566000B11D3FBF6627782F892F9A2F620F711DBA
:10567000811D911D42E0660F771F881F991F4A9573
:10568000D1F708958EBD00000DB407FEFDCF8EB595
:1056900008950F931F93CF93DF93E091C70CF09180
:1056A000C80C82819381A481B581181619061A0647
:1056B0001B06E4F48091C60C80FF18C082B3909161
:1056C000E205869541E08427282F21709E7F292BB3
:1056D0002093E2058091E1058170822339F0809169
:1056E000570681608093570680E014DFE091C70C75
:1056F000F091C80C86819781A085B185181619068E
:105700001A061B062CF58091C60C81FD21C08091E4
:1057100006012091E20530E0992787FD909580955C
:105720009095990F880B982F82279327807299273D
:10573000822793278093E2059091E1059072982348
:1057400039F08091570680628093570681E0E2DE4F
:10575000E091C70CF091C80C82859385A485B5852E
:10576000181619061A061B060CF045C09091C60CB7
:105770008091E20592FF21C09091ED059923D9F126
:1057800023B190E022952F7031E02327022F017082
:1057900010E01195019511090827192704701127A8
:1057A000082719270093E2058091E1058470802382
:1057B00011F18091570684601AC020B190E02695BF
:1057C0002170C22F20E0D22FD195C195D109C827D1
:1057D000D927C074DD27C827D927C093E205809157
:1057E000E10580748C2339F08091570680648093A2
:1057F000570682E08FDE8091E2058093E105DF911C
:10580000CF911F910F9108954F925F926F927F9267
:105810008F929F92AF92BF92CF92DF92EF92FF92C0
:105820000F931F93CF93DF9300D01F92CDB7DEB7B6
:105830008C01DC014D905D906D907C9013971496D7
:105840008D909D90AD90BC90179718968D919D91DD
:105850000D90BC91A02D89839A83AB83BC83A30157
:105860009201C301B2010E94F3B36B017C01A50157
:105870009401C501B4010E94F3B39B01AC01C701BF
:10588000B6010E94ECB76B017C0129813A814B8102
:105890005C81CA01B9010E94F3B39B01AC01C7014D
:1058A000B6010E94ECB70E9457BA9B01AC0160E0C0
:1058B00070E080E89FE30E94C8B86B017C019B0107
:1058C000AC01C301B2010E94F3B3F801608371839C
:1058D00082839383A7019601C501B4010E94F3B3AB
:1058E000D80114966D937D938D939C931797A70180
:1058F000960169817A818B819C810E94F3B3F801C2
:1059000060877187828793870F900F900F900F9019
:10591000DF91CF911F910F91FF90EF90DF90CF908B
:10592000BF90AF909F908F907F906F905F904F90BF
:1059300008954F925F926F927F928F929F92AF9253
:10594000BF92CF92DF92EF92FF92CF93DF93CDB7CA
:10595000DEB728970FB6F894DEBF0FBECDBF2496F2
:10596000AEADBFAD24978D919D910D90BC91A02DB2
:1059700089839A83AB83BC832296EEADFFAD2297D9
:10598000C080D180E280F380AEADBFAD8D909D90A0
:10599000AD90BC902E8D3F8D48A159A1C501B40199
:1059A0000E94F3B32B013C012AA53BA54CA55DA5A4
:1059B000C701B6010E94F3B39B01AC01C301B20160
:1059C0000E94ECB72B013C012EA93FA948AD59AD6F
:1059D00069817A818B819C810E94F3B39B01AC0128
:1059E000C301B2010E94ECB76D837E838F839887D9
:1059F0002AA13BA14CA15DA1C501B4010E94F3B352
:105A00002B013C012EA53FA548A959A9C701B60104
:105A10000E94F3B39B01AC01C301B2010E94ECB739
:105A20002B013C012AAD3BAD4CAD5DAD69817A8166
:105A30008B819C810E94F3B39B01AC01C301B20135
:105A40000E94ECB72B013C012A8D3B8D4C8D5D8D66
:105A5000C501B4010E94F3B34B015C012EA13FA12B
:105A600048A559A5C701B6010E94F3B39B01AC013B
:105A7000C501B4010E94ECB76B017C012AA93BA9C6
:105A80004CA95DA969817A818B819C810E94F3B3C5
:105A90009B01AC01C701B6010E94ECB7EEADFFADB2
:105AA00060837183828393838D819E81AF81B8856A
:105AB0002296EEADFFAD229780839183A283B383BC
:105AC0002496AEADBFAD24974D925D926D927C92BF
:105AD000139728960FB6F894DEBF0FBECDBFDF91A7
:105AE000CF91FF90EF90DF90CF90BF90AF909F90BD
:105AF0008F907F906F905F904F9008954F925F923C
:105B00006F927F928F929F92AF92BF92CF92DF92CD
:105B1000EF92FF920F931F93CF93DF93CDB7DEB732
:105B2000C454D1090FB6F894DEBF0FBECDBF8C01AF
:105B30008091EF03882309F43AC1C090E90ED09018
:105B4000EA0EE090EB0EF090EC0E2091ED0E30910D
:105B5000EE0E4091EF0E5091F00E29AB3AAB4BABED
:105B60005CAB4090F10E5090F20E6090F30E70908E
:105B7000F40E8091F50E9091F60EA091F70EB09173
:105B8000F80E25968CAF9DAFAEAFBFAF2597209195
:105B9000F90E3091FA0E4091FB0E5091FC0E2DAB98
:105BA0003EAB4FAB58AF8090FD0E9090FE0EA09094
:105BB000FF0EB090000F4091010F5091020F6091C5
:105BC000030F7091040F8091050F9091060FA09123
:105BD000070FB091080F89AF9AAFABAFBCAF809100
:105BE000E50E9091E60EA091E70EB091E80E898344
:105BF0009A83AB83BC834D825E826F82788689866E
:105C00009A86AB86BC86CD86DE86EF86F88A259698
:105C10008CAD9DADAEADBFAD2597898B9A8BAB8B0F
:105C2000BC8B4D8B5E8B6F8B788F29A93AA94BA9C2
:105C30005CA9298F3A8F4B8F5C8F8DA99EA9AFA944
:105C4000B8AD8D8F9E8FAF8FB8A329AD3AAD4BAD58
:105C50005CAD29A33AA34BA35CA32091F003309140
:105C6000F1034091F2035091F303D8016D917D91BE
:105C70008D919C910E94EBB76DA77EA78FA798ABE3
:105C80002091F4033091F5034091F6035091F7030E
:105C9000F80164817581868197810E94EBB720E0CD
:105CA00030E04FE353E40E94EBB769A77AA78BA7D4
:105CB0009CA72091F8033091F9034091FA03509189
:105CC000FB03D80118966D917D918D919C911B9746
:105CD0000E94EBB76DA37EA38FA398A7CE018596F4
:105CE0009F938F9304969F938F9304969F938F9384
:105CF000EDB7FEB7B4970FB6F894FEBF0FBEEDBF79
:105D0000ADB7BEB7119684E2FE01319601900D92B7
:105D10008A95E1F70EDE20E030E0A9016DA57EA5B1
:105D20008FA598A90E94ECB72091F0033091F10360
:105D30004091F2035091F3030E94ECB7D8016D93A8
:105D40007D938D939C93139720E030E04FE353E4D1
:105D500069A57AA58BA59CA50E94ECB72091F403B8
:105D60003091F5034091F6035091F7030E94ECB790
:105D7000F80164837583868397832091F8033091BB
:105D8000F9034091FA035091FB036DA17EA18FA10D
:105D900098A50E94ECB7D80118966D937D938D93CA
:105DA0009C931B970FB6F894DEBF0FBECDBFCC5BA4
:105DB000DF4F0FB6F894DEBF0FBECDBFDF91CF919E
:105DC0001F910F91FF90EF90DF90CF90BF90AF9019
:105DD0009F908F907F906F905F904F900895CF929B
:105DE000DF92EF92FF920F931F93CF93DF93CDB784
:105DF000DEB72C970FB6F894DEBF0FBECDBF6C0197
:105E00007B018A018091EF03882309F4A5C02091CA
:105E1000F0033091F1034091F2035091F303F60146
:105E200060817181828193810E94EBB769877A8753
:105E30008B879C872091F4033091F5034091F60302
:105E40005091F703F70160817181828193810E94F3
:105E5000EBB720E030E04FE353E40E94EBB76D83F3
:105E60007E838F8398872091F8033091F9034091C6
:105E7000FA035091FB03F801608171818281938163
:105E80000E94EBB769837A838B839C83CE01019652
:105E90009F938F9304969F938F9304969F938F93D2
:105EA0008DB79EB784970FB6F8949EBF0FBE8DBF77
:105EB000ADB7BEB7119684E2E5EEFEE001900D921B
:105EC0008A95E1F736DD20E030E0A90169857A8521
:105ED0008B859C850E94ECB72091F0033091F103F3
:105EE0004091F2035091F3030E94ECB7F6016083F6
:105EF00071838283938320E030E04FE353E46D812C
:105F00007E818F8198850E94ECB72091F4033091B7
:105F1000F5034091F6035091F7030E94ECB7F701A7
:105F200060837183828393832091F8033091F90316
:105F30004091FA035091FB0369817A818B819C81A6
:105F40000E94ECB7F80160837183828393830FB65C
:105F5000F894DEBF0FBECDBF2C960FB6F894DEBF0F
:105F60000FBECDBFDF91CF911F910F91FF90EF90AA
:105F7000DF90CF9008954F925F926F927F928F92B1
:105F80009F92AF92BF92CF92DF92EF92FF920F93C8
:105F90001F93CF93DF932C0121EF37E081E090E056
:105FA000F90145915491441655060CF062C0AC01BC
:105FB00041505109DA01AA0FBB1FAA0FBB1FA15103
:105FC000B84FFD0165917491440F551F440F551F43
:105FD0004351584FFA0165907490FC01EE0FFF1F7A
:105FE000EE0FFF1FE151F84FA590B490FD01059110
:105FF0001491F901C591D491FA0185909490882764
:1060000077FD8095982F0E9494B36B017C01B201BB
:1060100066197709882777FD8095982F0E9494B399
:106020002B013C01B501601B710B882777FD809522
:10603000982F0E9494B39B01AC01C301B2010E944E
:10604000F3B32B013C01BE0168197909882777FD5C
:106050008095982F0E9494B39B01AC01C301B201BB
:106060000E94C8B89B01AC01C701B6010E94ECB701
:1060700011C001962C5F3F4F8A33910509F090CFF4
:10608000E3EDF8E065917491882777FD8095982F6E
:106090000E9494B3DF91CF911F910F91FF90EF90E9
:1060A000DF90CF90BF90AF909F908F907F906F9038
:1060B0005F904F9008954F925F926F927F928F9270
:1060C0009F92AF92BF92CF92DF92EF92FF92CF93C7
:1060D000DF93CDB7DEB72C970FB6F894DEBF0FBEB7
:1060E000CDBF8091EA039091EB03A091EC03B091B6
:1060F000ED0389839A83AB83BC836091CF0C70914D
:10610000D00C882777FD8095982F0E9494B3298121
:106110003A814B815C810E94EBB76B017C016093FB
:10612000DD057093DE058093DF059093E0052091F7
:10613000E2033091E3034091E4035091E5030E94B0
:10614000F3B36D837E838F8398876093D9057093B3
:10615000DA058093DB059093DC052091D50530911D
:10616000D6054091D7055091D805C701B6010E94C8
:10617000ECB74B015C016093D5057093D605809315
:10618000D7059093D8052091DE033091DF0340912D
:10619000E0035091E1030E94F3B369877A878B870C
:1061A0009C876093D1057093D2058093D30590931B
:1061B000D40520ED3CEC4CE45DE36091DA03709192
:1061C000DB038091DC039091DD030E94F3B32B018C
:1061D0003C012091CD053091CE054091CF055091E5
:1061E000D00569817A818B819C810E94EBB79B01EC
:1061F000AC01C301B2010E94F3B32B013C0123E3C4
:1062000033E343E75FE36091C9057091CA0580916C
:10621000CB059091CC050E94F3B39B01AC01C30167
:10622000B2010E94ECB72B013C016093C905709349
:10623000CA058093CB059093CC0589819A81AB8167
:10624000BC818093CD059093CE05A093CF05B093EC
:10625000D00529853A854B855C856D817E818F814E
:1062600098850E94ECB7A30192010E94EBB72B0125
:106270003C0120E030E04FE753E40E9412BA20E0F6
:1062800030E0A9011816ACF4C701B6010E9412BA99
:1062900018166CF5A7019601C501B4010E94EBB771
:1062A0006093D5057093D6058093D7059093D80554
:1062B0001EC0C301B2010E948EB387FF22C020E03E
:1062C00030E0A901C701B6010E948EB387FF16C056
:1062D000A7019601C501B4010E94EBB76093D505F3
:1062E0007093D6058093D7059093D80507C0412CAD
:1062F000512C8FE7682E83E4782E03C0412C512C5B
:106300003201C301B2012C960FB6F894DEBF0FBE66
:10631000CDBFDF91CF91FF90EF90DF90CF90BF90F6
:10632000AF909F908F907F906F905F904F90089567
:106330004F925F926F927F928F929F92AF92BF9295
:10634000CF92DF92EF92FF920F931F93CF93DF9341
:1063500000D01F92CDB7DEB70091D30C1091D40CB2
:106360008090E6039090E703A090E803B090E903E3
:10637000B801882777FD8095982F0E9494B3A501D6
:1063800094010E94EBB76B017C016093C50570938B
:10639000C6058093C7059093C80520ED3CEC4CE4FE
:1063A0005DE36091CE037091CF038091D003909113
:1063B000D1030E94F3B32B013C012091C105309120
:1063C000C2054091C3055091C405C501B4010E94A6
:1063D000EBB79B01AC01C301B2010E94F3B32B01E7
:1063E0003C0123E333E343E75FE36091BD05709134
:1063F000BE058091BF059091C0050E94F3B39B013B
:10640000AC01C301B2010E94ECB769837A838B832C
:106410009C836093BD057093BE058093BF059093E8
:10642000C0058092C1059092C205A092C305B092AA
:10643000C40520E030E040E251E4C701B6010E940B
:1064400012BA181624F481E08093BC0589C020E0BC
:1064500030E040E251ECC701B6010E948EB387FDE7
:1064600002C0012B21F481E08093BC059DC0809186
:10647000BC05882351F01092B8051092B90510920E
:10648000BA051092BB051092BC052091D60330913D
:10649000D7034091D8035091D903C701B6010E9498
:1064A000F3B32B013C016093B4057093B505809361
:1064B000B6059093B7052091B8053091B905409184
:1064C000BA055091BB05C701B6010E94ECB74B015C
:1064D0005C016093B8057093B9058093BA059093F9
:1064E000BB052091D2033091D3034091D403509146
:1064F000D5030E94F3B39B01AC016093B005709388
:10650000B1058093B2059093B305C301B2010E9417
:10651000ECB729813A814B815C810E94EBB72B015A
:106520003C0120E030E04FE753E40E9412BA20E043
:1065300030E0A9011816DCF4C701B6010E9412BAB6
:10654000181674F4A7019601C501B4010E94EBB7B7
:106550006093B8057093B9058093BA059093BB0515
:10656000412C512C9FE7692E93E4792E20C0C30162
:10657000B2010E948EB387FF1AC020E030E0A9016B
:10658000C701B6010E948EB387FF0EC0A701960116
:10659000C501B4010E94EBB76093B8057093B905CB
:1065A0008093BA059093BB05412C512C3201C30155
:1065B000B2010F900F900F900F90DF91CF911F912C
:1065C0000F91FF90EF90DF90CF90BF90AF909F9092
:1065D0008F907F906F905F904F9008956091EA0345
:1065E0007091EB038091EC039091ED0308954F922D
:1065F0005F926F927F928F929F92AF92BF92CF9253
:10660000DF92EF92FF920F931F93CF93DF932C01B2
:106610002FE037E081E090E0F90145915491441674
:1066200055060CF062C0AC0141505109DA01AA0FC5
:10663000BB1FAA0FBB1FA35FB84FFD0165917491EB
:10664000440F551F440F551F455F584FFA01659081
:106650007490FC01EE0FFF1FEE0FFF1FE35FF84F7A
:10666000A590B490FD0105911491F901C591D491C3
:10667000FA0185909490882777FD8095982F0E9445
:1066800094B36B017C01B20166197709882777FD05
:106690008095982F0E9494B32B013C01B501601B9B
:1066A000710B882777FD8095982F0E9494B39B01EA
:1066B000AC01C301B2010E94F3B32B013C01BE0146
:1066C00068197909882777FD8095982F0E9494B3DF
:1066D0009B01AC01C301B2010E94C8B89B01AC018F
:1066E000C701B6010E94ECB711C001962C5F3F4F65
:1066F0008032910509F090CFE9E8F7E06591749157
:10670000882777FD8095982F0E9494B3DF91CF91D1
:106710001F910F91FF90EF90DF90CF90BF90AF90BF
:106720009F908F907F906F905F904F9008956091B1
:10673000E6037091E7038091E8039091E9030895DF
:1067400080E00E94AD2A60933407709335078093F0
:1067500036079093370781E00E94AD2A609338078F
:106760007093390780933A0790933B0782E00E9429
:10677000AD2A60933C0770933D0780933E0790934A
:106780003F0708958091C60C9FB780FF09C0F89419
:1067900080910B018E7F80930B019FBF8FEF08C00C
:1067A000F89480910B01816080930B019FBF81E081
:1067B000809348028091C60C9FB781FF09C0F8946E
:1067C00080910B01826080930B019FBF8FEF08C007
:1067D000F89480910B018D7F80930B019FBF81E026
:1067E000809349028091C60C9FB782FF09C0F8943C
:1067F00080910B018B7F80930B019FBF8FEF08C0AF
:10680000F89480910B01846080930B019FBF81E01D
:1068100080934A028091C60C9FB783FF09C0F89409
:1068200080910B01806480930B019FBF8FEF08C0A4
:10683000F89480910B018F7B80930B019FBF81E0C7
:1068400080934B0208954F925F926F927F92AF9226
:10685000BF92CF92DF92EF92FF920F931F93CF934D
:10686000DF938C01EB01FC0147A050A461A472A44A
:10687000AFA0B8A4C9A4DAA49501A601C301B201CE
:106880000E948EB387FF40C0A3019201C301B201F1
:106890000E94F3B32B013C01F80183A994A9A5A997
:1068A000B6A9BC01CD0190589B01AC010E94ECB788
:1068B000F80127A530A941A952A90E94F3B39B0171
:1068C000AC01C301B2010E94EBB70E9457BA7B0131
:1068D0008C019B01AC01B501C6010E948EB387FFFC
:1068E00002C0750186019701A801B501C6010E9489
:1068F0008EB3882349F0A701B8014FA358A769A711
:106900007AA7888181608883DF91CF911F910F9151
:10691000FF90EF90DF90CF90BF90AF907F906F90FF
:106920005F904F9008958F929F92AF92BF92CF92B7
:10693000DF92EF92FF920F931F93CF93DF9300D0DC
:106940001F92CDB7DEB711EA812E13E0912E09E830
:10695000A02E03E0B02E09E613E0C12CD12C760165
:10696000C394F40161917191819191914F01F5016D
:1069700021913191419151915F0129833A834B8358
:106980005C830E9492B329813A814B815C810E9491
:10699000F3B30E9435B9F801619371938193919398
:1069A0008F01C616D706E806F90610F46B017C01C4
:1069B000F1EB8F16F3E09F06A1F66FEF7FEFCB01AF
:1069C000A70196010E9494B7209378063093790628
:1069D00040937A0650937B060F900F900F900F9084
:1069E000DF91CF911F910F91FF90EF90DF90CF90AB
:1069F000BF90AF909F908F9008959091C00095FFA9
:106A0000FCCF8093C60008950F931F93CF93DF931D
:106A10001F921F92CDB7DEB7FC0184918F010F5FEB
:106A20001F4F811102C08B0107C069837A83E5DFA4
:106A3000F80169817A81F1CFD8018D918D01882388
:106A400011F0DBDFF9CF0F900F90DF91CF911F9105
:106A50000F910895EF92FF921F93CF93DF931F92B0
:106A6000CDB7DEB7182FE5EEF7E084917F012FEF69
:106A7000E21AF20A882329F09983BFDFF70199818E
:106A8000F4CFE12FF92F84917F019FEFE91AF90AE2
:106A9000882319F0B2DFF701F6CFECECF7E0849130
:106AA0007F01AFEFEA1AFA0A882319F0A6DFF7018F
:106AB000F6CF0F90DF91CF911F91FF90EF90089547
:106AC000CF93DF93E5EEFAE08491EF0121968823DE
:106AD00019F093DFFE01F8CFEDEBF7E08491EF01C1
:106AE0002196882319F089DFFE01F8CFDF91CF913D
:106AF00008953FB7F8942091C3078091C207821789
:106B000059F0E22FF0E0EE5BF84F808190E02F5FCC
:106B10002F772093C30702C08FEF9FEF3FBF0895E9
:106B2000FF920F931F93CF93DF93F62EFC012081EA
:106B30002B3311F1009159060430F0F41091AF0598
:106B4000C12FD0E0F0E61F9F90011124BC01C901C4
:106B5000895D9B4F0E94E7BBC65FD94FF8821F5FDC
:106B6000143018F41093AF0502C01092AF050F5FF8
:106B70000093590681E001C080E0DF91CF911F9121
:106B80000F91FF9008958091AD059091AE0500970B
:106B900031F04AE050E060E070E00C9406B260E052
:106BA00070E0CB0108958091AD059091AE050097FE
:106BB00031F04AE050E060E070E00C94D5B060E065
:106BC00070E0CB010895EFDF97FD0CC0ECDF6F3F65
:106BD00071058105910509F014F4E5DF01C06FEF3F
:106BE000862F089580E008958091AD059091AE05BF
:106BF000892B39F0E8DF91E0811101C090E0892F05
:106C0000089581E008951F93CF93DF938091AD05A0
:106C10009091AE050097E1F0FC01EF011191212F59
:106C20002F7D79F0153411F01536B9F7188260E030
:106C300070E00E946DAF1883562F472F382F292FF1
:106C40000BC060E070E0DF91CF911F910C946DAFAD
:106C500050E040E030E020E0652F742F832F922F2A
:106C6000DF91CF911F910895CF92DF92EF92FF9223
:106C7000C0909C03D0909D03E0909E03F0909F03F2
:106C80008091A003882321F120E030E0A901C70111
:106C9000B6010E948EB38823D9F020E030E040E0B6
:106CA0005FE3C701B6010E94F3B39B01AC010E94F0
:106CB000F3B32BED3FE049E450E40E94F3B39B01B2
:106CC000AC0160E070E080E89FE30E94C8B804C0B7
:106CD00060E070E080E89FE360937D0670937E063D
:106CE00080937F0690938006FF90EF90DF90CF9087
:106CF0000895CF92DF92EF92FF92CF93DF93EC0152
:106D000080913002882309F442C0C0901602D090CE
:106D10001702E0901802F0901902A701960168810D
:106D200079818A819B810E9412BA181624F4C88244
:106D3000D982EA82FB82C0901A02D0901B02E090B6
:106D40001C02F0901D02A70196016C817D818E814D
:106D50009F810E9412BA181624F4CC82DD82EE8242
:106D6000FF82C0901E02D0901F02E0902002F0909F
:106D70002102A7019601688579858A859B850E94F5
:106D800012BA181624F4C886D986EA86FB86DF91E3
:106D9000CF91FF90EF90DF90CF90089580E1E6E4EF
:106DA000F3E0AAEFB5E001900D928A95E1F708951E
:106DB000AF92BF92CF92DF92EF92FF920F931F9309
:106DC000CF93DF93C82FDD27C7FDD0958E01000F2D
:106DD000111F000F111FF801E251FA4F20E030E0BF
:106DE000A90160817181828193810E94ECB7F801D1
:106DF000E85DF84F20813181428153810E94ECB7D8
:106E00006B017C01F801E051FC4F60837183828348
:106E100093830B55184FF801659175918591949165
:106E20008E01000F111F000F111F980124503C4FBD
:106E30005901A70196010E94ECB7F50160837183A7
:106E4000828393830F54184FF80165917591859152
:106E50009491CC0FDD1FCC0FDD1FCA5EDD4FA70163
:106E600096010E94ECB7688379838A839B83DF91C4
:106E7000CF911F910F91FF90EF90DF90CF90BF9037
:106E8000AF90089581548A3148F5482F50E0FA01B7
:106E900063E0F595E7956A95E1F7EE5BFC4F20819D
:106EA00030E0877002C0359527958A95E2F720FF7C
:106EB00015C0FA01E85DFC4F2081222339F0809152
:106EC0001C0490911D04820F911D02C080E090E08F
:106ED0009093AE058093AD0581E0089580E008951C
:106EE00083E5D0DF882349F08EDE609367067093D8
:106EF00068068093690690936A0684E5C3DF882359
:106F000049F081DE609363067093640680936506A2
:106F10009093660682E4B6DF882349F034DE6093FE
:106F20005F0670936006809361069093620688E521
:106F3000A9DF882349F067DE6093790370937A03B1
:106F400080937B0390937C0389E59CDF882349F041
:106F50005ADE60937D0370937E0380937F0390934A
:106F600080038AE58FDF882349F04DDE609381033B
:106F700070938203809383039093840385E482DF7C
:106F8000882349F040DE60938503709386038093E5
:106F9000870390938803089575DF882339F081E093
:106FA0002091AD053091AE05232B09F480E00895C2
:106FB00020912D0F90912E0F81E0291301C080E0C8
:106FC0000895F6DF882331F080912E0F8F5F8F7048
:106FD00080932E0F08958CE0E4E3F7E0AAEFB5E08C
:106FE00001900D928A95E1F70895EF92FF920F9329
:106FF0001F93CF93DF93EC017B01198218821B82D0
:107000001A821D821C8261157105B9F1FB01019084
:107010000020E9F78F0101501109061B170BB80179
:107020006F5F7F4F80E090E00E94EBBA009759F0CD
:10703000998388831B830A832C813D81232B81F4D0
:10704000FC0110820DC088819981009711F00E9487
:10705000DEAE198218821D821C821B821A820DC02C
:107060001D830C83B70188819981DF91CF911F9196
:107070000F91FF90EF900C94E7BBDF91CF911F91A0
:107080000F91FF90EF9008958F929F92AF92BF92D1
:10709000CF92DF92EF92FF926B017C010E941F2B37
:1070A0004B015C01C114D104E104F104E1F00E9440
:1070B0001F2B681979098A099B09683E734081056D
:1070C000910580F321E0C21AD108E108F10888EEA9
:1070D000880E83E0981EA11CB11CC114D104E104E8
:1070E000F10429F7DFCFFF90EF90DF90CF90BF90B2
:1070F000AF909F908F900895CF93DF93282F30E02B
:10710000F901E95BF14F8491F901EA58F24FD4910A
:10711000F901E454F24FC491CC2391F081110E9403
:10712000CB2AEC2FF0E0EE0FFF1FE557F84FA591AB
:10713000B4912C912D2381E090E021F480E002C0F5
:1071400080E090E0DF91CF9108950F931F93CF934C
:10715000DF931F92CDB7DEB7282F30E0F901E95B4E
:10716000F14F8491F901EA58F24F1491F901E45476
:10717000F24F04910023C9F0882321F069830E9413
:10718000CB2A6981E02FF0E0EE0FFF1FEE5BF24F9C
:10719000A591B4919FB7F8948C91611103C010959B
:1071A000812301C0812B8C939FBF0F90DF91CF91E2
:1071B0001F910F9108952FB7F89460915C0F709113
:1071C0005D0F80915E0F90915F0F2FBF08950F9319
:1071D0001F93CF93DF93EC018881813011F4EBDFB3
:1071E00004C069857A858B859C850D811E812F81E0
:1071F0003885601B710B820B930B28EE33E040E067
:1072000050E00E9494B789819A81AB81BC81280F9C
:10721000391F4A1F5B1FCA01B901DF91CF911F912E
:107220000F910895CF92DF92EF92FF92C090EA0300
:10723000D090EB03E090EC03F090ED036091CF0C65
:107240007091D00C68507109882777FD8095982F30
:107250000E9494B39B01AC01C701B6010E948EB39A
:1072600087FF1CC020E030E040E050E4C701B601D9
:107270000E94ECB70E9435B97093010D6093000D28
:107280009ADF605A75418F4F9F4F6093020D709344
:10729000030D8093040D9093050D08C01092020D0C
:1072A0001092030D1092040D1092050DFF90EF90B7
:1072B000DF90CF900895CF92DF92EF92FF92C0902F
:1072C000E603D090E703E090E803F090E9036091D3
:1072D000D30C7091D40C6D507109882777FD80957F
:1072E000982F0E9494B39B01AC01C701B6010E9484
:1072F0008EB387FF1CC020E030E040E050E4C701BF
:10730000B6010E94ECB70E9435B97093070D6093E7
:10731000060D51DF605E714B8F4F9F4F6093080DDC
:107320007093090D80930A0D90930B0D08C0109275
:10733000080D1092090D10920A0D10920B0DFF907E
:10734000EF90DF90CF90089536DF609356037093EF
:107350005703809358039093590308958091A9058A
:107360009091AA05A091AB05B091AC0580930A025B
:1073700090930B02A0930C02B0930D028091A7058D
:107380009091A8059093130280931202DDCF809113
:107390000A0290910B02A0910C02B0910D02809311
:1073A000A9059093AA05A093AB05B093AC05809175
:1073B0001202909113029093A8058093A70584E68A
:1073C00090E09093130280931202BECF2F923F92CF
:1073D0004F925F926F927F928F929F92AF92BF92E5
:1073E000CF92DF92EF92FF920F931F93CF93DF9391
:1073F000CDB7DEB76E970FB6F894DEBF0FBECDBF28
:10740000EBECFAE084918F010F5F1F4F882319F096
:10741000F4DAF801F7CFE3ECFAE084918F010F5F23
:107420001F4F882319F0E9DAF801F7CF919903C0CB
:1074300005EF12E002C000EF12E0D8018D918D013E
:10744000882311F0DADAF9CF8AE0D7DAEBEBFAE049
:1074500084918F010F5F1F4F882319F0CEDAF80156
:10746000F7CF8091060187FD03C005EF12E002C04F
:1074700000EF12E0F80181918F01882311F0BDDA4D
:10748000F9CF8AE0BADAE3EBFAE084918F010F5F7B
:107490001F4F882319F0B1DAF801F7CF1C9903C008
:1074A00005EF12E002C000EF12E0D8018D918D01CE
:1074B000882311F0A2DAF9CF8AE09FDAEBEAFAE04A
:1074C00084918F010F5F1F4F882319F096DAF8011E
:1074D000F7CF019B03C005EF12E002C000EF12E0FE
:1074E000F80181918F01882311F087DAF9CF8AE0C2
:1074F00084DAEAE9FAE084918F010F5F1F4F882355
:1075000019F07BDAF801F7CF80E79EE00E94B64CD5
:107510006B017C011092CF0E1092D00E1092D10E02
:107520001092D20E4FEC5EE064E080E79EE00E9495
:10753000E34B8090CF0E9090D00EA090D10EB090E3
:10754000D20E40907F0E5090800E6090810E709011
:10755000820E80E79EE00E94C84D0091C50EF0E1CA
:107560008F229924AA24BB24A7019601222733271E
:107570004427507429833A834B835C83A701960187
:1075800022273327442750722D833E834F83588709
:10759000A7019601222733274427507129873A876C
:1075A0004B875C87A7019601222733274427587011
:1075B0002D873E874F87588BA701960122273327B7
:1075C00044275470298B3A8B4B8B5C8BA701960117
:1075D00022273327442752702D8B3E8B4F8B588F99
:1075E000A70196012227307844275527298F3A8F03
:1075F0004B8F5C8F12013FE1232233245527472D07
:10760000362D252D3901AFE16A227724B1E1969517
:10761000879577956795BA95D1F7162F1170E6E99A
:10762000FAE08491BF016F5F7F4F882339F06D8F3F
:107630007E8FE3D96D8D7E8DFB01F3CFE0E9FAE01B
:107640008491BF016F5F7F4F882339F06D8F7E8FEC
:10765000D4D96D8D7E8DFB01F3CFB1016F5F7F4F6C
:1076600080E090E04AE00E940077EEE8FAE0849142
:107670002F01BFEF4B1A5B0A882319F0BED9F20124
:10768000F6CFB3016F5F7F4F80E090E04AE00E9449
:107690000077E7E8FAE084913F012FEF621A720A5F
:1076A000882319F0AAD9F301F6CF612F70E080E0AA
:1076B00090E00E948D7780918B0E90918C0EA0911E
:1076C0008D0EB0918E0E892B8A2B8B2B09F45CC00A
:1076D000E8E7FAE084913F013FEF631A730A8823D9
:1076E00019F08BD9F301F6CF0F77602F660F607812
:1076F000602B772767FD7095872F972F0E948D77D6
:107700008091260690912706A0912806B09129061F
:10771000892B8A2B8B2B11F1EFE6FAE084918F01F4
:107720000F5F1F4F882319F068D9F801F7CF6091D8
:107730002A0670912B0680912C0690912D0620919F
:1077400026063091270640912806509129060E946E
:1077500094B7CA01B9014AE00E940077E7E6FAE06F
:1077600084918F010F5F1F4F882319F046D9F801CC
:10777000F7CFB7016F71772780E090E04AE00E9471
:107780000077EBE5FAE00BC0EEE7FAE084918F01B9
:107790000F5F1F4F8823A9F330D9F801F7CF8491E9
:1077A0008F010F5F1F4F882319F027D9F801F7CFFA
:1077B000609116067091170680911806909119062F
:1077C00020912606309127064091280650912906DF
:1077D0000E9494B7CA01B9014AE00E940077892843
:1077E0008A288B2859F4E7E5FAE084918F010F5F2E
:1077F0001F4F882319F001D9F801F7CFF7FE0BC00E
:10780000E3E5FAE084918F010F5F1F4F882319F0A1
:10781000F4D8F801F7CF89819A81AB81BC81892B9B
:107820008A2B8B2B59F0EEE4FAE084918F010F5FE5
:107830001F4F882319F0E1D8F801F7CF2D813E8141
:107840004F815885232B242B252B59F0E9E4FAE0AE
:1078500084918F010F5F1F4F882319F0CED8F80154
:10786000F7CF89859A85AB85BC85892B8A2B8B2B95
:1078700059F0E3E4FAE084918F010F5F1F4F8823F2
:1078800019F0BBD8F801F7CF2D853E854F85588973
:10789000232B242B252B59F0EDE3FAE084918F0163
:1078A0000F5F1F4F882319F0A8D8F801F7CF8989F7
:1078B0009A89AB89BC89892B8A2B8B2B59F0E7E3FA
:1078C000FAE084918F010F5F1F4F882319F095D83C
:1078D000F801F7CF2D893E894F89588D232B242B12
:1078E000252B59F0E3E3FAE084918F010F5F1F4FDE
:1078F000882319F082D8F801F7CF898D9A8DAB8D46
:10790000BC8D892B8A2B8B2B59F0E9E2FAE084910C
:107910008F010F5F1F4F882319F06FD8F801F7CF41
:107920008AE06BD88BEF9DE00E94B64C6B017C0126
:1079300010925A0E10925B0E10925C0E10925D0E19
:107940004AE55EE064E08BEF9DE00E94E34B8090AF
:107950005A0E90905B0EA0905C0EB0905D0E409021
:107960000A0E50900B0E60900C0E70900D0E8BEF67
:107970009DE00E94C84D0091500EA0E18A229924FA
:10798000AA24BB24A7019601222733274427507439
:1079900029833A834B835C83A701960122273327EF
:1079A000442750722D833E834F835887A701960149
:1079B000222733274427507129873A874B875C87D2
:1079C000A701960122273327442758702D873E8729
:1079D0004F87588BA70196012227332744275470DD
:1079E000298B3A8B4B8B5C8BA7019601222733277F
:1079F000442752702D8B3E8B4F8B588FA7019601D9
:107A00002227307844275527298F3A8F4B8F5C8F58
:107A100012013FE1232233245527472D362D252DF2
:107A20003901AFE16A227724F1E196958795779540
:107A30006795FA95D1F7162F1170E5E2FAE0849177
:107A4000BF016F5F7F4F882341F06D8F7E8F0E9453
:107A5000FD346D8D7E8DFB01F2CFEFE1FAE0849174
:107A6000BF016F5F7F4F882341F06D8F7E8F0E9433
:107A7000FD346D8D7E8DFB01F2CFB1016F5F7F4FC5
:107A800080E090E04AE00E940077EDE1FAE0849126
:107A90002F01BFEF4B1A5B0A882321F00E94FD34AF
:107AA000F201F5CFB3016F5F7F4F80E090E04AE0D5
:107AB0000E940077E6E1FAE084913F012FEF621A1D
:107AC000720A882321F00E94FD34F301F5CF612F63
:107AD00070E080E090E00E948D778091160E90918A
:107AE000170EA091180EB091190E892B8A2B8B2B93
:107AF00009F45FC0E7E0FAE084913F013FEF631AC9
:107B0000730A882321F00E94FD34F301F5CF0F772B
:107B1000602F660F6078602B772767FD7095872F41
:107B2000972F0E948D778091260690912706A0912D
:107B30002806B0912906892B8A2B8B2B19F1EEEFA1
:107B4000F9E084918F010F5F1F4F882321F00E947D
:107B5000FD34F801F6CF60912E0670912F068091CA
:107B600030069091310620912606309127064091EB
:107B70002806509129060E9494B7CA01B9014AE02B
:107B80000E940077E6EFF9E084918F010F5F1F4FAD
:107B9000882321F00E94FD34F801F6CFB7016F7100
:107BA000772780E090E04AE00E940077EAEEF9E073
:107BB0000CC0EDE0FAE084918F010F5F1F4F882326
:107BC000A9F30E94FD34F801F6CF84918F010F5F75
:107BD0001F4F882321F00E94FD34F801F6CF6091F9
:107BE0001A0670911B0680911C0690911D0620912B
:107BF00026063091270640912806509129060E94BA
:107C000094B7CA01B9014AE00E94007789288A28FE
:107C10008B2861F4E6EEF9E084918F010F5F1F4F2E
:107C2000882321F00E94FD34F801F6CFF7FE0CC046
:107C3000E2EEF9E084918F010F5F1F4F882321F05E
:107C40000E94FD34F801F6CF89819A81AB81BC8115
:107C5000892B8A2B8B2B61F0EDEDF9E084918F015C
:107C60000F5F1F4F882321F00E94FD34F801F6CFEB
:107C70002D813E814F815885232B242B252B61F0AC
:107C8000E8EDF9E084918F010F5F1F4F882321F009
:107C90000E94FD34F801F6CF89859A85AB85BC85B5
:107CA000892B8A2B8B2B61F0E2EDF9E084918F0117
:107CB0000F5F1F4F882321F00E94FD34F801F6CF9B
:107CC0002D853E854F855889232B242B252B61F04C
:107CD000ECECF9E084918F010F5F1F4F882321F0B6
:107CE0000E94FD34F801F6CF89899A89AB89BC8955
:107CF000892B8A2B8B2B61F0E6ECF9E084918F01C4
:107D00000F5F1F4F882321F00E94FD34F801F6CF4A
:107D10002D893E894F89588D232B242B252B61F0EB
:107D2000E2ECF9E084918F010F5F1F4F882321F06F
:107D30000E94FD34F801F6CF898D9A8DAB8DBC8DF4
:107D4000892B8A2B8B2B61F0E8EBF9E084918F0172
:107D50000F5F1F4F882321F00E94FD34F801F6CFFA
:107D60008AE00E94FD3486E89DE00E94B64C6B01DB
:107D70007C011092E50D1092E60D1092E70D109225
:107D8000E80D45EE5DE064E086E89DE00E94E34B8F
:107D90008090E50D9090E60DA090E70DB090E80D75
:107DA0004090950D5090960D6090970D7090980DA5
:107DB00086E89DE00E94C84D0091DB0DA0E18A227B
:107DC0009924AA24BB24A7019601222733274427FC
:107DD000507429833A834B835C83A7019601222741
:107DE0003327442750722D833E834F835887A70142
:107DF0009601222733274427507129873A874B87DA
:107E00005C87A701960122273327442758702D87C6
:107E10003E874F87588BA701960122273327442797
:107E20005470298B3A8B4B8B5C8BA70196012227D0
:107E30003327442752702D8B3E8B4F8B588FA701D1
:107E400096012227307844275527298F3A8F4B8F68
:107E50005C8F12013FE1232233245527472D362D15
:107E6000252D3901AFE16A22772451E19695879556
:107E7000779567955A95D1F7162F1170E4EBF9E0D5
:107E80008491BF016F5F7F4F882341F06D8F7E8F9C
:107E90000E94FD346D8D7E8DFB01F2CFEEEAF9E09C
:107EA0008491BF016F5F7F4F882341F06D8F7E8F7C
:107EB0000E94FD346D8D7E8DFB01F2CFB1016F5FAD
:107EC0007F4F80E090E04AE00E940077ECEAF9E022
:107ED00084912F01BFEF4B1A5B0A882321F00E9487
:107EE000FD34F201F5CFB3016F5F7F4F80E090E08A
:107EF0004AE00E940077E5EAF9E084913F012FEF24
:107F0000621A720A882321F00E94FD34F301F5CF32
:107F1000612F70E080E090E00E948D778091A10D4C
:107F20009091A20DA091A30DB091A40D892B8A2B45
:107F30008B2B09F45FC0E6E9F9E084913F013FEF44
:107F4000631A730A882321F00E94FD34F301F5CFF0
:107F50000F77602F660F6078602B772767FD70952D
:107F6000872F972F0E948D77809126069091270664
:107F7000A0912806B0912906892B8A2B8B2B19F109
:107F8000EDE8F9E084918F010F5F1F4F882321F006
:107F90000E94FD34F801F6CF6091320670913306ED
:107FA000809134069091350620912606309127065F
:107FB00040912806509129060E9494B7CA01B90140
:107FC0004AE00E940077E5E8F9E084918F010F5FB5
:107FD0001F4F882321F00E94FD34F801F6CFB7012E
:107FE0006F71772780E090E04AE00E940077E9E730
:107FF000F9E00CC0ECE9F9E084918F010F5F1F4FAD
:108000008823A9F30E94FD34F801F6CF84918F01F3
:108010000F5F1F4F882321F00E94FD34F801F6CF37
:1080200060911E0670911F06809120069091210696
:108030002091260630912706409128065091290666
:108040000E9494B7CA01B9014AE00E9400778928CA
:108050008A288B2861F4E5E7F9E084918F010F5FAE
:108060001F4F882321F00E94FD34F801F6CFF7FE60
:108070000CC0E1E7F9E084918F010F5F1F4F882367
:1080800021F00E94FD34F801F6CF89819A81AB81FD
:10809000BC81892B8A2B8B2B61F0ECE6F9E0849173
:1080A0008F010F5F1F4F882321F00E94FD34F801DC
:1080B000F6CF2D813E814F815885232B242B252BF4
:1080C00061F0E7E6F9E084918F010F5F1F4F88238D
:1080D00021F00E94FD34F801F6CF89859A85AB85A1
:1080E000BC85892B8A2B8B2B61F0E1E6F9E084912A
:1080F0008F010F5F1F4F882321F00E94FD34F8018C
:10810000F6CF2D853E854F855889232B242B252B93
:1081100061F0EBE5F9E084918F010F5F1F4F882339
:1081200021F00E94FD34F801F6CF89899A89AB8944
:10813000BC89892B8A2B8B2B61F0E5E5F9E08491D2
:108140008F010F5F1F4F882321F00E94FD34F8013B
:10815000F6CF2D893E894F89588D232B242B252B33
:1081600061F0E1E5F9E084918F010F5F1F4F8823F3
:1081700021F00E94FD34F801F6CF898D9A8DAB8DE8
:10818000BC8D892B8A2B8B2B61F0E7E4F9E084917D
:108190008F010F5F1F4F882321F00E94FD34F801EB
:1081A000F6CF8AE00E94FD3481E19DE00E94B64C4A
:1081B0006B017C011092700D1092710D1092720D76
:1081C0001092730D40E75DE064E081E19DE00E9464
:1081D000E34B8090700D9090710DA090720DB09057
:1081E000730D4090200D5090210D6090220D7090E5
:1081F000230D81E19DE00E94C84D0091660DA0E134
:108200008A229924AA24BB24A70196012227332776
:108210004427507429833A834B835C83A7019601DA
:1082200022273327442750722D833E834F8358875C
:10823000A7019601222733274427507129873A87BF
:108240004B875C87A7019601222733274427587064
:108250002D873E874F87588BA7019601222733270A
:1082600044275470298B3A8B4B8B5C8BA70196016A
:1082700022273327442752702D8B3E8B4F8B588FEC
:10828000A70196012227307844275527298F3A8F56
:108290004B8F5C8F12013FE1232233245527472D5A
:1082A000362D252D3901AFE16A22772431E19695EB
:1082B0008795779567953A95D1F7162F1170E2E477
:1082C000F9E08491BF016F5F7F4F882341F06D8F8C
:1082D0007E8F0E94FD346D8D7E8DFB01F2CFECE32D
:1082E000F9E08491BF016F5F7F4F882341F06D8F6C
:1082F0007E8F0E94FD346D8D7E8DFB01F2CFB1012A
:108300006F5F7F4F80E090E04AE00E940077EAE3F1
:10831000F9E084912F01BFEF4B1A5B0A882321F00B
:108320000E94FD34F201F5CFB3016F5F7F4F80E013
:1083300090E04AE00E940077E3E3F9E084913F0196
:108340002FEF621A720A882321F00E94FD34F30194
:10835000F5CF612F70E080E090E00E948D778091F2
:108360002C0D90912D0DA0912E0DB0912F0D892BDC
:108370008A2B8B2B09F45FC0E4E2F9E084913F0182
:108380003FEF631A730A882321F00E94FD34F30142
:10839000F5CF0F77602F660F6078602B772767FD2A
:1083A0007095872F972F0E948D7780912606909148
:1083B0002706A0912806B0912906892B8A2B8B2BA2
:1083C00019F1EBE1F9E084918F010F5F1F4F8823D2
:1083D00021F00E94FD34F801F6CF609136067091CD
:1083E0003706809138069091390620912606309103
:1083F000270640912806509129060E9494B7CA0189
:10840000B9014AE00E940077E3E1F9E084918F012D
:108410000F5F1F4F882321F00E94FD34F801F6CF33
:10842000B7016F71772780E090E04AE00E94007703
:10843000E7E0F9E00CC0EAE2F9E084918F010F5F18
:108440001F4F8823A9F30E94FD34F801F6CF8491D1
:108450008F010F5F1F4F882321F00E94FD34F80128
:10846000F6CF6091220670912306809124069091A8
:108470002506209126063091270640912806509126
:1084800029060E9494B7CA01B9014AE00E94007708
:1084900089288A288B2861F4E3E0F9E084918F0130
:1084A0000F5F1F4F882321F00E94FD34F801F6CFA3
:1084B000F7FE0CC0EFEFF8E084918F010F5F1F4FC4
:1084C000882321F00E94FD34F801F6CF89819A813A
:1084D000AB81BC81892B8A2B8B2B61F0EAEFF8E012
:1084E00084918F010F5F1F4F882321F00E94FD347C
:1084F000F801F6CF2D813E814F815885232B242B07
:10850000252B61F0E5EFF8E084918F010F5F1F4F9D
:10851000882321F00E94FD34F801F6CF89859A85E1
:10852000AB85BC85892B8A2B8B2B61F0EFEEF8E0B5
:1085300084918F010F5F1F4F882321F00E94FD342B
:10854000F801F6CF2D853E854F855889232B242BA6
:10855000252B61F0E9EEF8E084918F010F5F1F4F4A
:10856000882321F00E94FD34F801F6CF89899A8989
:10857000AB89BC89892B8A2B8B2B61F0E3EEF8E069
:1085800084918F010F5F1F4F882321F00E94FD34DB
:10859000F801F6CF2D893E894F89588D232B242B46
:1085A000252B61F0EFEDF8E084918F010F5F1F4FF5
:1085B000882321F00E94FD34F801F6CF898D9A8D31
:1085C000AB8DBC8D892B8A2B8B2B61F0E5EDF8E010
:1085D00084918F010F5F1F4F882321F00E94FD348B
:1085E000F801F6CF8AE06E960FB6F894DEBF0FBEA4
:1085F000CDBFDF91CF911F910F91FF90EF90DF9052
:10860000CF90BF90AF909F908F907F906F905F9032
:108610004F903F902F900C94FD34CF93DF931F9297
:108620001F92CDB7DEB7789484B5826084BD84B5DF
:10863000816084BD85B5826085BD85B5816085BD5D
:1086400080916E00816080936E0010928100809115
:10865000810082608093810080918100816080939D
:108660008100809180008160809380008091B100C2
:1086700084608093B1008091B00081608093B000ED
:10868000809191008260809391008091910081603F
:108690008093910080919000816080939000809100
:1086A000A10082608093A1008091A10081608093ED
:1086B000A1008091A00081608093A00080912101A1
:1086C000826080932101809121018160809321014A
:1086D0008091200181608093200180917A008460E4
:1086E00080937A0080917A00826080937A008091F2
:1086F0007A00816080937A0080917A00806880930C
:108700007A001092C10082E08093C0001092C500F0
:1087100087E08093C4008091C10080618093C10094
:108720008091C10088608093C1008091C100806801
:108730008093C100E2EEFBE084918F010F5F1F4F39
:10874000882321F00E94FD34F801F6CFE9EBFCE02C
:1087500084918F010F5F1F4F882321F00E94FD3409
:10876000F801F6CFF4B6F0FE0CC0E9EDFBE0849121
:108770008F010F5F1F4F882321F00E94FD34F80105
:10878000F6CFF1FE0CC0E8ECFBE084918F010F5FA7
:108790001F4F882321F00E94FD34F801F6CFF2FE2E
:1087A0000CC0E6EBFBE084918F010F5F1F4F882325
:1087B00021F00E94FD34F801F6CFF3FE0CC0E5EA8B
:1087C000FBE084918F010F5F1F4F882321F00E94EF
:1087D000FD34F801F6CFF5FE0CC0E4E9FBE084912E
:1087E0008F010F5F1F4F882321F00E94FD34F80195
:1087F000F6CF14BEEDE8FBE084918F010F5F1F4FB1
:10880000882321F00E94FD34F801F6CF80E20E9417
:10881000FD34E6E8FBE084918F010F5F1F4F882352
:1088200021F00E94FD34F801F6CF8AE00E94FD3469
:10883000E9EBFCE084918F010F5F1F4F882321F04B
:108840000E94FD34F801F6CFE6E7FBE084918F014A
:108850000F5F1F4F882321F00E94FD34F801F6CFEF
:10886000E2E6FBE084918F010F5F1F4F882321F028
:108870000E94FD34F801F6CFE9E2FBE084918F011C
:108880000F5F1F4F882321F00E94FD34F801F6CFBF
:10889000E9EBFCE084918F010F5F1F4F882321F0EB
:1088A0000E94FD34F801F6CFE2E1FBE084918F01F4
:1088B0000F5F1F4F882321F00E94FD34F801F6CF8F
:1088C000E9EBFCE084918F010F5F1F4F882321F0BB
:1088D0000E94FD34F801F6CF8091600F9091610FF6
:1088E0009E012F5F3F4F009719F426563F4002C06C
:1088F000281B390B3A83298369817A8183E09BE0C5
:108900000E941E7960ED74E08CEE9AE00E941E7960
:108910008AE00E94FD3481E080930A0680930B0672
:1089200080930C0680930D060E949B588CE0EEEE1F
:10893000F5E0AAEFB5E001900D928A95E1F70E946B
:108940001B616D9A8091010180618093010180918A
:1089500001018860809301019D9A809101018062EC
:108960008093010188E00E94055180910101886097
:108970008093010186E00E94055187ED80937A0083
:1089800010927E0010927D0080917E008160809325
:108990007E0080917E00846080937E0080E888BDA8
:1089A00080916E00846080936E006AEF70E080E0DA
:1089B00090E00E94443885E090E09093E805809331
:1089C000E70560E08091290290912A020E94F73227
:1089D00020E030E040EA50E40E948EB387FF0AC0F6
:1089E0008091290290912A02409790932A028093C5
:1089F0002902E7CF81E391E090932C0280932B0230
:108A000060E08091E5059091E6050E94F73220E054
:108A100030E848E953E40E9412BA181654F48091E1
:108A2000E5059091E60540969093E6058093E5056F
:108A3000E7CF80912702909128020E94BB2F20E06F
:108A400030E040EA50E40E948EB387FF0AC0809174
:108A50002702909128024097909328028093270242
:108A6000E8CF8091E3059091E4050E94BB2F20E0C0
:108A700030E046E153E40E9412BA181654F4809193
:108A8000E3059091E40540969093E4058093E30517
:108A9000E8CF28E288E190E00FB6F894A89580939B
:108AA00060000FBE2093600080910A01886080936F
:108AB0000A0180910A01806180930A0180910A0174
:108AC000806280930A010E9461A680912101887FC3
:108AD00081608093210180E79EE00E94C17565E07E
:108AE00080E79EE00E949C4D8BEF9DE00E94C17547
:108AF00065E08BEF9DE00E949C4D86E89DE00E9422
:108B0000C17581E19DE00E94C17563E080E79EE050
:108B10000E94E64D63E08BEF9DE00E94E64D65E02C
:108B200086E89DE00E94E64D8091D50D9091D60D8E
:108B3000A091D70DB091D80D8F788093D50D9093DB
:108B4000D60DA093D70DB093D80D45ED5DE06CEE3A
:108B500086E89DE038D68091D50D9091D60DA091F4
:108B6000D70DB091D80D8F77987F8093D50D9093C6
:108B7000D60DA093D70DB093D80D45ED5DE06CEE0A
:108B800086E89DE020D662E086E89DE00E94FB4DED
:108B900065E086E89DE0D0D78FEF9FEFAFE0B0E0D3
:108BA00080932C0D90932D0DA0932E0DB0932F0D2F
:108BB0004CE25DE064E981E19DE005D660E081E1A1
:108BC0009DE0AED680910A01816080930A01809178
:108BD0000A01826080930A0180910A018460809377
:108BE0000A0180910A01806480930A010F9A179A02
:108BF0000E9A169A0D9A159A0C9A149A9998A19A07
:108C000024982C9A809107018F77809307019FB752
:108C1000F894809108018068809308019FBF0998AB
:108C2000119A389A4098179A1092EA05399A419801
:108C3000169A1092EB053A9A4298159A1092EC0502
:108C40003B9A4398149A809180008C7F8093800097
:108C500080918100877E8860809381008091800070
:108C60008F738093800080918100887F82608093E1
:108C7000810080E090E490938900809388001092B6
:108C800085001092840080916F00826080936F0055
:108C900081E08093E90578940E94C2331092ED053B
:108CA0008091010188608093010180915906843090
:108CB00030F40E94484F811102C00E944D70809193
:108CC0005906882391F00E9401118091590688234A
:108CD00061F0815080935906809158068F5F809390
:108CE0005806843010F01092580680915706882359
:108CF000A9F1E9EBFCE084918F010F5F1F4F8823FE
:108D000021F00E94FD34F801F6CFEAEAFCE08491FC
:108D10008F010F5F1F4F882321F00E94FD34F8015F
:108D2000F6CF8091570680FDE4C38091570684FDFD
:108D3000E0C38091570681FDF7C38091570685FDFA
:108D4000F3C38091570682FD0AC48091570686FDC1
:108D500006C48AE00E94FD341092570680912D02CD
:108D6000815080932D0281117EC18AE080932D0273
:108D70000E94D837882309F476C180912E0F9091F4
:108D80003A06981709F44CC080912E0F80933A064A
:108D90001092360610923706109238061092390655
:108DA0001092320610923306109234061092350655
:108DB00010922E0610922F06109230061092310655
:108DC00010922A0610922B0610922C0610922D0655
:108DD0001092260610922706109228061092290655
:108DE0001092220610922306109224061092250655
:108DF00010921E0610921F06109220061092210655
:108E000010921A0610921B0610921C0610921D0654
:108E10001092160610921706109218061092190654
:108E20001092CF0E1092D00E1092D10E1092D20E40
:108E30004FEC5EE062E180E79EE0C5D480911606CB
:108E400090911706A0911806B09119064091CF0E87
:108E50005091D00E6091D10E7091D20E840F951F5B
:108E6000A61FB71F8093160690931706A0931806A7
:108E7000B093190610925A0E10925B0E10925C0E6F
:108E800010925D0E4AE55EE062E18BEF9DE09BD4BF
:108E900080911A0690911B06A0911C06B0911D06A8
:108EA00040915A0E50915B0E60915C0E70915D0E78
:108EB000840F951FA61FB71F80931A0690931B0659
:108EC000A0931C06B0931D061092E50D1092E60DBE
:108ED0001092E70D1092E80D45EE5DE062E186E844
:108EE0009DE071D480911E0690911F06A0912006EE
:108EF000B09121064091E50D5091E60D6091E70D8E
:108F00007091E80D840F951FA61FB71F80931E0652
:108F100090931F06A0932006B09321061092700D27
:108F20001092710D1092720D1092730D40E75DE07A
:108F300062E181E19DE047D4809122069091230671
:108F4000A0912406B09125064091700D5091710DAD
:108F50006091720D7091730D840F951FA61FB71F3E
:108F60008093220690932306A0932406B0932506AF
:108F700080E79EE0FBD471708827992700912A062C
:108F800010912B0620912C0630912D06060F171FED
:108F9000281F391F00932A0610932B0620932C06B6
:108FA00030932D068BEF9DE0E1D4717088279927CF
:108FB00000912E0610912F06209130063091310637
:108FC000060F171F281F391F00932E0610932F0618
:108FD000209330063093310686E89DE0C7D4717047
:108FE0008827992700913206109133062091340684
:108FF00030913506060F171F281F391F00933206C0
:1090000010933306209334063093350681E19DE0BA
:10901000ADD47170882799270091360610913706D4
:109020002091380630913906060F171F281F391F67
:10903000009336061093370620933806309339068E
:109040008091260690912706A0912806B0912906C6
:109050000196A11DB11D8093260690932706A0932B
:109060002806B093290680E79EE080D48C010F711A
:10907000112780911406909115060817190709F415
:1090800081C01093150600931406ECE8FCE084916F
:109090007F019FEFE91AF90A882321F00E94FD342D
:1090A000F701F5CFB80180E090E00E9492B320E094
:1090B00030E040E85FE30E94ECB720E030E040E0C1
:1090C0005DE30E94F3B36B017C0180E79EE06FD506
:1090D000882329F02CEE31E548E35EE304C026E660
:1090E00036E646EA5EE3C701B6010E94F3B320E923
:1090F00032EC45EF5DE30E94C8B823EF34E045EB66
:109100005FE30E94C8B820E030E04AE754E40E94E0
:10911000F3B342E00E94B377E1E8FCE084917F0181
:109120009FEFE91AF90A882321F00E94FD34F70124
:10913000F5CFB8016F5F7F4F80E090E04AE00E947A
:109140000077E4E7FCE084918F010F5F1F4F8823D5
:1091500021F00E94FD34F801F6CF80E79EE027D58C
:10916000682F70E080E090E00E948D77E1E7FCE0FE
:1091700084918F010F5F1F4F882321F00E94FD34DF
:10918000F801F6CF8BEF9DE0F1D38C010F71112721
:1091900080911206909113060817190709F481C0EF
:1091A0001093130600931206EFE5FCE084917F0113
:1091B0009FEFE91AF90A882321F00E94FD34F70194
:1091C000F5CFB80180E090E00E9492B320E030E05B
:1091D00040E85FE30E94ECB720E030E040E05DE370
:1091E0000E94F3B36B017C018BEF9DE0E0D48823F8
:1091F00029F02CEE31E548E35EE304C026E636E6CE
:1092000046EA5EE3C701B6010E94F3B320E932ECFF
:1092100045EF5DE30E94C8B823EF34E045EB5FE320
:109220000E94C8B820E030E04AE754E40E94F3B35B
:1092300042E00E94B377E4E5FCE084917F019FEF78
:10924000E91AF90A882321F00E94FD34F701F5CFCD
:10925000B8016F5F7F4F80E090E04AE00E940077A6
:10926000E7E4FCE084918F010F5F1F4F882321F01A
:109270000E94FD34F801F6CF8BEF9DE098D4682F63
:1092800070E080E090E00E948D77E4E4FCE084915F
:109290008F010F5F1F4F882321F00E94FD34F801DA
:1092A000F6CF86E89DE062D38C010F711127809183
:1092B0001006909111060817190709F481C0109340
:1092C000110600931006E2E3FCE084917F019FEF1A
:1092D000E91AF90A882321F00E94FD34F701F5CF3D
:1092E000B80180E090E00E9492B320E030E040E8D6
:1092F0005FE30E94ECB720E030E040E05DE30E94D5
:10930000F3B36B017C0186E89DE051D4882329F0FA
:109310002CEE31E548E35EE304C026E636E646EA95
:109320005EE3C701B6010E94F3B320E932EC45EFDA
:109330005DE30E94C8B823EF34E045EB5FE30E9491
:10934000C8B820E030E04AE754E40E94F3B342E0BA
:109350000E94B377E7E2FCE084917F019FEFE91A76
:10936000F90A882321F00E94FD34F701F5CFB801F6
:109370006F5F7F4F80E090E04AE00E940077EAE173
:10938000FCE084918F010F5F1F4F882321F00E9422
:10939000FD34F801F6CF86E89DE009D4682F70E02F
:1093A00080E090E00E948D77E7E1FCE084918F01FE
:1093B0000F5F1F4F882321F00E94FD34F801F6CF84
:1093C00081E19DE0D3D28C010F71112780910E06AF
:1093D00090910F060817190709F481C010930F0622
:1093E00000930E06E4E0FCE084917F019FEFE91A10
:1093F000F90A882321F00E94FD34F701F5CFB80166
:1094000080E090E00E9492B320E030E040E85FE32B
:109410000E94ECB720E030E040E05DE30E94F3B34F
:109420006B017C0181E19DE0C2D3882329F02CEE01
:1094300031E548E35EE304C026E636E646EA5EE34D
:10944000C701B6010E94F3B320E932EC45EF5DE3BA
:109450000E94C8B823EF34E045EB5FE30E94C8B830
:1094600020E030E04AE754E40E94F3B342E00E9477
:10947000B377E9EFFBE084917F019FEFE91AF90AE6
:10948000882321F00E94FD34F701F5CFB8016F5F0A
:109490007F4F80E090E04AE00E940077ECEEFBE036
:1094A00084918F010F5F1F4F882321F00E94FD34AC
:1094B000F801F6CF81E19DE07AD3682F70E080E07B
:1094C00090E00E948D77E9EEFBE084918F010F5FC1
:1094D0001F4F882321F00E94FD34F801F6CF0E942F
:1094E000087280E090E0892B09F4DFCB0E94000035
:1094F000DCCB60914B0670914C0680914D069091AB
:109500004E060E9494B320913B0630913C06409158
:109510003D0650913E060E94F3B3AB01BC0186EAC2
:109520009CE00E940A8205CC60914F067091500623
:1095300080915106909152060E9494B320913F066B
:109540003091400640914106509142060E94F3B38B
:10955000AB01BC0182EA9CE00E940A82F2CB6091DE
:1095600053067091540680915506909156060E94BC
:1095700094B32091430630914406409145065091A2
:1095800046060E94F3B3AB01BC018EE99CE00E9449
:109590000A82DFCB0CB405FC0DC01EBC00000DB46C
:1095A00007FEFDCF9EB51EBC00000DB407FEFDCF2B
:1095B0008EB508951EBC00000DB407FEFDCF8EB51C
:1095C0001EBC00000DB407FEFDCF9EB50895FB0143
:1095D0004081FC0120813181342768E0A901440FDA
:1095E000551F37FD07C09A016150C1F7FC01318357
:1095F000208308959A01F1E22F27F0E13F27F4CF6D
:1096000090E0FC01EA58F24F2491FC01E454F24F3F
:109610008491882399F090E0880F991FFC01E45A07
:10962000F24FA591B4918E5B924FFC01859194917C
:109630009FB7F8948C91822B8C939FBF08951F93B2
:10964000CF93DF93182FEB01DBDF209711F460E05D
:1096500004C0CF3FD10539F461E0812FDF91CF9174
:109660001F910C94A538E12FF0E0E95BF14F449194
:1096700050E0FA013197E231F10508F09BC0EC5758
:10968000FF4F0C94DBBA84B5806884BDC7BD97C01A
:1096900084B5806284BDC8BD92C08091800080681E
:1096A00080938000D0938900C093880088C0809107
:1096B0008000806280938000D0938B00C0938A00EA
:1096C0007EC080918000886080938000D0938D0060
:1096D000C0938C0074C08091B00080688093B0000B
:1096E000C093B3006CC08091B00080628093B000E2
:1096F000C093B40064C08091900080688093900013
:10970000D0939900C09398005AC0809190008062D5
:1097100080939000D0939B00C0939A0050C080919A
:109720009000886080939000D0939D00C0939C002F
:1097300046C08091A00080688093A0008091A00026
:109740008F7B8093A000D093A900C093A80037C05E
:109750008091A00080628093A000D093AB00C09362
:10976000AA002DC08091A00088608093A000D093B3
:10977000AD00C093AC0023C080912001806880932D
:109780002001D0932901C093280119C080912001A4
:10979000806280932001D0932B01C0932A010FC0D7
:1097A00080912001886080932001D0932D01C09387
:1097B0002C0105C0C038D1050CF04ECF48CFDF9149
:1097C000CF911F910895EF92FF920F931F93CF9324
:1097D000DF937C01162FEA010FB7F89480915C06A5
:1097E000811121C0E1EFFDE08491EBEAFDE094916D
:1097F000E82FF0E0EE0FFF1FE45AF24FA591B4916D
:109800008C91892321F461E085E30E94A53885E3EA
:10981000F7DE8CB580618CBD8CB580648CBD84E333
:10982000EFDE83E3EDDE80915C068F5F80935C0664
:109830000FBF8DE58CBD81E08DBD60E0F7018185B6
:109840000E94A538812F0E94422BF7018583212F8A
:1098500030E0220F232F221F330B232B69F08B8143
:109860000E94422B8A810E94422B89810E94422BB6
:1098700088810E94422B49C08DDE8CDE61E0F701B9
:1098800081850E94A53860E0F70181850E94A53896
:10989000812F0E94422B80E00E94422B90E0A0E0AA
:1098A000B0E0BA2FA92F982F882788839983AA839D
:1098B000BB8380E00E94422B488159816A817B8171
:1098C000482B762F652F542F4427488359836A836A
:1098D0007B8380E00E94422B488159816A817B8191
:1098E000482B762F652F542F4427488359836A834A
:1098F0007B8380E00E94422B088119812A813B8171
:10990000082B088319832A833B8361E0F701818553
:10991000DF91CF911F910F91FF90EF900C94A5389C
:109920000F931F93462F50E060E070E022E0440F59
:10993000551F661F771F2A95D1F744705527662754
:109940007727FC0103851485258536850B7F402B01
:10995000512B622B732B4387548765877687AC0125
:10996000455F5F4F60E81F910F912DCFCF93DF933D
:10997000EC01C15ADF4F188219821A821B82AE0194
:109980006FE621DF688179818A819B81DF91CF91A8
:1099900008958F929F92AF92BF92CF92DF92EF92F3
:1099A000FF920F931F93CF93DF93CDB7DEB72A9724
:1099B0000FB6F894DEBF0FBECDBF7C018B01D6DFA2
:1099C00092FFA2C081E0F701868380915D0681113C
:1099D0009DC08FE29FE00E94E7386B017C013CE371
:1099E000832E912CA12CB12CA50194010E9494B737
:1099F000CA01B901A50194010E9494B7952EC9012D
:109A0000FE0131965F01F1E8CF16F1E5DF06F1E0E6
:109A1000EF06F104E0F07F936F9368E170E00E943D
:109A2000B4BA9F938F93B901842F992D28E130E028
:109A300040E050E00E9494B73F932F9384E19EE072
:109A40009F938F93BF92AF920E9460B31AC0243647
:109A5000310558F47F936F9368E170E00E94B4BAC7
:109A60009F938F938AE09EE006C07F936F933F930E
:109A70002F9382E09EE09F938F93BF92AF920E94BC
:109A800060B30FB6F894DEBF0FBECDBFF501819174
:109A90005F01882319F00E94FD34F8CFE4E4FEE072
:109AA00084917F015FEFE51AF50A811103C0E12C73
:109AB000F12C15C00E94FD34F701F2CFE816F9062B
:109AC000A8F4F80180819181009781F0FC01EE0DEE
:109AD000FF1D80810E94FD34FFEFEF1AFF0AF8019D
:109AE00084819581E816F9064CF302C080E0F2CF3C
:109AF000E2E2FEE084918F010F5F1F4F882331F077
:109B00000E94FD34F801F6CF80E001C081E080932F
:109B10005D062A960FB6F894DEBF0FBECDBFDF916B
:109B2000CF911F910F91FF90EF90DF90CF90BF905A
:109B3000AF909F908F900895CF92DF92EF92FF9217
:109B40000F931F93AC014D5A5F4F062F10E020E09A
:109B500030E0980111270027002711272F7733279E
:109B6000FA01C080D180E280F380F0E8EF220C2976
:109B70001D292E293F29FA01008311832283338373
:109B80006DEE1F910F91FF90EF90DF90CF901BCE65
:109B9000CF93DF93EC01C15BDF4FAE016CE613DEC8
:109BA000688179818A819B81DF91CF910895F0DF6F
:109BB0006627772782709927E1E1969587957795B3
:109BC0006795EA95D1F7862F817008950F931F93BB
:109BD000AC01415B5F4F6F70FA01008111812281FE
:109BE0003381007F062B00831183228333836CEE45
:109BF0001F910F91E8CDCF92DF92EF92FF920F93DA
:109C00001F93AC01415B5F4F062F10E020E030E076
:109C1000FFE0000F111F221F331FFA95D1F7002715
:109C2000107821703327FA01C080D180E280F38060
:109C3000E894D7F8E0F80C291D292E293F29008344
:109C40001183228333836CEE1F910F91FF90EF906D
:109C5000DF90CF90B8CDCF93DF93EC018F81D0DC34
:109C60008A85CEDC8885CCDC8985CADC61E08F8181
:109C70000E94A53860E08A850E94A53860E088854A
:109C80000E94A53861E089850E94A538AE01455F34
:109C90005F4F60E8CE0197DDAE01415B5F4F6CEE38
:109CA000CE0191DDAE014D5A5F4F6DEECE018BDDE1
:109CB000AE01455A5F4F60EFCE0185DDAE01415FD9
:109CC0005F4F60E9CE017FDD68E0CE017FDF61E0BC
:109CD000CE0191DF81E08C83DF91CF910895CF9207
:109CE000DF92EF92FF920F93FC01AEEACA2EA7E437
:109CF000DA2EA1EEEA2EADE3FA2EC082D182E28204
:109D0000F382168213861486158616861786108AA5
:109D1000118A128A138A148A158A168A178A108E53
:109D2000118E128E138E148E158E168E178E10A213
:109D300011A212A213A214A215A216A217A210A673
:109D400011A612A613A614A615A616A617A610AA43
:109D500011AA12AA13AA14AA15AA16AA17AA10AE13
:109D600011AE12AE13AE14AE15AE16AEDC01DF9618
:109D70001D921D921D921C92139714961D921D9276
:109D80001D921C92139714961D921D921D921C9267
:109D9000139714961D921D921D921C921397149660
:109DA0001D921D921D921C92139714961D921D9246
:109DB0001D921C92139714961D921D921D921C9237
:109DC0001397149680E8C82E84E0D82E85E0E82EFC
:109DD000F12CCD92DD92ED92FC92139714961D9288
:109DE0001D921D921C92139714961D921D921D9206
:109DF0001C92139714961D921D921D921C921397FC
:109E000014961D921D921D921C92139714961D92EA
:109E10001D921D921C92139714961D921C921482EF
:109E20006783428720870187CF010F91FF90EF90D2
:109E3000DF90CF9010CFCF92DF92EF92FF920F93EF
:109E40001F93AC01415B5F4F062F10E020E030E034
:109E5000302F2227112700270027112722273F70A4
:109E6000FA01C080D180E280F380F0EFFF220C295C
:109E70001D292E293F29FA01008311832283338370
:109E80006CEE1F910F91FF90EF90DF90CF909BCCE5
:109E9000BF92CF92DF92EF92FF920F931F93CF93D7
:109EA000DF93CDB7DEB76E970FB6F894DEBF0FBE67
:109EB000CDBF60915A0670915B066115710571F115
:109EC0004DE150E08E010F5F1F4FC8010E9437B374
:109ED0001E8EF8017F01E01AF10AB190BB2039F122
:109EE0008AE0B812F7CF23C0B80185E39DE00E9455
:109EF000043582E20E94FD348AE00E94FD34BB20DA
:109F000069F18FEFE81AF80A80915A0690915B0682
:109F10008E0D9F1D90935B0680935A0681E02091E1
:109F20005A0630915B06232BE1F480E01AC0F80159
:109F3000EE0DFF1D108260E0C8010E94903588235D
:109F400069F3E9EBFCE084916F019FEFC91AD90A2C
:109F5000882351F20E94FD34F601F5CF80E090E0B5
:109F6000D9CF6E960FB6F894DEBF0FBECDBFDF918E
:109F7000CF911F910F91FF90EF90DF90CF90BF9006
:109F80000895CF92DF92EF92FF92C0900606D09094
:109F90000706E0900806F09009062091950330919D
:109FA00096034091970350919803C701B6010E9410
:109FB000F3B30E941DBA6093290F70932A0F809308
:109FC0002B0F90932C0FC701B6010E9430B92FB709
:109FD000F8946093A00C7093A10C8093A20C9093C2
:109FE000A30C2FBF1092190F10921A0F10921B0F73
:109FF00010921C0FFF90EF90DF90CF900895FF928A
:10A000000F931F93CF93DF93F090080481E0F8261D
:10A0100000910904082710910A041827F11002C0C2
:10A02000002319F0E9EBFCE004C01111FBCF80E044
:10A0300048C08491EF012196882321F00E94FD34CD
:10A04000FE01F7CFEFE2FDE08491EF012196882336
:10A0500021F00E94FD34FE01F7CFFF2059F0EDE220
:10A06000FDE08491EF012196882321F00E94FD34C8
:10A07000FE01F7CF002359F0EBE2FDE08491EF0100
:10A080002196882321F00E94FD34FE01F7CF1111A3
:10A0900003C0E1E2FDE00BC0E9E2FDE08491EF01E5
:10A0A00021968823B1F30E94FD34FE01F7CF8491FD
:10A0B000EF012196882321F00E94FD34FE01F7CFA5
:10A0C00081E0DF91CF911F910F91FF900895CF9282
:10A0D000DF92EF92FF920F931F93CF93DF937CEE6B
:10A0E000E72E72E0F72E06E413E0CAEFD5E0EEE1CA
:10A0F000CE2EE4E0DE2EF70181917F010E944237EF
:10A100008823D1F00E940336F6012081211104C07A
:10A1100020912204222329F0288139814A815B8100
:10A1200003C020E030E0A9010E94ECB7F801608391
:10A1300071838283938309C088819981AA81BB81BD
:10A14000F80180839183A283B3830C5F1F4F249611
:10A15000FFEFCF1ADF0A80EFE81682E0F80659F623
:10A1600086E40E94CC378823C9F00E94033620E0A1
:10A1700030E0A9010E9412BA181684F40E94033636
:10A1800020E030E040E752E40E94C8B860930A0241
:10A1900070930B0280930C0290930D028091260421
:10A1A00083FD2AC060915203709153038091540340
:10A1B00090915503209106063091070640910806BC
:10A1C00050910906E091560FEE23B1F00E94EBB7D3
:10A1D0009B01AC016091480F7091490F80914A0F2B
:10A1E00090914B0F0E94ECB76093480F7093490F0A
:10A1F00080934A0F90934B0FDF91CF911F910F9156
:10A20000FF90EF90DF90CF900895E82FF0E0E95BAA
:10A21000F14F849190E0FC013797EC30F105F8F4B0
:10A22000EA56FF4F0C94DBBA8091B100887F8460BE
:10A230008093B100089580919100887F846080931D
:10A24000910008958091A100887F84608093A1008F
:10A25000089580912101887F846080932101089571
:10A260008F929F92AF92BF92CF92DF92EF92FF9226
:10A270000F931F93CF93DF931F921F92CDB7DEB73B
:10A280007C01490180915E06811147C08B015B0111
:10A29000A40EB51E0A151B0509F43FC0F701C080C6
:10A2A000D180F80161918F016983C6016A830E94A0
:10A2B00054B66A81681729F1C6010E947DB6C601AD
:10A2C0000E9454B699818917E1F0E9EBFCE0849192
:10A2D0008F010F5F1F4F882321F00E94FD34F8018A
:10A2E000F6CFE7E0FDE084918F010F5F1F4F8823D9
:10A2F00021F00E94FD34F801F6CF81E080935E06E4
:10A300000CC0BE016F5F7F4FC40161D9F70180812E
:10A310009181019691838083BDCF0F900F90DF9143
:10A32000CF911F910F91FF90EF90DF90CF90BF9052
:10A33000AF909F908F900895AF92BF92CF92DF928F
:10A34000EF92FF920F931F93CF93DF931F92CDB79E
:10A35000DEB78C016B017A01590180915E06811193
:10A360001BC0F801808191810E9454B68983F60157
:10A3700081936F01BE016F5F7F4FC50128D9F8013E
:10A38000408151814F5F5F4F51834083F1E0EF1A6D
:10A39000F108E114F10429F70F90DF91CF911F919B
:10A3A0000F91FF90EF90DF90CF90BF90AF90089506
:10A3B000CF93DF93FC011682862F0E94FD34E0EFDD
:10A3C000FCE08491EF012196882321F00E94FD3466
:10A3D000FE01F7CFDF91CF9108950F931F93CF9395
:10A3E000DF93EC01862F0E94FD34EAECFCE08491BF
:10A3F0008F010F5F1F4F882321F00E94FD34F80169
:10A40000F6CF8E81882319F0EFEBFCE002C0E4EC7C
:10A41000FCE08491EF012196882321F00E94FD3415
:10A42000FE01F7CF8AE0DF91CF911F910F910C943D
:10A43000FD344F925F926F927F928F929F92AF9274
:10A44000BF92CF92DF92EF92FF920F931F93CF9321
:10A45000DF936C017B018A01E90180900A029090F0
:10A460000B02A0900C02B0900D02FA012081318104
:10A470004281538160910206709103068091040627
:10A48000909105060E948EB387FF2DC048805980A9
:10A490006A807B8020E030E0A901B201C3010E9404
:10A4A0008EB3811107C0ECE3F7E185919591A591F9
:10A4B000B49102C0C201D30180930A0290930B02AF
:10A4C000A0930C02B0930D02F80180819181A281CA
:10A4D000B3818093020690930306A0930406B09381
:10A4E00005060E94876F488059806A807B8020E043
:10A4F00030E0A901B201C3010E948EB3811108C0EE
:10A5000040903302509034026090350270903602D1
:10A51000C201D30180930A0290930B02A0930C0214
:10A52000B0930D02F60180819181A281B381809365
:10A53000FA059093FB05A093FC05B093FD05F70188
:10A5400080819181A281B3818093FE059093FF0564
:10A55000A0930006B09301060E94876FF801208146
:10A56000318142815381609102067091030680918E
:10A570000406909105060E9412BA18168CF5D88030
:10A58000E980FA80CB8120E030E0A9016D2D7E2D9D
:10A590008F2D9C2F0E948EB3811107C0ECE3F7E151
:10A5A00085919591A591B49104C08D2D9E2DAF2DCF
:10A5B000BC2F80930A0290930B02A0930C02B093DD
:10A5C0000D02F80180819181A281B38180930206FE
:10A5D00090930306A0930406B09305060E94876F2C
:10A5E0000E94345E80920A0290920B02A0920C02AA
:10A5F000B0920D02DF91CF911F910F91FF90EF90DC
:10A60000DF90CF90BF90AF909F908F907F906F9092
:10A610005F904F9008959A0142E056E00ACF9B0167
:10A62000AC016EEF75E08AEF95E003CF3F924F9259
:10A630005F926F927F928F929F92AF92BF92CF92D2
:10A64000DF92EF92FF920F931F93CF93DF93CDB7DB
:10A65000DEB7E8970FB6F894DEBF0FBECDBF5B0143
:10A660004A01FC018081813009F4D3C1823009F0B4
:10A6700020C180E090E0A6EEB2E4898B9A8BAB8B90
:10A68000BC8B80E090E0ADE2B3E48D8B9E8BAF8B12
:10A69000B88F80E090E0A0E8BFE3898F9A8FAB8FFE
:10A6A000BC8F80E090E0A0ECBFE78D8F9E8FAF8FD6
:10A6B000B8A3FB018081882309F4ABC10091060691
:10A6C0001091070620910806309109066091020654
:10A6D000709103068091040690910506C090FE05D6
:10A6E000D090FF05E0900006F09001064090FA053A
:10A6F0005090FB056090FC057090FD0549825A82E0
:10A700006B827C82CD82DE82EF82F88669877A87CF
:10A710008B879C870D871E872F87388B20E030E042
:10A7200040E85FE30E9412BA19A21AA21BA21CA25F
:10A7300087FD15C0AE014F5D5F4FBE016B5E7F4F61
:10A74000CE01419668DF19A21AA21BA21CA2BE016B
:10A750006F5D7F4FCE01499662DF312C5EC0BE0136
:10A760006F5D7F4FCE0149965ADF19A21AA21BA234
:10A770001CA2AE014F5D5F4FBE016B5E7F4FCE01ED
:10A78000419649DFEACFB801882777FD8095982F59
:10A790000E9494B326E331E642E85DE30E94F3B3FE
:10A7A0002B013C010E944DBAF401C080D180E280AF
:10A7B000F380A70196010E94F3B320E030E046EE5B
:10A7C00052E40E94ECB76DAB7EAB8FAB98AFC30188
:10A7D000B2010E94C5B8A70196010E94F3B320E020
:10A7E00030E04DE253E40E94ECB769AB7AAB8BAB3F
:10A7F0009CAB19A21AA21BA21CA2AE014F5D5F4F17
:10A80000BE016F5C7F4FCE01C59605DF0F5F1F4F06
:10A810000A30110509F0B7CF3394F501808138165D
:10A8200018F400E010E0AFCF19A21AA21BA21CA2DC
:10A83000AE014F5D5F4FBE016B5E7F4FCE01419613
:10A84000EADE29853A854B855C85698D7A8D8B8D0D
:10A850009C8D0E948EB319A21AA21BA21CA21816CC
:10A86000A4F0BE016F5D7F4FCE010996D8DE19A21C
:10A870001AA21BA21CA2AE014F5D5F4FBE016B5F0F
:10A880007F4FCE010196C7DEC4C0AE014F5D5F4F62
:10A89000BE016B5F7F4FCE010196BDDE19A21AA2E9
:10A8A0001BA21CA2BE016F5D7F4FCE010996B7DED1
:10A8B000B0C080E090E0A4E3B2E489A39AA3ABA384
:10A8C000BCA300E010E02DE233E40DA31EA32FA3F0
:10A8D00038A740E050E060E87FE349A75AA76BA79C
:10A8E0007CA780E090E0A0ECBFE78DA79EA7AFA774
:10A8F000B8ABC12CD12CE6EEEE2EE2E4FE2EC98AD6
:10A90000DA8AEB8AFC8A0D8B1E8B2F8B388F498F4E
:10A910005A8F6B8F7C8F8D8F9E8FAF8FB8A3809156
:10A92000060690910706A0910806B091090640918D
:10A93000020650910306609104067091050600918D
:10A94000FE051091FF052091000630910106C09090
:10A95000FA05D090FB05E090FC05F090FD05C9825A
:10A96000DA82EB82FC820D831E832F83388749872E
:10A970005A876B877C878D879E87AF87B88B19AA8C
:10A980001AAA1BAA1CAAAE014F5C5F4FBE016B5EE8
:10A990007F4FCE0141963FDE19AA1AAA1BAA1CAA14
:10A9A000BE016F5C7F4FCE01499639DE10E0212F4A
:10A9B00030E0F501808190E09595879519AA1AAA53
:10A9C0001BAA1CAA28173907C4F4AE014F5C5F4FBD
:10A9D000BE016B5D7F4FCE0181961DDE19AA1AAABA
:10A9E0001BAA1CAAAE014F5C5F4FBE016B5E7F4F7E
:10A9F000CE01419610DE1F5FDACF9E012F5C3F4FE4
:10AA0000AE01475F5F4FBE016B5F7F4FCE01019686
:10AA100010DDE8960FB6F894DEBF0FBECDBFDF9114
:10AA2000CF911F910F91FF90EF90DF90CF90BF904B
:10AA3000AF909F908F907F906F905F904F903F90DE
:10AA40000895CF92DF92EF92FF921F93CF93DF93FF
:10AA5000CDB7DEB72C970FB6F894DEBF0FBECDBFD3
:10AA6000182F8091ED05811709F468C080E090E00F
:10AA7000A0EAB0E48D839E83AF83B887C0900B04B7
:10AA8000D0900C04E0900D04F0900E0420E030E033
:10AA9000A901C701B6010E948EB387FF0CC0A701B0
:10AAA000960160E070E080EA90E40E94EBB76D836D
:10AAB0007E838F8398872091020630910306409110
:10AAC0000406509105066D817E818F8198850E94D4
:10AAD00012BA181654F419821A821B821C82BE0103
:10AAE0006F5F7F4FCE0105969ADD4091FA05509138
:10AAF000FB056091FC057091FD0549875A876B87BE
:10AB00007C874091FE055091FF0560910006709191
:10AB100001064D835E836F83788719821A821B82B8
:10AB20001C829E012F5F3F4F42E056E0BE016B5FEB
:10AB30007F4FCE0109967DDC1093ED0580E02C96C9
:10AB40000FB6F894DEBF0FBECDBFDF91CF911F913E
:10AB5000FF90EF90DF90CF9008950F931F93CF93C6
:10AB6000DF93CDB7DEB728970FB6F894DEBF0FBEE0
:10AB7000CDBF00E010E020E830EC0D831E832F8372
:10AB8000388720E030E040E752E40E94C8B869838B
:10AB90007A838B839C83BE016F5F7F4FCE010596C6
:10ABA0003EDD10915706109257060E94A03384E3B1
:10ABB00097E00E947E2D40913C0750913D076091A7
:10ABC0003E0770913F07409302065093030660933F
:10ABD0000406709305060E941B6112FB112710F9F1
:10ABE00081E0812728960FB6F894DEBF0FBECDBF57
:10ABF000DF91CF911F910F9108952F923F924F9225
:10AC00005F926F927F928F929F92AF92BF92CF92FC
:10AC1000DF92EF92FF920F931F93CF93DF93CDB705
:10AC2000DEB768970FB6F894DEBF0FBECDBF9C8B22
:10AC30008B8B1B014D8B2E8BFC016081718182817E
:10AC400093816D877E878F87988BF101C080D1803B
:10AC5000E280F380C986DA86EB86FC864090F403B6
:10AC60005090F5036090F6037090F7032091F00385
:10AC70003091F1034091F2035091F3030E94EBB73E
:10AC80004B015C012FE632E143E85AEB0E9412BA15
:10AC900087FD24C022E430E045E253E4C501B4015D
:10ACA0000E948EB31816D4F0A3019201C701B60119
:10ACB0000E94EBB76B017C0121E338E040EC50ECE3
:10ACC0000E9412BA87FD0AC022E430E04FE353E449
:10ACD000C701B6010E948EB318162CF4612C712C9A
:10ACE00000EC1FE70DC2C0900A02D0900B02E0906A
:10ACF0000C02F0900D0280916C06811107C08091CA
:10AD0000300280936B0681E080936C068091330261
:10AD100090913402A0913502B091360280930A02DC
:10AD200090930B02A0930C02B0930D0219821A8229
:10AD30001B821C82AE014F5F5F4FBE01675F7F4F7A
:10AD4000CE010D9668DC81E07CDE811163C10E943A
:10AD5000A43904E010E0812C912CA12CB1E4BB2E8D
:10AD6000412C512C80E2682E81E4782E60E070E066
:10AD700080EF93E4F2DE882309F469C001501109E1
:10AD80000115110589F5E0E6FFE084918F010F5F61
:10AD90001F4F882321F00E94FD34F801F6CF80E098
:10ADA00090E0A0E0B1E48D839E83AF83B88780E01C
:10ADB00090E0A8ECB2E489839A83AB83BC83BE01A4
:10ADC0006B5F7F4FCE0101962ADC1092060610922F
:10ADD000070610920806109209060E94876FD1D8C4
:10ADE00043D781E59FE086C0E9E7FFE084919F01BA
:10ADF0002F5F3F4F882341F02F8B388F0E94FD3407
:10AE00002F89388DF901F2CF8D829E82AF82B8866C
:10AE100049825A826B827C82BE016B5F7F4FCE017A
:10AE20000196FDDB1A8A19821A821B821C82FCE0C1
:10AE3000F98B1D829E012E5E3F4FAE014F5F5F4F2B
:10AE4000BE016F5E7F4FCE010596F0DB8FCF80E0B5
:10AE500090E0A0E0B1E48D839E83AF83B88720E0CB
:10AE600030E040EA50E46091020670910306809160
:10AE70000406909105060E94ECB769837A838B8360
:10AE80009C83BE016B5F7F4FCE010196C8DB04E05F
:10AE900010E0812C912CF0E8AF2EFFE3BF2E412C67
:10AEA000512CA0E26A2EA1E47A2E48C080E090E006
:10AEB000A0E0B1E48D839E83AF83B88780E090E00B
:10AEC000A8ECB2E489839A83AB83BC83BE016B5F39
:10AED0007F4FCE010196A3DB109206061092070663
:10AEE00010920806109209060E94876F4AD8BCD6B5
:10AEF0008FE19FE00E94BAA78D829E82AF82B886C2
:10AF000049825A826B827C82BE016B5F7F4FCE0189
:10AF1000019685DB1A8A19821A821B821C828CE0B8
:10AF2000898B1D829E012E5E3F4FAE014F5F5F4FAA
:10AF3000BE016F5E7F4FCE01059678DB60E070E06A
:10AF400080E792E40ADE882319F101501109011506
:10AF5000110569F4EEE2FFE084918F010F5F1F4F4E
:10AF6000882309F4A3CF0E94FD34F801F5CFE7E46C
:10AF7000FFE084919F012F5F3F4F882309F4BCCFEE
:10AF80002F8B388F0E94FD342F89388DF901F1CF36
:10AF90008090020690900306A0900406B0900506EB
:10AFA0002091F8033091F9034091FA035091FB038B
:10AFB000C501B4010E94EBB720910B0430910C0441
:10AFC00040910D0450910E040E94ECB73B018C019E
:10AFD0009D8991111BC080E090E0A0E0B1E48983DD
:10AFE0009A83AB83BC8320E030E040EA50E4C501A3
:10AFF000B4010E94ECB76D837E838F839887BE0176
:10B000006F5F7F4FCE0105960ADB08C080E019DD37
:10B01000882321F0612C712C00EC1FE780916B06D6
:10B0200080933002EE89E33008F440C0EDE9FFE0A0
:10B0300084915F019FEFA91AB90A882321F00E9429
:10B04000FD34F501F5CFEB89FC8960817181828146
:10B05000938143E00E94B377E8E9FFE084915F01C8
:10B060009FEFA91AB90A882321F00E94FD34F50147
:10B07000F5CFF101608171818281938143E00E946B
:10B08000B377E3E9FFE084915F019FEFA91AB90A62
:10B09000882321F00E94FD34F501F5CF43E0B30190
:10B0A000C8010E94B3778AE00E94FD34C0920A0270
:10B0B000D0920B02E0920C02F0920D029301A801D3
:10B0C000B301C8010E9498BA8823D1F0E5EEFAE0F6
:10B0D00084917F019FEFE91AF90A882321F00E94E9
:10B0E000FD34F701F5CFE3E8FFE084917F019FEFA6
:10B0F000E91AF90A882321F00E94FD34F701F5CFFF
:10B10000B301C80168960FB6F894DEBF0FBECDBF7D
:10B11000DF91CF911F910F91FF90EF90DF90CF9033
:10B12000BF90AF909F908F907F906F905F904F9067
:10B130003F902F9008952F923F924F925F926F927F
:10B140007F928F929F92AF92BF92CF92DF92EF92B7
:10B15000FF920F931F93CF93DF93CDB7DEB7CC55FC
:10B16000D1090FB6F894DEBF0FBECDBF2DB73EB7E5
:10B170006B963FAF2EAF6B9761961FAE1EAE619779
:10B1800084E690E02F969FAF8EAF2F979E01215BB4
:10B190003F4F44E050E0BE016F5B7F4FCE01835BC9
:10B1A0009F4FCAD89E01215B3F4F42E050E0BE0155
:10B1B000655B7F4FCE01835B9F4FBED843E050E07D
:10B1C000BE016F5B7F4F8FEF92E00E94EEBB892B39
:10B1D00009F439C022968FAD2297863539F08FE376
:10B1E00022968FAF229723961FAE2397E9EBFCE0C0
:10B1F00084918F010F5F1F4F882321F00E94FD343F
:10B20000F801F6CFE6E0FFE084918F010F5F1F4F5A
:10B21000882321F00E94FD34F801F6CFBE016F5B58
:10B220007F4F8DEF9EE00E940435EFEEFEE08491AB
:10B230008F010F5F1F4F882321F00E94FD34F8011A
:10B24000F6CF81D6E7C46DB67EB621961CAE1DAE94
:10B250001EAE1FAE219761961FAE1EAE61979E0176
:10B26000215B3F4F41E050E0BE01695A7F4FCE0164
:10B27000835B9F4F61D880E1E3E5F2E0DE019196C8
:10B2800001900D928A95E1F780E1E3E6F2E0DE01BC
:10B29000519601900D928A95E1F780E1E3E7F2E0A3
:10B2A0009E012F5F3F4F7901D90101900D928A9540
:10B2B000E1F76896CFAC6897D12C33E0C30ED11C70
:10B2C000CC0CDD1CCC0CDD1C8DB79EB78C199D09F8
:10B2D0000FB6F8949EBF0FBE8DBFEDB7FEB7319687
:10B2E0004F012DB73EB72C193D090FB6F8943EBF5C
:10B2F0000FBE2DBF8DB79EB701965C01EDB7FEB7AF
:10B30000EC19FD090FB6F894FEBF0FBEEDBF0DB7E7
:10B310001EB70F5F1F4F9E01215B3F4FA601B40177
:10B32000CE01835B9F4F08D89E01215B3F4FA60152
:10B33000B501CE01835B9F4F0E949C519E01215B12
:10B340003F4FA601B801CE01835B9F4F0E949C51E5
:10B3500068964FAD689750E04E5F5F4F21EA33E04B
:10B360006D963FAF2EAF6D9761EB73E0A9E8B3E048
:10B3700080E090E020E030E04217530714F06401D1
:10B3800005C0F1E2CF2ED12CCC0EDD1EC80ED91E89
:10B39000F60120803180428053802D923D924D9263
:10B3A0005D924217530714F0650105C0E1E1CE2E0E
:10B3B000D12CCC0EDD1EC80ED91EF60120803180A6
:10B3C00042805380FB012192319241925192BF0100
:10B3D0004217530714F0680101C06701C80ED91E57
:10B3E000F60120803180428053806D96EEADFFAD36
:10B3F0006D9721923192419251926D96FFAFEEAFCF
:10B400006D972F5F3F4F04962430310509F0B4CF7C
:10B410009E01215B3F4F44E050E069EC73E0CE01B8
:10B42000835B9F4F0E949C519E01215B3F4F44E0F4
:10B4300050E061EC73E0CE01835B9F4F0E949C5112
:10B440009E01215B3F4F44E050E065EC73E0CE018C
:10B45000835B9F4F0E949C519E01215B3F4F44E0C4
:10B4600050E067E676E0CE01835B9F4F0E949C51DF
:10B470009E01215B3F4F44E050E063E676E0CE0161
:10B48000835B9F4F0E949C519E01215B3F4F44E094
:10B4900050E06FE576E0CE01835B9F4F0E949C51A8
:10B4A0009E01215B3F4F40E150E069E773E0CE0130
:10B4B000835B9F4F0E949C519E01215B3F4F4CE05C
:10B4C00050E06EEE75E0CE01835B9F4F0E949C5171
:10B4D0009E01215B3F4F44E050E0BE01635C7F4F23
:10B4E000CE01835B9F4F0E949C519E01215B3F4F89
:10B4F00041E050E0BE016A5A7F4FCE01835B9F4F0F
:10B500000E949C519E01215B3F4F44E050E0BE01F0
:10B51000635C7F4FCE01835B9F4F0E949C519E01D5
:10B52000215B3F4F41E050E0BE016B5A7F4FCE019F
:10B53000835B9F4F0E949C519E01215B3F4F41E0E6
:10B5400050E0BE016C5A7F4FCE01835B9F4F0E943B
:10B550009C516696EFAC669765968FAD6597E89EB1
:10B560007001112400E010E00E151F0581F09E010E
:10B57000215B3F4F44E050E0BE01635C7F4FCE0152
:10B58000835B9F4F0E949C510F5F1F4FEDCF6196D1
:10B590000EAD1FAD61972F968EAD9FAD2F979093F7
:10B5A0002F0280932E029E01215B3F4F44E050E02A
:10B5B0006BE074E0CE01835B9F4F0E949C516196CB
:10B5C0001FAF0EAF61979E01215B3F4F44E250E0F9
:10B5D00065EE7EE0CE01835B9F4F0E949C519E01F1
:10B5E000215B3F4F41E050E0BE016D5A7F4FCE01DD
:10B5F000835B9F4F0E949C519E01215B3F4F41E026
:10B6000050E0BE016E5A7F4FCE01835B9F4F0E9478
:10B610009C519E01215B3F4F44E050E0BE016B5CBA
:10B620007F4FCE01835B9F4F0E949C519E01215B07
:10B630003F4F44E050E0BE016F5C7F4FCE01835B23
:10B640009F4F0E949C516496EFAC649763968FADB8
:10B650006397E89E7001112400E010E09E01215BD9
:10B660003F4F0E151F0569F044E050E0BE01635CDA
:10B670007F4FCE01835B9F4F0E949C510F5F1F4FF6
:10B68000EDCF41E050E0BE01685A7F4FCE01835BB1
:10B690009F4F0E949C519E01215B3F4F44E050E030
:10B6A000BE01635C7F4FCE01835B9F4F0E949C5124
:10B6B0009E01215B3F4F41E050E0BE016F5A7F4F3A
:10B6C000CE01835B9F4F0E949C5121961CAE1DAE04
:10B6D0001EAE1FAE21971DE011509E01215B3F4F12
:10B6E00044E050E0BE01112341F0635C7F4FCE0186
:10B6F000835B9F4F0E949C51EFCF675C7F4FCE01D1
:10B70000835B9F4F0E949C519E01215B3F4F44E011
:10B7100050E0BE016B5C7F4FCE01835B9F4F0E9468
:10B720009C519E01215B3F4F44E050E0BE016F5CA5
:10B730007F4FCE01835B9F4F0E949C519E01215BF6
:10B740003F4F44E050E0BE01635C7F4FCE01835B1E
:10B750009F4F0E949C51112311F004E03EC021969E
:10B76000CCACDDACEEACFFAC219720E030E84BE395
:10B7700055E4C701B6010E948EB3882371F3C092CD
:10B78000D603D092D703E092D803F092D9039E015A
:10B79000215B3F4F44E050E062ED73E0CE01835BFC
:10B7A0009F4F0E949C519E01215B3F4F44E050E01F
:10B7B0006EEC73E0CE01835B9F4F0E949C519E0113
:10B7C000215B3F4F44E050E0BE01635C7F4FCE0100
:10B7D000835B9F4F0E949C5110C0015071F09E01ED
:10B7E000215B3F4F44E050E0BE01635C7F4FCE01E0
:10B7F000835B9F4F0E949C51F0CF1F5F153009F073
:10B800009DCF9E01215B3F4F42E050E0BE01675B50
:10B810007F4FCE01835B9F4F0E949C519E01215B15
:10B820003F4F44E050E0BE01635C7F4FCE01835B3D
:10B830009F4F0E949C512196CCACDDACEEACFFAC8E
:10B84000219720E030E84BE355E4C701B6010E94A0
:10B850008EB3882301F1C092E203D092E303E09219
:10B86000E403F092E5039E01215B3F4F44E050E08A
:10B870006EED73E0CE01835B9F4F0E949C519E0151
:10B88000215B3F4F44E050E06AED73E0CE01835B03
:10B890009F4F0E949C519E01215B3F4F42E050E030
:10B8A000BE01695B7F4FCE01835B9F4F0E949C511D
:10B8B0009E01215B3F4F41E050E0BE01685A7F4F3F
:10B8C000CE01835B9F4F0E949C5119E011509E0155
:10B8D000215B3F4F112359F044E050E0BE01635C0F
:10B8E0007F4FCE01835B9F4F0E949C51EFCF41E081
:10B8F00050E060EA73E0CE01835B9F4F0E949C5151
:10B900009E01215B3F4F44E050E0BE01635C7F4FEE
:10B91000CE01835B9F4F0E949C5111110EC0219656
:10B920008CAD9DADAEADBFAD219780939C03909340
:10B930009D03A0939E03B0939F031F5F153001F7F3
:10B940009E01215B3F4F42E050E0BE016B5B7F4FA9
:10B95000CE01835B9F4F0E949C5127966EAD7FADB9
:10B96000279780E79EE00E94DD749E01215B3F4F98
:10B9700042E050E0BE016B5B7F4FCE01835B9F4F87
:10B980000E949C5127966EAD7FAD27978BEF9DE06F
:10B990000E94DD749E01215B3F4F42E050E0BE01FA
:10B9A0006B5B7F4FCE01835B9F4F0E949C5127961C
:10B9B0006EAD7FAD279786E89DE00E94DD749E0105
:10B9C000215B3F4F42E050E0BE016B5B7F4FCE01F9
:10B9D000835B9F4F0E949C519E01215B3F4F42E041
:10B9E00050E0BE016B5B7F4FCE01835B9F4F0E9497
:10B9F0009C519E01215B3F4F42E050E0BE016B5BDA
:10BA00007F4FCE01835B9F4F0E949C519E01215B23
:10BA10003F4F42E050E0BE016B5B7F4FCE01835B46
:10BA20009F4F0E949C5127966EAD7FAD279781E175
:10BA30009DE00E94DD749E01215B3F4F42E050E09B
:10BA4000BE016B5B7F4FCE01835B9F4F0E949C5179
:10BA50009E01215B3F4F42E050E0BE016B5B7F4F98
:10BA6000CE01835B9F4F0E949C519E01215B3F4F03
:10BA700042E050E0BE016B5B7F4FCE01835B9F4F86
:10BA80000E949C519E01215B3F4F42E050E0BE016D
:10BA90006B5B7F4FCE01835B9F4F0E949C519E0149
:10BAA000215B3F4F44E050E0BE01635C7F4FCE011D
:10BAB000835B9F4F0E949C519E01215B3F4F44E05E
:10BAC00050E0BE01635C7F4FCE01835B9F4F0E94BD
:10BAD0009C5113E0115088F0F4E01F9FB001112435
:10BAE000615F7B4F9E01215B3F4F44E050E0CE0100
:10BAF000835B9F4F0E949C51EDCF61962EAD3FAD71
:10BB000061972D968EAD9FAD2D972817390709F0B7
:10BB100039C0F9D1E9EBFCE084918F010F5F1F4F31
:10BB2000811103C00FEF12E004C00E94FD34F80140
:10BB3000F3CFF80181918F01882319F00E94FD3421
:10BB4000F8CF2F966EAD7FAD2F976456710982EDB9
:10BB50009EE00E941E7961964EAD5FAD619760E0F8
:10BB600070E085EC9EE00E947177E2ECFEE084914B
:10BB70008F010F5F1F4F882309F447C00E94FD34D7
:10BB8000F801F5CFE5EEFAE084918F010F5F1F4FCA
:10BB9000882321F00E94FD34F801F6CFE2EAFEE0AE
:10BBA00084918F010F5F1F4F882321F00E94FD3485
:10BBB000F801F6CF2D966EAD7FAD2D9780E090E029
:10BBC0004AE00E940077EDE9FEE084918F010F5F6B
:10BBD0001F4F882321F00E94FD34F801F6CF6196B3
:10BBE0006EAD7FAD619780E090E04AE00E94007703
:10BBF000EDE8FEE084918F010F5F1F4F882321F055
:10BC00000E94FD34F801F6CF9ED10FB6F8947EBEA7
:10BC10000FBE6DBE80E00E94D48290915E0681E0EE
:10BC200089276B962EAD3FAD6B970FB6F8943EBF4C
:10BC30000FBE2DBFC45ADF4F0FB6F894DEBF0FBE44
:10BC4000CDBFDF91CF911F910F91FF90EF90DF90CB
:10BC5000CF90BF90AF909F908F907F906F905F90AC
:10BC60004F903F902F9008950E94D837882319F065
:10BC70000E940872F9CF08952F923F924F925F92DF
:10BC80006F927F928F929F92AF92BF92CF92DF92EC
:10BC9000EF92FF920F931F93CF93DF9300D01F92E9
:10BCA000CDB7DEB77B018A0119012091890330915C
:10BCB0008A0340918B0350918C03DC016D917D913F
:10BCC0008D919C910E94F3B30E941DBA4B015C01BF
:10BCD00060931D0F70931E0F80931F0F9093200F82
:10BCE00020918D0330918E0340918F0350919003EA
:10BCF000F70160817181828193810E94F3B30E9478
:10BD00001DBA6B017C016093210F7093220F809309
:10BD1000230F9093240F209191033091920340912F
:10BD2000930350919403D8016D917D918D919C91D5
:10BD30000E94F3B30E941DBA2B013C016093250FB2
:10BD40007093260F8093270F9093280F20919503CF
:10BD5000309196034091970350919803F1016081CF
:10BD60007181828193810E94F3B30E941DBA609316
:10BD7000290F70932A0F80932B0F90932C0F6983B8
:10BD80007A838B839C8370DF2FB7F8948092940C16
:10BD90009092950CA092960CB092970CC092980C31
:10BDA000D092990CE0929A0CF0929B0C40929C0CD1
:10BDB00050929D0C60929E0C70929F0C69817A81CA
:10BDC0008B819C816093A00C7093A10C8093A20C3A
:10BDD0009093A30C2FBF1092090F10920A0F10928C
:10BDE0000B0F10920C0F80E1EDE0FFE0DF011D92E0
:10BDF0008A95E9F70F900F900F900F90DF91CF91F8
:10BE00001F910F91FF90EF90DF90CF90BF90AF9078
:10BE10009F908F907F906F905F904F903F902F906A
:10BE20000895EF92FF920F931F93CF93DF93CDB7B7
:10BE3000DEB72C970FB6F894DEBF0FBECDBF09E872
:10BE400013E08BE3E82E86E0F82EF8012191319182
:10BE5000419151918F0160E070E080E89FE30E9482
:10BE6000C8B8F70161937193819391937F01F3E0D7
:10BE700009391F0751F78091FA059091FB05A091B0
:10BE8000FC05B091FD0589839A83AB83BC838091C7
:10BE9000FE059091FF05A0910006B09101068D83EB
:10BEA0009E83AF83B8878091020690910306A0918C
:10BEB0000406B091050689879A87AB87BC87AE01D7
:10BEC000475F5F4FBE016B5F7F4FCE0101960E94BF
:10BED000EF2E26E036E0AE01475F5F4FBE016B5F9D
:10BEE0007F4FCE010196C8DE0E9493342C960FB688
:10BEF000F894DEBF0FBECDBFDF91CF911F910F91A0
:10BF0000FF90EF9008950E9493348BDF0E943436A7
:10BF100080E00E94D83681E00E94D83682E00E94FC
:10BF2000D83680910B0490910C04A0910D04B0912F
:10BF30000E048093220290932302A0932402B093D4
:10BF400025020C9461A60F931F93CF93DF93CDB777
:10BF5000DEB72C970FB6F894DEBF0FBECDBF09E851
:10BF600013E061EB73E041EA53E020E030E0F901D7
:10BF7000EE5DFF4E85919591A591B491F801819365
:10BF80009193A193B1938F01F901EE5EFF4E8591DC
:10BF90009591A591B491FB0181939193A193B19354
:10BFA000BF01F901EE5FFF4E85919591A591B49186
:10BFB000FA0181939193A193B193AF012C5F3F4F0D
:10BFC00020313105A1F680E090E0AAEFB4E480933F
:10BFD000C9039093CA03A093CB03B093CC0340E072
:10BFE00050E86BE375E44093C1035093C203609340
:10BFF000C3037093C4038093C5039093C603A093B7
:10C00000C703B093C8031092670610926806109297
:10C01000690610926A0680E29EE4A0E0B0E0809398
:10C020005F0690936006A0936106B093620610923B
:10C03000630610926406109265061092660680E010
:10C0400090E0A0E4B1E48093790390937A03A09305
:10C050007B03B0937C0380937D0390937E03A09336
:10C060007F03B09380038DEC9CECACECBEE380933B
:10C07000810390938203A0938303B093840380E0B1
:10C0800090E0A0E2B1E48093850390938603A093AF
:10C090008703B09388031CE0EEEEF5E0DF01812F0B
:10C0A0001D928A95E9F70E9488A689E891E4A0EBA1
:10C0B000BFEB80930B0490930C04A0930D04B093FA
:10C0C0000E0487ED93EAAEE9B1E48093D603909332
:10C0D000D703A093D803B093D90380E898E5A0E8EC
:10C0E000BEE38093D2039093D303A093D403B09381
:10C0F000D50381E09DECA3ECB3E48093CE03909351
:10C10000CF03A093D003B093D1038DE39AE2A0ECC8
:10C11000B3E48093E2039093E303A093E403B0932A
:10C12000E50387E790E3ADE3B1E48093DE0390930A
:10C13000DF03A093E003B093E10389ED9CE2A3E465
:10C14000B5E48093DA039093DB03A093DC03B09310
:10C15000DD031092A00380E090E0A0E4B0E48093BF
:10C160009C0390939D03A0939E03B0939F03109212
:10C17000E90510929B0360EC73E080E79EE00E946B
:10C18000DD7460EC73E08BEF9DE00E94DD7460EC89
:10C1900073E086E89DE00E94DD7462EE74E081E168
:10C1A0009DE00E94DD74E3E8F2E0DE01119601906B
:10C1B0000D921A95E1F713E01150C8F0A4E01A9F10
:10C1C00090011124E1E0F0E0EC0FFD1FE20FF31FFE
:10C1D0006081718182819381F901E15FFB4F60830E
:10C1E000718382839383812F0E9421A6E5CF8BDE0A
:10C1F000E9EBFCE084918F010F5F1F4F882321F052
:10C200000E94FD34F801F6CFEFEDFFE084918F013D
:10C210000F5F1F4F882321F00E94FD34F801F6CFF5
:10C220002C960FB6F894DEBF0FBECDBFDF91CF9135
:10C230001F910F9108950F931F93CF93DF93CDB765
:10C24000DEB72C970FB6F894DEBF0FBECDBF80913E
:10C25000020690910306A0910406B0910506409154
:10C26000FE055091FF056091000670910106009156
:10C27000FA051091FB052091FC053091FD0509831D
:10C280001A832B833C834D835E836F8378878987F2
:10C290009A87AB87BC87AE01475F5F4FBE016B5F7C
:10C2A0007F4FCE0101960E94EF2E26E036E0AE01D0
:10C2B000475F5F4FBE016B5F7F4FCE010196DCDCB5
:10C2C0002C960FB6F894DEBF0FBECDBFDF91CF9195
:10C2D0001F910F9108959F92AF92BF92CF92DF92DC
:10C2E000EF92FF920F931F93CF93DF939CEEA92EB3
:10C2F00092E0B92E0AEF15E0CEEED5E0912CF501D3
:10C3000081915F010E9442378823F9F00E94033631
:10C310006B017C01288139814A815B810E94EBB7E6
:10C320009B01AC01F80160817181828193810E943F
:10C33000ECB7F8016083718382839383C882D982CA
:10C34000EA82FB82892D0E94D83693940C5F1F4F9E
:10C350002496F3E09F12D3CF6EDFDF91CF911F9130
:10C360000F91FF90EF90DF90CF90BF90AF909F9094
:10C370000C9466782F923F924F925F926F927F92C9
:10C380008F929F92AF92BF92CF92DF92EF92FF92E5
:10C390000F931F93CF93DF93CDB7DEB7C058D1096A
:10C3A0000FB6F894DEBF0FBECDBF5B014A01390165
:10C3B0002896EFAE2897FBAE24960FAF24972C96C5
:10C3C0001FAF2C973C2C2091890330918A03409118
:10C3D0008B0350918C03DC016D917D918D919C912B
:10C3E0000E94F3B30E941DBAE8966CAF7DAF8EAF8A
:10C3F0009FAFE89720918D0330918E0340918F037A
:10C4000050919003F50160817181828193810E9436
:10C41000F3B30E941DBAEC966CAF7DAF8EAF9FAFA9
:10C42000EC972091910330919203409193035091A6
:10C430009403D4016D917D918D919C910E94F3B3F1
:10C440000E941DBAC458DF4F688379838A839B8317
:10C45000CC57D0402091950330919603409197039B
:10C4600050919803F30160817181828193810E94D0
:10C47000F3B30E941DBAA3966CAF7DAF8EAF9FAF92
:10C48000A39780911D0F90911E0FA0911F0FB09147
:10C49000200FE8968CAC9DACAEACBFACE897881A88
:10C4A000990AAA0ABB0A8FAA98AEA9AEBAAE809121
:10C4B000210F9091220FA091230FB091240FEC96A1
:10C4C0008CAC9DACAEACBFACEC97881A990AAA0AAA
:10C4D000BB0A8BAA9CAAADAABEAA8091250F9091F7
:10C4E000260FA091270FB091280FC458DF4F488026
:10C4F00059806A807B80CC57D040481A590A6A0A12
:10C500007B0A8091260483FF0EC0A3968CAC9DAC61
:10C51000AEACBFACA3978092290F90922A0FA09245
:10C520002B0FB0922C0F8091290F90912A0FA09180
:10C530002B0FB0912C0FA3968CAC9DACAEACBFACC6
:10C54000A397881A990AAA0ABB0A09F48BC080919A
:10C55000CD03811141C060911402709115028827AA
:10C5600077FD8095982F0E9494B39B01AC01609158
:10C57000E6037091E7038091E8039091E9030E943C
:10C580008EB387FF29C0A3968CAC9DACAEACBFAC7C
:10C59000A3978092290F90922A0FA0922B0FB0920E
:10C5A0002C0FE9EBFCE084918F010F5F1F4F882374
:10C5B00021F00E94FD34F801F6CFE4ECFFE0849115
:10C5C0008F010F5F1F4F882321F00E94FD34F80177
:10C5D000F6CF812C912C540175016401B7FE07C080
:10C5E000CC24DD247601C818D908EA08FB0860913C
:10C5F00095037091960380919703909198030E9400
:10C6000030B99B01AC01A8ECB0E00E94D2B76C1528
:10C610007D058E059F054CF5A3968CAC9DACAEAC0C
:10C62000BFACA3978092290F90922A0FA0922B0F54
:10C63000B0922C0FE9EBFCE084918F010F5F1F4F4C
:10C64000882321F00E94FD34F801F6CFE5EAFFE0EF
:10C6500084918F010F5F1F4F882321F00E94FD34CA
:10C66000F801F6CF812C912C54018FA998ADA9AD7A
:10C67000BAAD8827B7FD83959927AA27BB27082F2E
:10C68000282E2BA93CA94DA95EA957FF03C0382F1E
:10C690003260232E77FE03C0422D4460242EB7FE65
:10C6A00003C0522D5860252E8091820681112BC027
:10C6B0008091EF03882339F180918106122D18278C
:10C6C0002FA938AD49AD5AAD232B242B252B09F4C6
:10C6D0001E7F2BA93CA94DA95EA9232B242B252B1A
:10C6E00009F41D7F411451046104710409F41B7F96
:10C6F00081149104A104B10409F4177F8127809368
:10C700008106111119C1032D10E0C501B4010E9469
:10C7100094B3F801EE0FFF1FEE0FFF1FE358F94F20
:10C7200020813181428153810E94F3B36B017C01EE
:10C73000F801EE0FFF1FEF5CFD4F608171818827CC
:10C7400077FD8095982F0E9494B39B01AC01C7019F
:10C75000B6010E94F3B32AE037ED43E25CE30E94A6
:10C76000F3B36B017C0120E030E0A9010E9412BA12
:10C7700018164CF420E030E040E05FE3C701B6015A
:10C780000E94ECB708C0A701960160E070E080E06D
:10C790009FE30E94EBB70E9430B923966CAF7DAF48
:10C7A0008EAF9FAF239780902D0F282D2F5F2F7076
:10C7B0006D962FAF6D9780912E0F6D968FAC6D9704
:10C7C000881103C00E940872F6CF80912D0F2DE4CE
:10C7D000829F50011124A5014C53584F58AB4FA7CD
:10C7E000DA011C9292962C920FA918AD29AD3AADA0
:10C7F00037FF07C030952095109501951F4F2F4F9B
:10C800003F4FEFA5F8A902831383248335838BA9B7
:10C810009CA9ADA9BEA9B7FF07C0B095A0959095FA
:10C8200081959F4FAF4FBF4FEFA5F8A986839783A0
:10C83000A087B187B301A20177FE07C0442755271F
:10C84000BA014419550966097709EFA5F8A9428785
:10C8500053876487758723968CAC9DACAEACBFAC18
:10C86000239786869786A08AB18A80179107A207A8
:10C87000B30714F4D901C80184179507A607B707B1
:10C8800014F4DB01CA0123968CAC9DACAEACBFACFA
:10C89000239788169906AA06BB0614F0D501C40191
:10C8A000EFA5F8A9828B938BA48BB58B0697A10576
:10C8B000B10510F40C946D6F809163039091640343
:10C8C000E95BFF4F91838083AFA5B8A911963C9295
:10C8D000012B022B032B09F01798EFA5F8A98681ED
:10C8E0009781A085B185892B8A2B8B2B09F016980F
:10C8F000EFA5F8A982859385A485B585892B8A2B18
:10C900008B2B09F0159823968CAC9DACAEACBFACCC
:10C91000239789288A288B2809F45FC180917C0697
:10C92000882319F0815080937C0631104DC11498F2
:10C9300080E280937C0648C180E1EDE1FFE0DE010A
:10C94000119601900D928A95E1F710FF1FC020E02B
:10C9500030E0A9016091890370918A0380918B0373
:10C9600090918C030E94F3B3011105C020E030E0E8
:10C9700040E85FE304C020E030E040E85FEB0E9465
:10C98000F3B30E9430B96B017C0103C0C12CD12CE0
:10C99000760111FF25C020E030E0A90160918D03F0
:10C9A00070918E0380918F03909190030E94F3B356
:10C9B0002BA93CA94DA95EA957FF05C020E030E096
:10C9C00040E85FEB04C020E030E040E85FE30E9415
:10C9D000F3B30E9430B96FA778AB89AB9AAB04C0B0
:10C9E0001FA618AA19AA1AAA12FF24C023E333E328
:10C9F00043EB5EE360919103709192038091930306
:10CA0000909194030E94F3B377FE05C020E030E0DC
:10CA100040E85FEB04C020E030E040E85FE30E94C4
:10CA2000F3B30E9430B923966CAF7DAF8EAF9FAF4A
:10CA3000239706C023961CAE1DAE1EAE1FAE2397D5
:10CA400013FF1FC020E030E0A901609195037091B1
:10CA5000960380919703909198030E94F3B3B7FED9
:10CA600005C020E030E040E85FEB04C020E030E0AB
:10CA700040E85FE30E94F3B30E9430B98B019C0150
:10CA800003C000E010E0980181E08093820660918D
:10CA9000290F70912A0F80912B0F90912C0F600F0E
:10CAA000711F821F931F0E9494B3209195033091B0
:10CAB000960340919703509198030E94C8B869A7C4
:10CAC0007AA78BA79CA76091250F7091260F809164
:10CAD000270F9091280F23962CAD3DAD4EAD5FAD45
:10CAE0002397620F731F841F951F0E9494B3209198
:10CAF00091033091920340919303509194030E94CB
:10CB0000C8B86DA37EA38FA398A76091210F7091E1
:10CB1000220F8091230F9091240F2FA538A949A9A6
:10CB20005AA9620F731F841F951F0E9494B320910E
:10CB30008D0330918E0340918F03509190030E949A
:10CB4000C8B869A37AA38BA39CA360911D0F7091B1
:10CB50001E0F80911F0F9091200F6C0D7D1D8E1D5B
:10CB60009F1D0E9494B32091890330918A034091C4
:10CB70008B0350918C030E94C8B8698B7A8B8B8B86
:10CB80009C8BC32C2896EFAC2897FBAC24960FAD5A
:10CB900024972C961FAD2C979E01275D3F4FAE0129
:10CBA0004B5D5F4FBE016F5D7F4FCE014196E2DB73
:10CBB0001092820680E1FE013196ADE1BFE0019066
:10CBC0000D928A95E1F79FCD309067062090680618
:10CBD0000091690610916A0608C0309063062090A3
:10CBE00064060091650610916606232D322DA8017A
:10CBF00028966FAD28977BAD24968FAD24972C9601
:10CC00009FAD2C970E948EB387FD02C00C94616F7C
:10CC10006FA978AD89AD9AAD0E9494B320913B067F
:10CC200030913C0640913D0650913E060E94F3B380
:10CC30006FAB78AF89AF9AAF698B7A8B8B8B9C8BFC
:10CC40006BA97CA98DA99EA90E9494B320913F064F
:10CC50003091400640914106509142060E94F3B344
:10CC60004B015C016D8B7E8B8F8B988FC301B20162
:10CC70000E9494B3209143063091440640914506AA
:10CC8000509146060E94F3B32B013C01698F7A8FC5
:10CC90008B8F9C8F20914706309148064091490622
:10CCA00050914A06C701B6010E94F3B36D8F7E8F83
:10CCB0008F8F98A3AFA5B8A912962D913D914D9154
:10CCC0005C9115972BAB3CAB4DAB5EAB2630310581
:10CCD0004105510514F51696CD90DD90ED90FC9030
:10CCE0001997B6E0CB16D104E104F104B4F4EFA532
:10CCF000F8A9C284D384E484F584F6E0CF16D10485
:10CD0000E104F10454F4DC01CB01BF77EFA5F8A9ED
:10CD100087A790ABA1ABB2AB2EC02FA938AD49AD60
:10CD20005AADCA01B9010E94F3B36B017C01A501A0
:10CD30009401C501B4010E94F3B39B01AC01C7018A
:10CD4000B6010E94ECB74B015C01A3019201C30143
:10CD5000B2010E94F3B39B01AC01C501B4010E9472
:10CD6000ECB70E9457BAAFA5B8A99F966D937D9373
:10CD70008D939C93D297AFA5B8A99F968D909D90C7
:10CD8000AD90BC90D297A7968CAE9DAEAEAEBFAE26
:10CD9000A797A501940160E070E080E89FE30E94FE
:10CDA000C8B862966CAF7DAF8EAF9FAF62979B01A4
:10CDB000AC01632D722DC8010E94F3B32B013C011D
:10CDC00080902D0F80912E0F881A282D2F702E966F
:10CDD0002FAF2E97A301920160E074E284E799E4FB
:10CDE0000E94C8B80E941DBA6B017C012E968FADBF
:10CDF0002E9782508630C0F580915F069091600634
:10CE0000A0916106B0916206C816D906EA06FB0633
:10CE100058F5BC01CD016C197D098E099F09660F7B
:10CE2000771F881F991F2E968FAC2E97082D10E024
:10CE300020E030E0A90198010E9494B7CA01B9012D
:10CE40000E9492B30E941DBA6C0D7D1D8E1D9F1D08
:10CE50000E9492B39B01AC0160E074E284E799E424
:10CE60000E94C8B82B013C01A3019201A7966CADAA
:10CE70007DAD8EAD9FADA7970E94F3B366966CAF64
:10CE80007DAF8EAF9FAF6697AFA5B8A993966D9310
:10CE90007D938D939C93969752968D909D90AD9097
:10CEA000BC9055978FAA98AEA9AEBAAEC501B40191
:10CEB0000E9492B32B966CAF7DAF8EAF9FAF2B9736
:10CEC000A30192010E94F3B30E94B2B80E9435B947
:10CED0006B017C01EFA5F8A967AB70AF81AF92AF92
:10CEE0009E012F5E3F4F2D963FAF2EAF2D9741EB0A
:10CEF00053E06F965FAF4EAF6F97BE016F5D7F4F90
:10CF00007EA76DA7CE0101966C969FAF8EAF6C97F2
:10CF1000212C312C90E89BAFAFE32496AFAF249740
:10CF20002D96EEADFFAD2D9761917191819191910B
:10CF30002D96FFAFEEAF2D97A30192010E94F3B3A0
:10CF40006C96AEADBFAD6C976D937D938D939D93B5
:10CF50006C96BFAFAEAF6C979B01AC015F776A96E2
:10CF60002CAF3DAF4EAF5FAF6A976F96AEADBFAD22
:10CF70006F978D909D90AD90BD906F96BFAFAEAF07
:10CF80006F97A50194016A966CAD7DAD8EAD9FAD96
:10CF90006A970E9412BA18160CF56A962CAD3DAD30
:10CFA0004EAD5FAD6A97C501B4010E94C8B8162F97
:10CFB000072FB82EA92E262F372F482F592FB10112
:10CFC0008BAD24969FAD24970E9412BA181634F4A4
:10CFD000212E302EBBAE2496AFAE24972D968EAC6C
:10CFE0009FAC2D97ADA4BEA48A149B0409F098CFE2
:10CFF00020E030E040E85FE3B1018BAD24969FADC7
:10D0000024970E948EB387FF44C05E0121E1A20EE7
:10D01000B11C8E010F5F1F4F91014BAD24965FAD88
:10D020002497D8016D917D918D919C910E94F3B3CD
:10D03000F80161937193819391938F01EA15FB0538
:10D0400059F791014BAD24965FAD249766966CAD70
:10D050007DAD8EAD9FAD66970E94F3B3AFA5B8A925
:10D0600093966D937D938D939C939697C701B6018C
:10D070000E9492B391014BAD24965FAD24970E941C
:10D08000F3B30E9435B9EFA5F8A967AB70AF81AFD4
:10D0900092AF62962CAD3DAD4EAD5FAD62972B96D3
:10D0A0006CAD7DAD8EAD9FAD2B970E94F3B32796EF
:10D0B0006CAF7DAF8EAF9FAF2797AFA5B8A916967F
:10D0C0008D909D90AD90BC9019978BAE9CAEADAEFF
:10D0D000BEAE1A964D905D906D907C901D978BA87A
:10D0E0009CA8ADA8BEA889288A288B28D1F48BAC2F
:10D0F0009CACADACBEAC89288A288B2891F4411435
:10D1000051046104710469F42091C1033091C20398
:10D110004091C3035091C4030E94F3B30E94B2B87C
:10D1200027C223968CAC9DACAEACBFAC23978928AC
:10D130008A288B2849F06091C9037091CA038091B5
:10D14000CB039091CC0308C06091C5037091C603D6
:10D150008091C7039091C80327962CAD3DAD4EAD8D
:10D160005FAD27970E94F3B30E94B2B80E9435B911
:10D170006B017C018091780690917906A0917A06E6
:10D18000B0917B06EFA5F8A986849784A088B18822
:10D1900023968CAE9DAEAEAEBFAE23978FA898AC53
:10D1A000A9ACBAAC88159905AA05BB0508F4D3C08B
:10D1B0008BA89CA8ADA8BEA889288A288B2861F1D5
:10D1C0002091690330916A0340916B0350916C0385
:10D1D0002C153D054E055F05F8F46FA978AD89ADB6
:10D1E0009AAD0E9485B74B015C01A70196016BA91E
:10D1F0007CA98DA99EA90E9485B786169706A806C8
:10D20000B90650F4C501B4012BA93CA94DA95EA9EA
:10D210000E9494B769017A018BAC9CACADACBEACFA
:10D2200089288A288B2861F120916D0330916E0343
:10D2300040916F03509170032C153D054E055F051D
:10D24000F8F46FA978AD89AD9AAD0E9485B74B010E
:10D250005C01A70196016BAD7CAD8DAD9EAD0E94CA
:10D2600085B786169706A806B90650F4C501B4011D
:10D270002BAD3CAD4DAD5EAD0E9494B769017A0116
:10D28000411451046104710441F120917103309102
:10D29000720340917303509174032C153D054E05A4
:10D2A0005F05D8F46FA978AD89AD9AAD0E9485B7B6
:10D2B0004B015C01A7019601C301B2010E9485B731
:10D2C00086169706A806B90640F4C501B401A30165
:10D2D00092010E9494B769017A0123968CAC9DACAF
:10D2E000AEACBFAC239789288A288B2809F444C1A7
:10D2F0002091750330917603409177035091780324
:10D300002C153D054E055F0508F036C16FA978ADB7
:10D3100089AD9AAD0E9485B74B015C01A7019601CA
:10D3200023966CAD7DAD8EAD9FAD23970E9485B7E2
:10D3300086169706A806B90608F01EC1C501B401F5
:10D3400023962CAD3DAD4EAD5FAD23970E9494B7B3
:10D3500069017A0111C18BA89CA8ADA8BEA8892833
:10D360008A288B2809F43FC06091690370916A0391
:10D3700080916B0390916C036C157D058E059F0564
:10D3800090F50E9492B32B962CAD3DAD4EAD5FADA6
:10D390002B970E94F3B34B015C016BA97CA98DA96B
:10D3A0009EA90E9494B36BAB7CAB8DAB9EABC701C7
:10D3B000B6010E9492B32BA93CA94DA95EA90E9477
:10D3C000F3B3A50194010E9412BA181664F42BA9B4
:10D3D0003CA94DA95EA9C501B4010E94C8B80E942C
:10D3E00035B96B017C018BAC9CACADACBEAC892873
:10D3F0008A288B2809F43FC060916D0370916E03F9
:10D4000080916F03909170036C157D058E059F05CB
:10D4100090F50E9492B32B962CAD3DAD4EAD5FAD15
:10D420002B970E94F3B34B015C016BAD7CAD8DADCE
:10D430009EAD0E9494B36BAB7CAB8DAB9EABC70132
:10D44000B6010E9492B32BA93CA94DA95EA90E94E6
:10D45000F3B3A50194010E9412BA181664F42BA923
:10D460003CA94DA95EA9C501B4010E94C8B80E949B
:10D4700035B96B017C014114510461047104B9F1A7
:10D4800060917103709172038091730390917403A2
:10D490006C157D058E059F0550F50E9492B32B9665
:10D4A0002CAD3DAD4EAD5FAD2B970E94F3B34B015C
:10D4B0005C01C301B2010E9494B32B013C01C7017E
:10D4C000B6010E9492B3A30192010E94F3B3A50199
:10D4D00094010E9412BA181654F4A3019201C501D6
:10D4E000B4010E94C8B80E9435B96B017C01239633
:10D4F0008CAC9DACAEACBFAC239789288A288B2816
:10D50000D9F16091750370917603809177039091C2
:10D5100078036C157D058E059F0570F50E9492B30A
:10D520002B962CAD3DAD4EAD5FAD2B970E94F3B366
:10D530004B015C0123966CAD7DAD8EAD9FAD239705
:10D540000E9494B32B013C01C701B6010E9492B323
:10D55000A30192010E94F3B3A50194010E9412BAA3
:10D56000181654F4A3019201C501B4010E94C8B871
:10D570000E9435B96B017C01EFA5F8A9ED5BFF4F67
:10D58000C082D182E282F382C701B6010E9492B3C7
:10D590006B017C0127962CAD3DAD4EAD5FAD27975D
:10D5A0000E94C8B8AB966CAF7DAF8EAF9FAFAB9704
:10D5B000AFA5B8A9D3966D937D938D939C93D69781
:10D5C00020E030E040E85BE4C701B6010E94F3B31D
:10D5D00020E034E244EF59E40E94C8B80E9430B918
:10D5E000EFA5F8A9668F778F80A391A383A08BAA5C
:10D5F00094A09FAEA5A0AFAAB6A02896BFAE2897CC
:10D600002E0121E1420E511C69E7262E63E0362EE1
:10D61000AE014F5F5F4F3A018BAE24969FAE2497C9
:10D620002C96AFAE2C972F96BFAE2F9710E0D3015C
:10D630008D909D90AD90BD903D01E894B7F8F101BB
:10D64000C190D190E190F1901F01A7019601C50111
:10D65000B4010E9412BA18160CF03EC0112389F1D1
:10D660002BA93FAD4FA928965FAD2897C701B601FA
:10D670000E94F3B36B017C012BAD24963FAD249740
:10D680002C964FAD2C972F965FAD2F97C501B40107
:10D690000E94F3B3A70196010E9412BA1816DCF497
:10D6A000A5019401C701B6010E94C8B86BAF2496CA
:10D6B0007FAF24972C968FAF2C972F969FAF2F97E5
:10D6C0000AC0CBAE2496DFAE24972C96EFAE2C97F3
:10D6D0002F96FFAE2F9711E06414750409F0A7CFC1
:10D6E0002E96FFAD2E97F23008F486C10091090FF7
:10D6F00010910A0F20900B0F30900C0F27E137EBA1
:10D7000041ED58E3B801C1010E9412BA18160CF09D
:10D7100073C121E0AC962FAFAC972BA93FAD4FA9B9
:10D7200028965FAD2897B801C1010E9412BA181659
:10D73000A4F0AC961FAEAC972BA93FAD4FA928968D
:10D740005FAD2897B801C1010E94C8B8E0966CAFE0
:10D750007DAF8EAF9FAFE09716C09801A1016BA976
:10D760007FAD8FA928969FAD28970E94C8B8E096F4
:10D770006CAF7DAF8EAF9FAFE0970BA91FAD2FA809
:10D7800028963FAC28974DE05FE06F965FAF4EAFB5
:10D790006F9769E773E0E2967FAF6EAFE297CE01D5
:10D7A0000196E4969FAF8EAFE497412C512C50E840
:10D7B000652E5FE3752E6B961FAE6B976F96AEADC1
:10D7C000BFAD6F97CD90DD90ED90FD906F96BFAFA0
:10D7D000AEAF6F97E496EEADFFADE4978190919078
:10D7E000A190B190E496FFAFEEAFE497AC96FFAD99
:10D7F000AC97FF2361F0E0962CAD3DAD4EAD5FAD33
:10D80000E097C701B6010E94F3B36B017C016B96F0
:10D810002FAD6B97222381F0A3019201C701B601BE
:10D820000E94F3B36B017C01A3019201C501B40115
:10D830000E94F3B34B015C01A5019401C701B6013D
:10D840000E9412BA20E030E0A9011816CCF4C501FC
:10D85000B4010E9412BA18164CF020E030E0A90181
:10D86000C701B6010E948EB387FF05C0A5019401D0
:10D87000C701B60118C0B7FAB094B7F8B09424C085
:10D88000C501B4010E948EB387FD09C020E030E0DD
:10D89000A901C701B6010E9412BA18168CF4A7019B
:10D8A0009601C501B4010E94EBB72E966FAF2E977B
:10D8B00063967FAF639767968FAF6797B92E20C047
:10D8C000F7FAF094F7F8F094A5019401C701B601B6
:10D8D0000E9412BA18165CF42E96CFAE2E9763965D
:10D8E000DFAE63976796EFAE6797BF2C09C02E96A1
:10D8F0008FAE2E9763969FAE63976796AFAE67978E
:10D90000E296AEADBFADE297CD90DD90ED90FD908B
:10D91000E296BFAFAEAFE297A70196012E966FAD2C
:10D920002E9763967FAD639767968FAD67979B2D14
:10D930000E9412BA1816ECF42E962FAD2E9763960D
:10D940003FAD639767964FAD67975B2DC701B601F3
:10D950000E94C8B89B01AC01C301B2010E94F3B39D
:10D960002B013C016B96BFAD6B97BF5F6B96BFAF52
:10D970006B976F96EEADFFAD6F97ED51FF4009F0DD
:10D980001DCF6B968FAC6B97882041F0A30192015D
:10D99000B801C1010E94F3B38B011C0124EA30E7F6
:10D9A0004DE75FE3B801C1010E94F3B36B017C0155
:10D9B0009B01AC01609174067091750680917606AA
:10D9C000909177060E9412BA18162CF5A7019601BD
:10D9D0006BAD24967FAD24972C968FAD2C972F9608
:10D9E0009FAD2F970E9412BA1816ACF4AFA5B8A934
:10D9F0008C9184608C9305C0EFA5F8A98081846028
:10DA000080830BAD24961FAD24972C962FAC2C97BA
:10DA10002F963FAC2F97C801D101EFA5F8A983A796
:10DA200094A7A5A7B6A7AB966CAD7DAD8EAD9FAD07
:10DA3000AB9790589B01AC010E94ECB7A7962CAD18
:10DA40003DAD4EAD5FADA7970E94F3B39B01AC0116
:10DA50006BE077ED83E29BE30E94EBB70E9457BA3D
:10DA60007B01782E892E9B01482F592FB801C101C7
:10DA70000E948EB387FF05C0902EA12EB22CC32C1E
:10DA800004C09E2CAF2CB72CC82C892D9A2DAB2D01
:10DA9000BC2DEFA5F8A987A390A7A1A7B2A7D08016
:10DAA0009701472D582D6BA97FAD8FA928969FAD63
:10DAB00028970E948EB3181614F083E001C081E00D
:10DAC000D82AAFA5B8A9DC9280E1FE013196ADE07D
:10DAD000BFE001900D928A95E1F78BA99FADAFA9A8
:10DAE0002896BFAD28978093090F90930A0FA093B3
:10DAF0000B0FB0930C0F8BAD24969FAD24972C96F3
:10DB0000AFAD2C972F96BFAD2F978093740690934F
:10DB10007506A0937606B09377062BA93FAD4FA963
:10DB200028965FAD2897BC01CD010E94C8B86DA3AF
:10DB30007EA38FA398A72BA93FAD4FA928965FADD1
:10DB40002897692D7A2D8B2D9C2D0E94C8B869A32A
:10DB50007AA38BA39CA3AE014B5D5F4FBE016F5DAB
:10DB60007F4F8FA598A90E94B77F6D968FAC6D9758
:10DB700080922D0FE8968CAC9DACAEACBFACE89714
:10DB800080921D0F90921E0FA0921F0FB092200F37
:10DB9000EC968CAC9DACAEACBFACEC978092210FF8
:10DBA0009092220FA092230FB092240FC458DF4FFF
:10DBB00088809980AA80BB80CC57D0408092250F66
:10DBC0009092260FA092270FB092280FA3968CACAC
:10DBD0009DACAEACBFACA3978092290F90922A0F58
:10DBE000A0922B0FB0922C0F80912D0F90912E0FA1
:10DBF000891B8F70843048F420912E0FE12CF12C7A
:10DC000080E090E04DE4D42EABC090902E0F9FA604
:10DC1000B0902D0F3DEFA32EBA0C2B2D2F70B22EEE
:10DC2000C12CD12CE12CF12C8FA4B81429F3E114D0
:10DC3000F10421F0D7018C9182FDDECFBA94BB2D87
:10DC4000BF70BB2EEDE4EB9F800111240C53184FE5
:10DC5000E114F10409F476C0C114D10409F472C0CE
:10DC6000D7019B967C909B979C968C909C979D96B9
:10DC70009C909D979E96AC909E97272D382D492D70
:10DC80005A2D97966D917D918D919C919A970E94B6
:10DC90008EB3882309F456C0F701608061FC46C04A
:10DCA000D60197962D903D904D905C909A97A20149
:10DCB0009101672D782D892D9A2D0E948EB318160B
:10DCC000ACF5A2019101C201B1010E94F3B31B01A5
:10DCD0002C01F70183A994A9A5A9B6A9BC01CD017E
:10DCE00090589B01AC010E94ECB7D7019F962D91F3
:10DCF0003D914D915C91D2970E94F3B39B01AC0191
:10DD0000C201B1010E94EBB70E9457BA1B016C011E
:10DD10009B01AC01672D782D892D9A2D0E948EB321
:10DD200087FD04C0722C832C9C2CAD2C872D982D44
:10DD3000A92DBA2DF70187A390A7A1A7B2A7862D79
:10DD400081608083670178016FCFD29E80011124AA
:10DD50000C53184F009749F42F5F2F70C7017801BB
:10DD600030912D0F2313F1CF12C0DC013C9131FD16
:10DD7000F3CFB701C058DF4F2883C058D0400E946E
:10DD80002334C058DF4F2881C058D040E5CF0097DA
:10DD900039F0FC01208121FD03C0B7010E9423342A
:10DDA00090902E0F00E010E02DE4822E892D99270F
:10DDB00087FD909520912D0F30E08217930709F48D
:10DDC0004AC0889E5001899EB00C112495012C53A5
:10DDD000384F590101151105C1F1D8018C9180FD11
:10DDE00004C0F901808180FF30C0D8019396CD90A6
:10DDF000DD90ED90FC909697A7019601F50167A143
:10DE000070A581A592A50E94C8B869A37AA38BA327
:10DE10009CA3A7019601D80197966D917D918D9154
:10DE20009C919A970E94C8B86DA37EA38FA398A7D0
:10DE3000AE014F5D5F4FBE016B5D7F4FC8010E9419
:10DE4000B77FF80180818E7F80839394F92DFF70D6
:10DE50009F2E8501ABCF0115110569F1D80193966D
:10DE6000CD90DD90ED90FC909697A70196016DEC1A
:10DE70007CEC8CE49DE30E94C8B869A37AA38BA3D1
:10DE80009CA3A7019601F80167A170A581A592A5A1
:10DE90000E94C8B86DA37EA38FA398A7AE014F5D63
:10DEA0005F4FBE016B5D7F4FC8010E94B77FD801F5
:10DEB0008C918E7F8C9380916F00826080936F0035
:10DEC0000CC028963FAC28972BAC24960FAD249716
:10DED0002C961FAD2C970C940866C058DF4F0FB6D8
:10DEE000F894DEBF0FBECDBFDF91CF911F910F9190
:10DEF000FF90EF90DF90CF90BF90AF909F908F906A
:10DF00007F906F905F904F903F902F900895CF92A9
:10DF1000EF92FF920F931F93CF93DF93CDB7DEB7AE
:10DF20002C970FB6F894DEBF0FBECDBFC0901B0478
:10DF30008091020690910306A0910406B091050617
:10DF40004091FE055091FF05609100067091010619
:10DF50000091FA051091FB052091FC053091FD051B
:10DF600009831A832B833C834D835E836F83788779
:10DF700089879A87AB87BC87AE01475F5F4FBE0139
:10DF80006B5F7F4FCE0101960E94EF2EE0900A0258
:10DF9000F0900B0200910C0210910D0226E036E089
:10DFA000AE01475F5F4FBE016B5F7F4FCE010196B1
:10DFB0000E94BA612C960FB6F894DEBF0FBECDBF9B
:10DFC000DF91CF911F910F91FF90EF90CF90089527
:10DFD0008F929F92AF92BF92CF92EF92FF920F9348
:10DFE0001F93CF93DF93CDB7DEB72C970FB6F8947E
:10DFF000DEBF0FBECDBF4B015C01C0901B04809102
:10E000004E0390914F03A0915003B0915103409162
:10E010004A0350914B0360914C0370914D03009162
:10E020004603109147032091480330914903098327
:10E030001A832B833C834D835E836F837887898724
:10E040009A87AB87BC87AE01475F5F4FBE016B5FAE
:10E050007F4FCE0101960E94EF2E8501740122E5CB
:10E0600033E0AE01475F5F4FBE016B5F7F4FCE0174
:10E0700001960E94BA612C960FB6F894DEBF0FBECF
:10E08000CDBFDF91CF911F910F91FF90EF90CF9077
:10E09000BF90AF909F908F9008958F929F92AF9274
:10E0A000BF92DF92EF92FF920F931F93CF93DF9374
:10E0B00080915906843008F017C12FB7F8948091E9
:10E0C000C2079091C3072FBF891B8F7709F40CC13A
:10E0D0000E9479352091E7063091E8068A3019F0E0
:10E0E0008D3009F0D0C01092E9062115310501F3F9
:10E0F000F901E957F94F10821092E8061092E706ED
:10E1000087E896E07C01FC01208101962032D1F362
:10E11000E7012E3411F0E12CF12C6AE270E0CE011F
:10E120000E94DCBB8C01E114F10409F474C06BE5BE
:10E1300071E1CE010E9446B3DD24D394892B11F402
:10E14000D12C09C06EE470E0CE0104960E94DCBBC5
:10E15000009709F07C014AE050E060E070E0C70100
:10E1600001960E94D5B060938306709384068093D5
:10E1700085069093860680905A0390905B03A0904A
:10E180005C03B0905D03FFEF8F1A9F0AAF0ABF0ACE
:10E19000681579058A059B0531F0D11004C061E04E
:10E1A00088E291E13DC00115110501F180E0F12CFB
:10E1B000FE01E80FF11D90819A3219F08F5FF92668
:10E1C000F7CF4AE050E060E070E0C80101960E949D
:10E1D000D5B00F2D10E020E030E060177107820706
:10E1E000930741F061E089E091E11AC061E08FEDB1
:10E1F00090E116C08091830690918406A0918506D7
:10E20000B091860680935A0390935B03A0935C03BE
:10E21000B0935D0312C0009781F060E08EE390E15F
:10E22000DF91CF911F910F91FF90EF90DF90BF9002
:10E23000AF909F908F900C946DA7809126028111D2
:10E240001CC067E470E0CE010E94DCBB0097A9F01F
:10E250004AE050E060E070E001960E94D5B0643082
:10E26000710558F4E8E6F0E18491EF0121968823E6
:10E2700021F00E94FD34FE01F7CF61E087E896E0CF
:10E280000E94903515CF2F3531050CF011CF8C350C
:10E29000B1F42FB7F8948091C2079091C3072FBFB4
:10E2A000891B8F7709F404CF0E9479359091E90694
:10E2B0009111FECE2091E7063091E80609C08B331C
:10E2C00019F491E09093E9069091E9069111F0CE4E
:10E2D000A9014F5F5F4F5093E8064093E706F901AD
:10E2E000E957F94F8083E4CEDF91CF911F910F91D1
:10E2F000FF90EF90DF90BF90AF909F908F90089528
:10E300008F929F92AF92BF92CF92DF92EF92FF9245
:10E310006091D30C7091D40C882777FD8095982F4D
:10E320000E9494B36B017C018090E6039090E70318
:10E33000A090E803B090E90380E20E94FD3484E5F8
:10E340000E94FD348AE30E94FD3442E0C501B4011D
:10E350000AD6B701A60182E390E10E940A82609189
:10E36000CF0C7091D00C882777FD8095982F0E9454
:10E3700094B36B017C018090EA039090EB03A09032
:10E38000EC03B090ED0380E20E94FD3482E40E9431
:10E39000FD348AE30E94FD3442E0C501B401E3D5B7
:10E3A000B701A60182E390E10E940A82EAE3F0E16C
:10E3B00084917F019FEFE91AF90A882321F00E94D6
:10E3C000FD34F701F5CFE091EE03F0E0E751F34FB4
:10E3D000608170E080E090E0A0D5E5E3F0E1849119
:10E3E0007F019FEFE91AF90A882321F00E94FD348A
:10E3F000F701F5CF6091E70C70E080E090E0FF90CE
:10E40000EF90DF90CF90BF90AF909F908F9085C599
:10E410008F929F92AF92BF92CF92DF92EF92FF9234
:10E420000F931F93CF93DF9300D000D0CDB7DEB70B
:10E4300080916203882381F00E94DB38C0905E03E4
:10E44000D0905F03E0906003F09061036C197D0948
:10E450008E099F0997FF58C280915906843028F48D
:10E460000E94484F811101C018DE0E94DB38C09025
:10E470006503D0906603E0906703F0906803C114D1
:10E48000D104E104F10481F1809056039090570388
:10E49000A0905803B09059038C0C9D1CAE1CBF1C5F
:10E4A0006B017C01C818D908EA08FB08F7FC1CC0FE
:10E4B000E5EEFAE084917F012FEFE21AF20A882359
:10E4C00021F00E94FD34F701F5CF60911C0470919A
:10E4D0001D0489E691E10E9404358AE00E94FD3422
:10E4E00080E691E10E94BAA7C0900E02D0900F0280
:10E4F000E0901002F0901102C114D104E104F10483
:10E50000C9F08090560390905703A0905803B090A4
:10E5100059038C0C9D1CAE1CBF1CAB01BC014819DF
:10E5200059096A097B0977FD05C00E94D8378823FD
:10E5300009F406C20E94DB38C090F606D090F706B8
:10E54000E090F806F090F9069B01AC012C193D090A
:10E550004E095F0957FD42C06B017C0134ECC30ECC
:10E5600039E0D31EE11CF11CC092F606D092F706EA
:10E57000E092F806F092F906079BEDC1069BEBC10D
:10E58000059BE9C12091E70C2111E5C1049BE3C182
:10E59000C090F206D090F306E090F406F090F506F5
:10E5A000C114D104E104F10461F0DC01CB018C1948
:10E5B0009D09AE09BF0980569A4EA109B109B7FD60
:10E5C000D3C19FB7F89480910201877F80930201A5
:10E5D0009FBF60E070E086E00E941F4B0E94DB3826
:10E5E000C090EE06D090EF06E090F006F090F106B5
:10E5F0006C197D098E099F0997FD52C00E94DB3876
:10E6000068577C4E8F4F9F4F6093EE067093EF06D6
:10E610008093F0069093F10663E073E0CE010196DB
:10E620000E94F537BE016F5F7F4F80E79EE00E943A
:10E63000C94C89819A810E94DEAE65E073E0CE010B
:10E6400001960E94F537BE016F5F7F4F8BEF9DE013
:10E650000E94C94C89819A810E94DEAE67E073E016
:10E66000CE0101960E94F537BE016F5F7F4F86E8AD
:10E670009DE00E94C94C89819A810E94DEAE69E0CA
:10E6800073E0CE0101960E94F537BE016F5F7F4FA8
:10E6900081E19DE00E94C94C89819A810E94DEAE91
:10E6A000109163030E94D837882391F0E0912E0FD8
:10E6B0004DE4E49FF0011124E55FF74F1081909144
:10E6C0002E0F80912D0F981719F09F5F9F70F9CF33
:10E6D000112341F10E94DB38C090EA06D090EB068E
:10E6E000E090EC06F090ED06C114D104E104F104D1
:10E6F00081F46B017C0154E6C50ED11CE11CF11CB8
:10E70000C092EA06D092EB06E092EC06F092ED069B
:10E7100035C19B01AC012C193D094E095F0957FF1A
:10E720002EC12CC11092EA061092EB061092EC0654
:10E730001092ED0660E070E088E00E941F4B0E949E
:10E7400070A910912F0F113009F024C1809120077A
:10E7500081110CC00E94DB3860931C0770931D0769
:10E7600080931E0790931F07109320078091140732
:10E7700081110DC00E94DB38609310077093110760
:10E78000809312079093130781E0809314070E94EF
:10E79000DB386B017C0180910807811114C0409126
:10E7A0004E0F50914F0F28EE33E0429FC001439F20
:10E7B000900D529F900D11249093070780930607A8
:10E7C00081E08093080780911C0790911D07A0911C
:10E7D0001E07B0911F07B701A601481B590B6A0B12
:10E7E0007B0B8091060790910707A0E0B0E04817E7
:10E7F00059076A077B07A0F18090520F9090530F42
:10E80000A090540FB090550F8FE29FE00E94E73820
:10E810006093520F7093530F8093540F9093550F42
:10E820000091400F1091410F2091420F3091430F02
:10E83000081919092A093B09060F171F281F391F34
:10E840000093400F1093410F2093420F3093430FDA
:10E85000C0921C07D0921D07E0921E07F0921F077E
:10E860008091FE0681111AC04091500F5091510FB6
:10E8700028EE33E0429FC001439F900D529F900DC0
:10E880001124A0E0B0E08093FA069093FB06A093D9
:10E89000FC06B093FD0681E08093FE068091100790
:10E8A00090911107A0911207B0911307B701A6012B
:10E8B000481B590B6A0B7B0B8091FA069091FB0663
:10E8C000A091FC06B091FD06481759076A077B071F
:10E8D00008F460C0C0921007D0921107E0921207AE
:10E8E000F09213078091560F882309F453C060916A
:10E8F0004C0F70914D0F6F5F7F4F40E150E08CE304
:10E900009FE00E945CB646C00E94DB386B017C0130
:10E910002091620330E0A8EEB3E00E94DCB7C60E9F
:10E92000D71EE81EF91EC0925E03D0925F03E092EC
:10E930006003F0926103E4DC8AE00E94FD348CCD38
:10E94000179A1092EA05169A1092EB05159A1092F2
:10E95000EC05149AEFCD6093F2067093F306809362
:10E96000F4069093F50614CE9FB7F89480910201B7
:10E970008860809302019FBF68E72CCE1FEF39EBC0
:10E98000139FC00111246FEF70E00E94C8BA6A5B48
:10E990007F4FD2CE26960FB6F894DEBF0FBECDBF06
:10E9A000DF91CF911F910F91FF90EF90DF90CF906B
:10E9B000BF90AF909F908F9008958F929F92AF924B
:10E9C000BF92DF92EF92FF920F931F93CF93DF934B
:10E9D000EC017B018DEC9CECACECBDE3888399836E
:10E9E000AA83BB8380E090E00E9492B325ED34E0DF
:10E9F00045E352E40E94F3B320E030E04AE754E4F8
:10EA00000E94C8B84B015C0120E932EC45EF5DE3A0
:10EA10000E94F3B326E636E646EA5EE30E94C8B8F3
:10EA200020E030E040E85FE30E94EBB70E9435B998
:10EA3000D62E8FE08D1588F1AE01415B5F4FFA0154
:10EA400080819181A281B381A26080839183A2831E
:10EA5000B3836CEECE010E94E34B2AE037ED43EA2C
:10EA60005CE3688179818A819B810E94ECB79B017C
:10EA7000AC01C501B4010E94F3B32CEE31E548E3CB
:10EA80005EE30E94C8B820E030E040E85FE30E9407
:10EA9000EBB70E9435B9D62E16C0CE010E94D74DD5
:10EAA000882389F0AE01415B5F4FFA01808191813B
:10EAB000A281B381AD7F80839183A283B3836CEE07
:10EAC000CE010E94E34B8D2D90E0A0E0B0E0BA2F84
:10EAD000A92F982F882788279F71AA27BB270F85E2
:10EAE000188929893A89107E802B912BA22BB32B70
:10EAF0008F87988BA98BBA8B5E01FFE0AF0EB11C9C
:10EB0000A50160E9CE010E94E34B6D2D70E080E02D
:10EB100090E00E9494B320E030E040E05FE30E9488
:10EB2000F3B30E9435B96F710F85188929893A8925
:10EB3000007E062B0F87188B298B3A8BA50160E985
:10EB4000CE010E94E34BCD58DF4FF982E882DF917E
:10EB5000CF911F910F91FF90EF90DF90BF90AF90FA
:10EB60009F908F9008951F93CF93DF93EC01162F02
:10EB7000BA0123DF612FCE01DF91CF911F910C9459
:10EB8000E681EF92FF920F931F93CF93DF93EC01F7
:10EB90000E942B4EFE01ED58FF4F60817181CE0126
:10EBA0000CDF64E0CE010E941B4F62E0CE010E94A8
:10EBB000FB4D65E0CE010E94E64D8E01015B1F4FCB
:10EBC000F80180819181A281B381B06180839183BA
:10EBD000A283B383A8016CEECE010E94E34BAE0189
:10EBE0004D595F4F80E890E0A0E0B0E0FA018083EB
:10EBF0009183A283B38361E9CE010E94E34BF801C4
:10EC000080819181A281B381806780839183A28377
:10EC1000B383A8016CEECE010E94E34BF801808122
:10EC20009181A281B3818F77987F92608083918355
:10EC3000A283B383A8016CEECE010E94E34B8B85C7
:10EC40009C85AD85BE859F7E8B879C87AD87BE8763
:10EC500004541109A80160E8CE010E94E34B8B85A2
:10EC60009C85AD85BE859F7D8B879C87AD87BE8744
:10EC7000A80160E8CE010E94E34B8B859C85AD85A1
:10EC8000BE8591608B879C87AD87BE87A80160E8B1
:10EC9000CE010E94E34B8B859C85AD85BE8580614E
:10ECA0008B879C87AD87BE87A80160E8CE010E9454
:10ECB000E34B8B859C85AD85BE858E7F8B879C873E
:10ECC000AD87BE87A80160E8CE010E94E34B8B852B
:10ECD0009C85AD85BE858D7F8B879C87AD87BE87E4
:10ECE000A80160E8CE010E94E34B7E01F3E5EF0E40
:10ECF000F11CF70180819181A281B381807F8160C5
:10ED000080839183A283B383A7016DEECE010E941D
:10ED1000E34BF7010081118122813381107F1A605A
:10ED20000083118322833383A7016DEECE010E94FD
:10ED3000E34B8FEF9FEFAFE0B0E08B8F9C8FAD8FF9
:10ED4000BE8FAE01455E5F4F64E9CE01DF91CF918A
:10ED50001F910F91FF90EF900C94E34BDF92EF9295
:10ED6000FF920F931F93CF93DF93EC01D62E1B8E50
:10ED70001C8E1D8E1E8E7C018BE1E80EF11CA701FE
:10ED800064E9CE010E94E34B61E0CE010E94904C09
:10ED90000FEF1FEF2FE030E00B8F1C8F2D8F3E8F7A
:10EDA000A70164E9CE010E94E34B60E0CE010E941E
:10EDB000904C4D2D50E060E070E0762F652F542F81
:10EDC000442744275170662777270B851C852D859E
:10EDD0003E851E7F402B512B622B732B4B875C870C
:10EDE0006D877E87AE01455F5F4F60E8CE01DF91A2
:10EDF000CF911F910F91FF90EF90DF900C94E34B18
:10EE0000AF92BF92CF92DF92EF92FF920F931F9338
:10EE1000CF93DF93CDB7DEB7A0970FB6F894DEBFE0
:10EE20000FBECDBF6115710581059105B1F1B12C02
:10EE3000C42ED12CE12CF12CAA24A394AB0C01E01C
:10EE400010E00C0F1D1F0B0D111DB7FC1A95A7012B
:10EE500096010E9494B7F8016083B901CA01611557
:10EE600071058105910511F41B2D12C0BA2CE4CF58
:10EE7000E1E0F0E0EC0FFD1FE10FF11D17FDFA9549
:10EE800080818A3040F490E3890F0E94FD34115054
:10EE90001F3F71F715C097E3F7CF80E3A0960FB639
:10EEA000F894DEBF0FBECDBFDF91CF911F910F91C0
:10EEB000FF90EF90DF90CF90BF90AF900C94FD3417
:10EEC000A0960FB6F894DEBF0FBECDBFDF91CF91F5
:10EED0001F910F91FF90EF90DF90CF90BF90AF9078
:10EEE0000895CF92DF92EF92FF92CF93DF936A0162
:10EEF0007B01FC018491EF012196882321F00E947F
:10EF0000FD34FE01F7CF4AE0C701B601DF91CF9192
:10EF1000FF90EF90DF90CF9073CFCF92DF92EF9280
:10EF2000FF926B017C0197FF0BC08DE20E94FD34C4
:10EF3000F094E094D094C094C11CD11CE11CF11C4D
:10EF40004AE0C701B601FF90EF90DF90CF9058CF15
:10EF5000BC0180E090E04AE053DF8DE00E94FD3488
:10EF60008AE00C94FD348F929F92AF92BF92CF9221
:10EF7000DF92EF92FF92CF936B017C01B42E20E0E1
:10EF800030E0A9010E948EB387FF07C08DE20E9486
:10EF9000FD34F7FAF094F7F8F094C0E060E070E028
:10EFA00080E09FE3CB1541F02DEC3CEC4CEC5DE3B5
:10EFB0000E94F3B3CF5FF6CF9B01AC01C701B6014E
:10EFC0000E94ECB76B017C010E9435B94B015C01DA
:10EFD0004AE016DFCC2389F1C501B4010E9492B347
:10EFE0009B01AC01C701B6010E94EBB76B017C012C
:10EFF0008EE20E94FD3420E030E040E251E4C7019F
:10F00000B6010E94F3B36B017C010E9430B94B0141
:10F01000AA2497FCA094BA2CC501B4017EDFC501D7
:10F02000B4010E9494B39B01AC01C701B6010E94D8
:10F03000EBB76B017C01C150F1F6CF91FF90EF90DF
:10F04000DF90CF90BF90AF909F908F9008950F93D7
:10F050001F93CF93DF93FC018491EF0121968111DF
:10F0600002C010E004C00E94FD34FE01F5CF03E0B1
:10F07000010F84E0189FE0011124FE01EB51F14FD4
:10F0800020E030E0A90160817181828193810E943A
:10F0900012BA87FD03C08BE20E94FD34CB51D14FE1
:10F0A000688179818A819B8146E05DDF80E20E94F0
:10F0B000FD341F5F1013DDCF8AE00E94FD3419304C
:10F0C000B1F6DF91CF911F910F9108954F925F920A
:10F0D0006F927F928F929F92AF92BF92CF92DF9268
:10F0E000EF92FF92CF93DF93E4EEF1E18491EF0191
:10F0F0002196882321F00E94FD34FE01F7CF609114
:10F10000FA057091FB058091FC059091FD0542E0A8
:10F110002ADFE0EEF1E18491EF012196882321F0CE
:10F120000E94FD34FE01F7CF6091FE057091FF054E
:10F13000809100069091010642E015DFECEDF1E1CF
:10F140008491EF012196882321F00E94FD34FE0175
:10F15000F7CF6091020670910306809104069091AA
:10F16000050642E000DFE8EDF1E18491EF01219630
:10F17000882321F00E94FD34FE01F7CF609106063E
:10F1800070910706809108069091090642E0EBDE37
:10F190008FB7F8944090940C5090950C6090960C1A
:10F1A0007090970C8090980C9090990CA0909A0C6D
:10F1B000B0909B0CC0909C0CD0909D0CE0909E0C4D
:10F1C000F0909F0C8FBFEEECF1E18491EF0121965E
:10F1D000882321F00E94FD34FE01F7CFC301B20164
:10F1E0009CDEEAECF1E18491EF012196882321F085
:10F1F0000E94FD34FE01F7CFC501B4018EDEE6ECBE
:10F20000F1E18491EF012196882321F00E94FD34E1
:10F21000FE01F7CFC701B60180DE8AE0DF91CF9112
:10F22000FF90EF90DF90CF90BF90AF909F908F9026
:10F230007F906F905F904F900C94FD340F931F93CD
:10F24000CF93DF938B01FC018491EF0121968823FA
:10F2500021F00E94FD34FE01F7CFB801882777FD29
:10F260008095982FDF91CF911F910F9156CE8F925D
:10F270009F92AF92BF92CF92DF92EF92FF920F9345
:10F280001F93CF93DF93CDB7DEB7C555D1090FB626
:10F29000F894DEBF0FBECDBF21961CAE1DAE1EAED4
:10F2A0001FAE219780E390E3A0E3B0E089AF9AAF6F
:10F2B000ABAFBCAF27961FAE1EAE279784E690E09B
:10F2C0002D969FAF8EAF2D9710925E069E012B5B01
:10F2D0003F4F44E050E0BE01675C7F4FCE01855B4D
:10F2E0009F4F0E9430512D968EAD9FAD2D97029667
:10F2F0002D969FAF8EAF2D9727961FAE1EAE2797E8
:10F3000081E066968FAF66979E012B5B3F4F41E091
:10F3100050E0BE016B5A7F4FCE01855B9F4F0E942C
:10F3200030519E012B5B3F4F40E150E069E873E0B4
:10F33000CE01855B9F4F0E9430519E012B5B3F4F5A
:10F3400040E150E061EB73E0CE01855B9F4F0E948E
:10F3500030519E012B5B3F4F40E150E061EA73E08A
:10F36000CE01855B9F4F0E9430519E012B5B3F4F2A
:10F3700044E050E069EC73E0CE01855B9F4F0E9452
:10F3800030519E012B5B3F4F44E050E061EC73E055
:10F39000CE01855B9F4F0E9430519E012B5B3F4FFA
:10F3A00044E050E065EC73E0CE01855B9F4F0E9426
:10F3B00030519E012B5B3F4F44E050E067E676E022
:10F3C000CE01855B9F4F0E9430519E012B5B3F4FCA
:10F3D00044E050E063E676E0CE01855B9F4F0E94FB
:10F3E00030519E012B5B3F4F44E050E06FE576E0EB
:10F3F000CE01855B9F4F0E9430519E012B5B3F4F9A
:10F4000040E150E069E773E0CE01855B9F4F0E94C9
:10F4100030519E012B5B3F4F4CE050E06EEE75E0AB
:10F42000CE01855B9F4F0E94305180E090E0A0E2CA
:10F43000B1E48DAB9EABAFABB8AF9E012B5B3F4F42
:10F4400044E050E0BE016B5C7F4FCE01855B9F4F77
:10F450000E94305165961FAE659721961CAE1DAE79
:10F460001EAE1FAE219783E064968FAF64976396BC
:10F470008FAF63979E012B5B3F4F41E050E0BE0191
:10F480006C5A7F4FCE01855B9F4F0E9430519E0189
:10F490002B5B3F4F44E050E0BE01635C7F4FCE01E9
:10F4A000855B9F4F0E9430519E012B5B3F4F41E097
:10F4B00050E0BE016D5A7F4FCE01855B9F4F0E9489
:10F4C00030519E012B5B3F4F41E050E0BE016E5A30
:10F4D0007F4FCE01855B9F4F0E9430511AE0115043
:10F4E00071F09E012B5B3F4F44E050E0BE01635C36
:10F4F0007F4FCE01855B9F4F0E943051F0CF279602
:10F500000EAD1FAD27972D968EAD9FAD2D97909385
:10F510002F0280932E029E012B5B3F4F44E050E070
:10F520006BE074E0CE01855B9F4F0E9430512796BF
:10F530001FAF0EAF27979E012B5B3F4F44E250E079
:10F5400065EE7EE0CE01855B9F4F0E94305183E0E7
:10F5500062968FAF629761968FAF619719AA1AAAC8
:10F560001BAA1CAA1DA61EA61FA618AA21961CAE81
:10F570001DAE1EAE1FAE21979E012B5B3F4F41E09B
:10F5800050E0BE016F5A7F4FCE01855B9F4F0E94B6
:10F5900030519E012B5B3F4F41E050E0BE01605B6C
:10F5A0007F4FCE01855B9F4F0E9430519E012B5BA8
:10F5B0003F4F44E050E0BE01635D7F4FCE01855B6D
:10F5C0009F4F0E9430519E012B5B3F4F44E050E023
:10F5D000BE016F5C7F4FCE01855B9F4F0E94305113
:10F5E0000AE010E0015011090115110571F09E01AA
:10F5F0002B5B3F4F44E050E0BE01635C7F4FCE0188
:10F60000855B9F4F0E943051EDCF60961FAE609793
:10F6100021961CAE1DAE1EAE1FAE21978FEF2F960A
:10F620008FAF2F979E012B5B3F4F41E050E0BE0113
:10F63000615B7F4FCE01855B9F4F0E9430519E01E1
:10F640002B5B3F4F44E050E0BE01635C7F4FCE0137
:10F65000855B9F4F0E9430519E012B5B3F4F41E0E5
:10F6600050E0BE01625B7F4FCE01855B9F4F0E94E1
:10F67000305121961CAE1DAE1EAE1FAE21971DE06F
:10F68000115071F09E012B5B3F4F44E050E0BE01F2
:10F69000635C7F4FCE01855B9F4F0E943051F0CF5E
:10F6A00084EB90E09AA789A780EF90E09CA78BA7B6
:10F6B00086E490E09EA38DA38EE690E098A78FA3AA
:10F6C0001AA219A21CA21BA29E012B5B3F4F44E071
:10F6D00050E0BE01675D7F4FCE01855B9F4F0E946A
:10F6E00030519E012B5B3F4F44E050E0BE016B5D0B
:10F6F0007F4FCE01855B9F4F0E9430519E012B5B57
:10F700003F4F44E050E0BE016F5D7F4FCE01855B0F
:10F710009F4F0E943051C12C90E8D92E9BE3E92ED7
:10F7200095E4F92E812C912C20E8A22E2FE3B22E05
:10F73000111138C09E012B5B3F4F44E050E066ED55
:10F7400073E0CE01855B9F4F0E9430519E012B5B81
:10F750003F4F44E050E062ED73E0CE01855B9F4F88
:10F760000E9430519E012B5B3F4F44E050E06EEC15
:10F7700073E0CE01855B9F4F0E94305121968CAE85
:10F780009DAEAEAEBFAE21979E012B5B3F4F44E0D6
:10F7900050E0BE01635C7F4FCE01855B9F4F0E94AE
:10F7A00030512AC02196CCAEDDAEEEAEFFAE219731
:10F7B0009E012B5B3F4F44E050E0BE01635C7F4FF6
:10F7C000CE01855B9F4F0E94305121961CAE1DAE2D
:10F7D0001EAE1FAE219704E0015071F09E012B5B1D
:10F7E0003F4F44E050E0BE01635C7F4FCE01855B3C
:10F7F0009F4F0E943051F0CF1F5F153009F098CF16
:10F8000084E190E025969FAF8EAF25979E012B5BFC
:10F810003F4F42E050E0BE016D5B7F4FCE01855B04
:10F820009F4F0E9430519E012B5B3F4F44E050E0C0
:10F8300062EE73E0CE01855B9F4F0E9430519E01C6
:10F840002B5B3F4F44E050E06EED73E0CE01855BF3
:10F850009F4F0E9430519E012B5B3F4F44E050E090
:10F860006AED73E0CE01855B9F4F0E94305180E2CC
:10F8700090E023969FAF8EAF23979E012B5B3F4F67
:10F8800042E050E0BE016F5B7F4FCE01855B9F4F32
:10F890000E9430512E961FAE2E9780E090E0A0E49B
:10F8A000B0E48D8F9E8FAF8FB8A380E090E0A4E38B
:10F8B000B2E4898F9A8FAB8FBC8F1D8A1E8A1F8AF4
:10F8C000188E198A1A8A1B8A1C8A1D861E861F8614
:10F8D000188A80E090E0A0E5B1E489879A87AB8739
:10F8E000BC871D821E821F82188680E090E0A0E007
:10F8F000B1E489839A83AB83BC839E012B5B3F4F2A
:10F9000041E050E0BE01635B7F4FCE01855B9F4FBE
:10F910000E9430519E012B5B3F4F44E050E0BE01FE
:10F92000635E7F4FCE01855B9F4F0E9430519E01E9
:10F930002B5B3F4F44E050E0BE01675E7F4FCE013E
:10F94000855B9F4F0E9430519E012B5B3F4F44E0EF
:10F9500050E0BE016B5E7F4FCE01855B9F4F0E94E2
:10F9600030519E012B5B3F4F44E050E0BE016F5E83
:10F970007F4FCE01855B9F4F0E9430519E012B5BD4
:10F980003F4F44E050E0BE01635F7F4FCE01855B97
:10F990009F4F0E9430519E012B5B3F4F44E050E04F
:10F9A000BE01675F7F4FCE01855B9F4F0E94305144
:10F9B0009E012B5B3F4F44E050E0BE016B5F7F4FE9
:10F9C000CE01855B9F4F0E9430519E012B5B3F4FC4
:10F9D00044E050E0BE016F5F7F4FCE01855B9F4FDB
:10F9E0000E9430519E012B5B3F4F41E050E060EAA6
:10F9F00073E0CE01855B9F4F0E94305110E01111E2
:10FA00000EC080919C0390919D03A0919E03B091A4
:10FA10009F0321968CAF9DAFAEAFBFAF21979E01E4
:10FA20002B5B3F4F44E050E0BE01635C7F4FCE0153
:10FA3000855B9F4F0E9430511F5F153001F7809109
:10FA4000E30E9091E40E2B969FAF8EAF2B979E0105
:10FA50002B5B3F4F42E050E0BE01675B7F4FCE0122
:10FA6000855B9F4F0E94305180916E0E90916F0E7A
:10FA70002B969FAF8EAF2B979E012B5B3F4F42E0A3
:10FA800050E0BE01675B7F4FCE01855B9F4F0E94B8
:10FA900030518091F90D9091FA0D2B969FAF8EAF5A
:10FAA0002B979E012B5B3F4F42E050E0BE01675B0E
:10FAB0007F4FCE01855B9F4F0E9430512B961FAE2A
:10FAC0001EAE2B979E012B5B3F4F42E050E0BE01E4
:10FAD000675B7F4FCE01855B9F4F0E9430512B9615
:10FAE0001FAE1EAE2B979E012B5B3F4F42E050E0B6
:10FAF000BE01675B7F4FCE01855B9F4F0E943051F7
:10FB00002B961FAE1EAE2B979E012B5B3F4F42E004
:10FB100050E0BE01675B7F4FCE01855B9F4F0E9427
:10FB200030518091840D9091850D2B969FAF8EAFB3
:10FB30002B979E012B5B3F4F42E050E0BE01675B7D
:10FB40007F4FCE01855B9F4F0E9430512B961FAE99
:10FB50001EAE2B979E012B5B3F4F42E050E0BE0153
:10FB6000675B7F4FCE01855B9F4F0E9430512B9684
:10FB70001FAE1EAE2B979E012B5B3F4F42E050E025
:10FB8000BE01675B7F4FCE01855B9F4F0E94305166
:10FB90002B961FAE1EAE2B979E012B5B3F4F42E074
:10FBA00050E0BE01675B7F4FCE01855B9F4F0E9497
:10FBB00030512B961FAE1EAE2B979E012B5B3F4FF5
:10FBC00042E050E0BE01675B7F4FCE01855B9F4FF7
:10FBD0000E94305121961CAE1DAE1EAE1FAE219765
:10FBE0009E012B5B3F4F44E050E0BE01635C7F4FC2
:10FBF000CE01855B9F4F0E9430519E012B5B3F4F92
:10FC000044E050E0BE01635C7F4FCE01855B9F4FB7
:10FC10000E94305113E0115088F084E0189FB00129
:10FC20001124615F7B4F9E012B5B3F4F44E050E00E
:10FC3000CE01855B9F4F0E943051EDCF80915E06D3
:10FC4000811153C02D960EAD1FAD2D9727968EAD09
:10FC50009FAD279729969FAF8EAF299784E690E0B6
:10FC60002D969FAF8EAF2D979E012B5B3F4F44E0AB
:10FC700050E06FEF72E0CE01855B9F4F0E943051E4
:10FC80009E012B5B3F4F42E050E0BE01695B7F4F1E
:10FC9000CE01855B9F4F0E943051E9EBFCE08491DF
:10FCA0007F019FEFE91AF90A882321F00E94FD34B1
:10FCB000F701F5CFB8016456710987EF91E1BEDA1B
:10FCC00029964EAD5FAD299760E070E08AEE91E134
:10FCD00008D9E7EEF1E184918F010F5F1F4F882370
:10FCE00021F00E94FD34F801F6CF90915E0681E08C
:10FCF0008927CB5ADF4F0FB6F894DEBF0FBECDBFBA
:10FD0000DF91CF911F910F91FF90EF90DF90CF90F7
:10FD1000BF90AF909F908F900895CF93DF93EC01A9
:10FD2000862F0E94FD34CD5ADF4F88819981AA81A8
:10FD3000BB8188279927AF77BB27CD01AA27BB278F
:10FD4000BC01660F771F6078682B772767FD709579
:10FD500083EA91E173DA8AE0DF91CF910C94FD346C
:10FD6000CF93C0912F0FC13009F448C0C23069F45D
:10FD70008FE29FE00E94E7386093300F7093310F5D
:10FD80008093320F9093330F18C01092340F10925B
:10FD9000350F1092360F1092370F1092380F1092C5
:10FDA000390F10923A0F10923B0F1092300F1092B1
:10FDB000310F1092320F1092330F81E080932F0F8A
:10FDC0000E94DB386093340F7093350F8093360FA9
:10FDD0009093370FC230A1F080913C0F90913D0F6E
:10FDE000019690933D0F80933C0F1092520F10920A
:10FDF000530F1092540F1092550F02C080E001C0B3
:10FE000081E0CF910895CF92DF92EF92FF920F930E
:10FE10001F93CF93DF93EB01FC016081718182819D
:10FE200093812CE3C22ED12CE12CF12CA701960159
:10FE30000E9494B7162F072FCA01B901A701960196
:10FE40000E9494B7F62EE72ECA01B90128E130E0EE
:10FE500040E050E00E9494B7FB01C9016DE671E0FB
:10FE60000E94B4BA9B014F2D5E2D21153105D9F0AA
:10FE70000F931F93EF92FF92FF93EF939F938F93B4
:10FE80003F932F938BE295E19F938F93DF93CF93D3
:10FE90000E9460B38DB79EB70E960FB6F8949EBFC2
:10FEA0000FBE8DBF5BC00097C9F00F931F93EF92F9
:10FEB000FF92FF93EF939F938F938BE195E19F9335
:10FEC0008F93DF93CF930E9460B3EDB7FEB73C965C
:10FED0000FB6F894FEBF0FBEEDBF40C03097B9F02B
:10FEE0000F931F93EF92FF92FF93EF938FE095E1B3
:10FEF0009F938F93DF93CF930E9460B38DB79EB78C
:10FF00000A960FB6F8949EBF0FBE8DBF27C0452B33
:10FF1000A9F00F931F93EF92FF9287E095E19F93D3
:10FF20008F93DF93CF930E9460B3EDB7FEB73896FF
:10FF30000FB6F894FEBF0FBEEDBF10C00F931F9316
:10FF400083E095E19F938F93DF93CF930E9460B3FB
:10FF50000F900F900F900F900F900F90DF91CF9117
:10FF60001F910F91FF90EF90DF90CF9008952F9207
:10FF70003F924F925F926F927F928F929F92AF9239
:10FF8000BF92CF92DF92EF92FF920F931F93CF9386
:10FF9000DF93CDB7DEB768970FB6F894DEBF0FBE1C
:10FFA000CDBF1C015B018A01DC01D7966D917D916B
:10FFB0008D919C91DA970E9492B36B017C01F501BF
:10FFC00020813181428153810E94F3B30E94B2B8F3
:10FFD0000E9435B969877A878B879C87D8012D91D4
:10FFE0003D914D915C91C701B6010E94F3B30E940F
:10FFF000B2B80E9435B96D877E878F87988B298527
:020000021000EC
:100000003A854B855C85283731054105510540F41B
:1000100088E790E0A0E0B0E089879A87AB87BC874B
:100020002D853E854F855889283731054105510575
:1000300040F488E790E0A0E0B0E08D879E87AF872E
:10004000B88B91012D5B3F4FD9018D919D910D9002
:10005000BC91A02D8D839E83AF83B887BC01CD0159
:100060000E9494B369837A838B839C8369857A85A4
:100070008B859C850E9492B3698B7A8B8B8B9C8B32
:1000800020E030E0A90169817A818B819C810E9406
:100090008EB3882339F1A7019601C701B6010E94EA
:1000A000F3B34B015C0129893A894B895C89CA0108
:1000B000B9010E94F3B39B01AC01C501B4010E94D8
:1000C000EBB74B015C0129813A814B815C81CA010C
:1000D000B9010E94ECB79B01AC01C501B4010E94BB
:1000E000C8B803C060E070E0CB010E94B2B80E94C3
:1000F00030B92B013C016D817E818F81988590956F
:100100008095709561957F4F8F4F9F4F0E9494B35C
:100110004B015C016D857E858F8598890E9492B325
:100120006D837E838F83988720E030E0A901C5012D
:10013000B4010E948EB3882349F12D813E814F8105
:100140005885CA01B9010E94F3B36D8B7E8B8F8BEA
:10015000988FA7019601C701B6010E94F3B39B01D6
:10016000AC016D897E898F89988D0E94EBB76B01F8
:100170007C01A5019401C501B4010E94ECB79B016B
:10018000AC01C701B6010E94C8B803C060E070E0CE
:10019000CB010E9461B9F10182889388A488B58857
:1001A00075016401C418D508E608F7080E9430B943
:1001B000C61AD70AE80AF90AF7FE6BC020E030E059
:1001C000A90169817A818B819C810E948EB38823E9
:1001D00009F447C029813A814B815C81CA01B90188
:1001E0000E94ECB76B017C01C501B4010E9492B37F
:1001F0009B01AC01C701B6010E94F3B36B017C0106
:1002000029893A894B895C89CA01B9010E94F3B3F3
:100210009B01AC01C701B6010E94EBB76B017C01E9
:100220002D813E814F815885CA01B9010E94F3B3E7
:100230009B01AC01C701B6010E94ECB76B017C01C8
:1002400020E030E040E850E469817A818B819C8134
:100250000E94F3B39B01AC01C701B6010E94C8B86C
:1002600003C060E070E0CB010E94B2B80E9430B9D8
:100270002B013C0197FF03C0412C512C3201481443
:1002800059046A047B0410F024013501C12CD12CDF
:1002900076018FB7F894D1019C9193FD22C0F101B2
:1002A000468A578A608E718EC40CD51CE61CF71CDA
:1002B0005A96CD92DD92ED92FC925D9729853A8512
:1002C0004B855C85DB962D933D934D935C93DE9738
:1002D000FF962D853E854F85588920833183428343
:1002E00053838FBF68960FB6F894DEBF0FBECDBFA5
:1002F000DF91CF911F910F91FF90EF90DF90CF9002
:10030000BF90AF909F908F907F906F905F904F9035
:100310003F902F900895FF920F931F93CF93DF93F9
:10032000EC0184E50E94CC37882351F10E94E3352B
:10033000F82E181614F5E9EBFCE084918F010F5F9D
:100340001F4F882321F00E94FD34F801F6CF8DE481
:100350000E94FD34BE0180E090E04AE00E940077F8
:100360006F2D772767FD709580EF94E10E941E79CD
:100370008AE00E94FD3481E008C08093EE0304C04F
:1003800080911B048093EE0380E0DF91CF911F9159
:100390000F91FF900895CF93DF938DED90E0BBDF39
:1003A000811111C083E50E94CC37882361F0C09190
:1003B000EE03D0E00E94D335FE01EE0FFF1FEF5C8D
:1003C000FD4F71836083DF91CF9108950F931F9349
:1003D000CF93DF93EC01862F0E94FD34E9EDF4E129
:1003E00084918F010F5F1F4F882321F00E94FD34FD
:1003F000F801F6CFCD58DF4F6881798180E090E039
:100400004AE00E9400778AE0DF91CF911F910F911F
:100410000C94FD34CF92DF92EF92FF92CF93DF9353
:100420006A017B01FC018491EF012196882321F070
:100430000E94FD34FE01F7CF42E0C701B601DF9113
:10044000CF91FF90EF90DF90CF900C94B377CF9344
:10045000DF93E9EBFCE08491EF012196882321F002
:100460000E94FD34FE01F7CF83E50E9442378823C6
:1004700021F00E94F43580933002E1E3F2E18491AF
:10048000EF012196882321F00E94FD34FE01F7CF71
:1004900080913002882319F0E9E2F2E102C0EDE236
:1004A000F2E18491EF012196882321F00E94FD342E
:1004B000FE01F7CFE1E2F2E18491EF01219688237A
:1004C00021F00E94FD34FE01F7CF4091FC035091D2
:1004D000FD036091FE037091FF038FE192E19ADFCB
:1004E0004091000450910104609102047091030452
:1004F0008CE192E18FDF40910404509105046091FA
:1005000006047091070489E192E184DFE1E1F2E100
:100510008491EF012196882321F00E94FD34FE0191
:10052000F7CF409116025091170260911802709116
:1005300019028FE092E16EDF40911A0250911B0286
:1005400060911C0270911D028CE092E163DF40918A
:100550001E0250911F02609120027091210289E0D9
:1005600092E158DF8AE0DF91CF910C94FD34CF9275
:10057000DF92EF92FF92CF93DF936A017B01FC0140
:100580008491EF012196882321F00E94FD34FE0121
:10059000F7CF42E0C701B601DF91CF91FF90EF9016
:1005A000DF90CF900C94B3770F931F93CF93C82F06
:1005B000882319F0E1ECF4E10CC0E9EBFCE0849154
:1005C0008F010F5F1F4F8823A9F30E94FD34F801AC
:1005D000F6CF84918F010F5F1F4F882321F00E9477
:1005E000FD34F801F6CF8AE00E94FD34C1112DC020
:1005F000E9EBFCE084918F010F5F1F4F882321F00E
:100600000E94FD34F801F6CFEEEAF4E184918F0107
:100610000F5F1F4F882321F00E94FD34F801F6CFB1
:100620008091A003882321F08AE00E94FD34ECC36E
:10063000E3EAF4E184918F010F5F1F4F882309F4EF
:10064000E3C30E94FD34F801F5CF40919C03509123
:100650009D0360919E0370919F038AE994E1DADE25
:100660008AE00E94FD348091A00381111BC0CC233D
:1006700019F0EFE8F4E10CC0E9EBFCE084918F01A4
:100680000F5F1F4F8823A9F30E94FD34F801F6CFB6
:1006900084918F010F5F1F4F882321F00E94FD344A
:1006A000F801F6CFC11124C0E9EBFCE084918F0181
:1006B0000F5F1F4F882321F00E94FD34F801F6CF11
:1006C000EEE7F4E184918F010F5F1F4F882321F043
:1006D0000E94FD34F801F6CFE9EBFCE084918F0134
:1006E0000F5F1F4F882321F00E94FD34F801F6CFE1
:1006F0004091890350918A0360918B0370918C0320
:1007000086E794E187DE40918D0350918E036091DE
:100710008F037091900383E794E17CDE4091910315
:1007200050919203609193037091940380E794E158
:1007300071DE4091950350919603609197037091FB
:1007400098038DE694E166DE8AE00E94FD34C111D3
:1007500024C0E9EBFCE084918F010F5F1F4F8823D9
:1007600021F00E94FD34F801F6CFEFE4F4E184912A
:100770008F010F5F1F4F882321F00E94FD34F80185
:10078000F6CFE9EBFCE084918F010F5F1F4F8823C8
:1007900021F00E94FD34F801F6CF4091B103509151
:1007A000B2036091B3037091B40386E494E132DE46
:1007B0004091B5035091B6036091B7037091B803AF
:1007C00083E494E127DE4091B9035091BA0360912C
:1007D000BB037091BC0380E494E11CDE4091BD0337
:1007E0005091BE036091BF037091C0038DE394E10B
:1007F00011DE8AE00E94FD34C11124C0E9EBFCE067
:1008000084918F010F5F1F4F882321F00E94FD34D8
:10081000F801F6CFEBE1F4E184918F010F5F1F4FF8
:10082000882321F00E94FD34F801F6CFE9EBFCE0CB
:1008300084918F010F5F1F4F882321F00E94FD34A8
:10084000F801F6CF4091A1035091A2036091A30358
:100850007091A40382E194E10E9471774091A50315
:100860005091A6036091A7037091A8038FE094E1D3
:100870000E9471774091A9035091AA036091AB0344
:100880007091AC038CE094E10E9471774091AD03CC
:100890005091AE036091AF037091B00389E094E191
:1008A0000E9471778AE00E94FD34C11124C0E9EBF7
:1008B000FCE084918F010F5F1F4F882321F00E947D
:1008C000FD34F801F6CFEFEBF3E184918F010F5F78
:1008D0001F4F882321F00E94FD34F801F6CFE9EB89
:1008E000FCE084918F010F5F1F4F882321F00E944D
:1008F000FD34F801F6CF4091C9035091CA036091CD
:10090000CB037091CC0386EB93E184DD4091C1036E
:100910005091C2036091C3037091C40383EB93E1D0
:1009200079DD4091C5035091C6036091C703709172
:10093000C80380EB93E16EDD8AE00E94FD34C111B3
:1009400024C0E9EBFCE084918F010F5F1F4F8823E7
:1009500021F00E94FD34F801F6CFECE3F3E184913D
:100960008F010F5F1F4F882321F00E94FD34F80193
:10097000F6CFE9EBFCE084918F010F5F1F4F8823D6
:1009800021F00E94FD34F801F6CF409167065091A6
:1009900068066091690670916A0683E393E13ADD27
:1009A00040916306509164066091650670916606F9
:1009B00080E393E12FDD40915F06509160066091E6
:1009C0006106709162068DE293E10E947177409119
:1009D000790350917A0360917B0370917C038AE2E2
:1009E00093E118DD40917D0350917E0360917F0378
:1009F0007091800387E293E10DDD40918103509176
:100A00008203609183037091840384E293E102DDA9
:100A1000409185035091860360918703709188030C
:100A200081E293E1F7DC8AE00E94FD34C11124C029
:100A3000E9EBFCE084918F010F5F1F4F882321F0C9
:100A40000E94FD34F801F6CFE3E1F3E184918F01D8
:100A50000F5F1F4F882321F00E94FD34F801F6CF6D
:100A6000E9EBFCE084918F010F5F1F4F882321F099
:100A70000E94FD34F801F6CF4091EE055091EF054C
:100A80006091F0057091F1058AE093E1C3DC40913B
:100A9000F2055091F3056091F4057091F50587E03A
:100AA00093E1B8DC4091F6055091F7056091F805A7
:100AB0007091F90584E093E1ADDC8AE00E94FD3499
:100AC000C11124C0E9EBFCE084918F010F5F1F4F3F
:100AD000882321F00E94FD34F801F6CFE0EFF2E127
:100AE00084918F010F5F1F4F882321F00E94FD34F6
:100AF000F801F6CFE9EBFCE084918F010F5F1F4F07
:100B0000882321F00E94FD34F801F6CF6091EF03B5
:100B100070E087EE92E10E941E798AE00E94FD3427
:100B2000C11124C0E9EBFCE084918F010F5F1F4FDE
:100B3000882321F00E94FD34F801F6CFE8EDF2E1C0
:100B400084918F010F5F1F4F882321F00E94FD3495
:100B5000F801F6CFE9EBFCE084918F010F5F1F4FA6
:100B6000882321F00E94FD34F801F6CF4091D6038E
:100B70005091D7036091D8037091D9038FEC92E123
:100B800049DC2CEA35EC47E25EE36091D2037091D8
:100B9000D3038091D4039091D5030E94C8B8AB01D0
:100BA000BC018CEC92E1E3DC2CEA35EC47E25EE33D
:100BB0006091CE037091CF038091D0039091D103C7
:100BC0000E94F3B3AB01BC0189EC92E1D0DC8AE076
:100BD0000E94FD34C1110CC0E9EBFCE084918F014F
:100BE0000F5F1F4F882321F00E94FD34F801F6CFDC
:100BF0004091E2035091E3036091E4037091E503B7
:100C000080EC92E107DC2CEA35EC47E25EE3609190
:100C1000DE037091DF038091E0039091E1030E9475
:100C2000C8B8AB01BC018DEB92E1A1DC2CEA35EC3C
:100C300047E25EE36091DA037091DB038091DC03AD
:100C40009091DD030E94F3B3AB01BC018AEB92E10A
:100C50008EDC8AE00E94FD34C11124C0E9EBFCE087
:100C600084918F010F5F1F4F882321F00E94FD3474
:100C7000F801F6CFE4EAF2E184918F010F5F1F4F94
:100C8000882321F00E94FD34F801F6CFE9EBFCE067
:100C900084918F010F5F1F4F882321F00E94FD3444
:100CA000F801F6CF40910B0450910C0460910D04B3
:100CB00070910E048BE992E1ADDB8AE00E94FD3475
:100CC000CC2319F00CE013E024C0E9EBFCE08491A4
:100CD0008F010F5F1F4F882321F00E94FD34F80120
:100CE000F6CFE2E8F2E184918F010F5F1F4F882376
:100CF00021F00E94FD34F801F6CFE9EBFCE084918D
:100D00008F010F5F1F4F8823E9F20E94FD34F80125
:100D1000F6CFF80181918F01882319F00E94FD34EC
:100D2000F8CF6091E30E7091E40E8FE792E10E949C
:100D30001E7960916E0E70916F0E8CE792E10E94A9
:100D40001E796091F90D7091FA0D89E792E10E9488
:100D50001E796091840D7091850D85E792E10E9466
:100D60001E798AE00E94FD34C11124C0E9EBFCE049
:100D700084918F010F5F1F4F882321F00E94FD3463
:100D8000F801F6CFECE5F2E184918F010F5F1F4F80
:100D9000882321F00E94FD34F801F6CFE9EBFCE056
:100DA00084918F010F5F1F4F882321F00E94FD3433
:100DB000F801F6CF40910F04509110046091110496
:100DC0007091120483E592E10E94717740911304BF
:100DD00050911404609115047091160480E592E11D
:100DE0000E94717740911704509118046091190482
:100DF00070911A048DE492E10E9471778AE0CF919C
:100E00001F910F910C94FD34E9EBFCE084918F016C
:100E10000F5F1F4F882309F418CC0E94FD34F8019E
:100E2000F5CFCF93DF9385E40E94CC37811110C0BA
:100E300080E50E944237882391F00E940336609338
:100E4000D6037093D7038093D8039093D90307C038
:100E50000E94E335882361F3E5EEFAE06AC089E495
:100E60000E944237882381F00E9403362CEA35EC39
:100E700047E25EE30E94F3B36093D2037093D3031F
:100E80008093D4039093D50384E40E94423788234F
:100E900081F00E9403362CEA35EC47E25EE30E94C3
:100EA000C8B86093CE037093CF038093D003909320
:100EB000D103E9EBFCE08491EF012196882321F036
:100EC0000E94FD34FE01F7CF4091D6035091D70325
:100ED0006091D8037091D90389E492E19BDA2CEAFE
:100EE00035EC47E25EE36091D2037091D3038091C9
:100EF000D4039091D5030E94C8B8AB01BC0185E42E
:100F000092E135DB2CEA35EC47E25EE36091CE03FB
:100F10007091CF038091D0039091D1030E94F3B3DD
:100F2000AB01BC0181E492E122DB10C00E94FD34E0
:100F3000FE018491EF0121968111F8CFCBEDD2E033
:100F40008991882319F00E94FD34FACF8AE0DF915D
:100F5000CF910C94FD34CF93DF93EC0181E08FA30C
:100F6000CE010D9620E1FC0111922A95E9F76D8DD5
:100F70007E8D6F5F7F4F40E150E00E945CB666E17E
:100F80008D8D9E8DDF91CF910C947DB68F929F9227
:100F9000AF92BF92CF92DF92EF92FF920F931F9387
:100FA000CF93DF93CDB7DEB760970FB6F894DEBF6F
:100FB0000FBECDBF490194E0890250011124F50113
:100FC000E650FA4F6F0110821182128213824D8710
:100FD0005E876F87788B0E941B614D855E856F856C
:100FE0007889F6014083518362837383C0901B0428
:100FF00020E030E0A901B801C4010E948EB3811144
:1010000008C0F501EC5CF84E85909590A590B490E1
:1010100004C0C801D4014C015D0180910206909189
:101020000306A0910406B09105064091FE0550917B
:10103000FF0560910006709101060091FA0510917C
:10104000FB052091FC053091FD0509831A832B8354
:101050003C834D835E836F83788789879A87AB87CC
:10106000BC87AE01475F5F4FBE016B5F7F4FCE0114
:1010700001960E94EF2E8501740126E036E0AE0154
:10108000475F5F4FBE016B5F7F4FCE0101960E94AD
:10109000BA610E94345E1092570660960FB6F894BB
:1010A000DEBF0FBECDBFDF91CF911F910F91FF909B
:1010B000EF90DF90CF90BF90AF909F908F9008956A
:1010C0002F923F924F925F926F927F928F929F9258
:1010D000AF92BF92CF92DF92EF92FF920F931F9346
:1010E000CF93DF93CDB7DEB7C255D1090FB6F894D1
:1010F000DEBF0FBECDBF9AAF89AF362EDC018D901B
:101100009D90AD90BC9013972401350177FA7094AF
:1011100077F870941496CD90DD90ED90FC90179731
:10112000D701C601B0588D8F9E8FAF8FB8A3A30192
:101130009201C301B2010E94F3B36DA37EA38FA3FA
:1011400098A72D8D3E8D4F8D58A1CA01B9010E94DF
:10115000F3B39B01AC016DA17EA18FA198A50E9464
:10116000ECB70E9457BA23966CAF7DAF8EAF9FAF9E
:1011700023978091FA059091FB05A091FC05B09111
:10118000FD058DA39EA3AFA3B8A7A5019401BC0143
:10119000CD010E94ECB72F966CAF7DAF8EAF9FAFA5
:1011A0002F978091FE059091FF05A0910006B091C8
:1011B000010689A79AA7ABA7BCA7A7019601BC0106
:1011C000CD010E94ECB763966CAF7DAF8EAF9FAF41
:1011D00063978091460390914703A0914803B09193
:1011E000490389AB9AABABABBCAB2F962CAD3DADF5
:1011F0004EAD5FAD2F97BC01CD010E94EBB76B01E7
:101200007C0180914A0390914B03A0914C03B091D3
:101210004D038DAB9EABAFABB8AF63962CAD3DAD80
:101220004EAD5FAD6397BC01CD010E94EBB74B01A2
:101230005C018091020690910306A0910406B09192
:1012400005068DA79EA7AFA7B8AB9C01AD01609125
:101250004E0370914F0380915003909151030E946F
:10126000EBB769A37AA38BA39CA3809152039091BF
:101270005303A0915403B091550327968CAF9DAFB3
:10128000AEAFBFAF27978091060690910706A09159
:101290000806B09109068BAF9CAFADAFBEAFA701FA
:1012A0009601C301B2010E94F3B32B966CAF7DAFE0
:1012B0008EAF9FAF2B97A50194016D8D7E8D8F8D85
:1012C00098A10E94F3B39B01AC012B966CAD7DAD50
:1012D0008EAD9FAD2B970E94ECB72B966CAF7DAF78
:1012E0008EAF9FAF2B97A5019401C301B2010E945D
:1012F000F3B34B015C01A70196016D8D7E8D8F8D3F
:1013000098A10E94F3B39B01AC01C501B4010E94F6
:10131000EBB72B962CAD3DAD4EAD5FAD2B970E943C
:101320005FB86B017C0120E030E0A9010E948EB320
:1013300087FF0AC02BED3FE049EC50E4C701B6013E
:101340000E94ECB76B017C01332051F02BED3FE0A4
:1013500049EC50E4C701B6010E94EBB76B017C0178
:1013600020E030E0A901C701B6010E948EB38111CF
:1013700020C029A93AA94BA95CA96DA17EA18FA182
:1013800098A50E948EB3811114C02DA93EA94FA922
:1013900058AD69A57AA58BA59CA50E948EB3811135
:1013A00008C09BEDC92E9FE0D92E99ECE92E90E460
:1013B000F92E23962CAD3DAD4EAD5FAD2397C70101
:1013C000B6010E94F3B39B01AC010E94F3B34B0141
:1013D0005C0129A13AA14BA15CA1CA01B9010E94FB
:1013E000F3B39B01AC01C501B4010E94ECB70E94AC
:1013F00057BA4B015C012FE632E143E85AE30E9401
:101400008EB387FD25C2C501B4010E9461B90E9457
:1014100035B97AA769A7DB01AB2B21F4E1E0F0E055
:10142000FAA7E9A729A53AA5B90180E090E00E94B2
:1014300092B34B015C019B01AC01C701B6010E9454
:10144000C8B86DA37EA38FA398A7A501940169A135
:101450007AA18BA19CA10E94C8B823966CAF7DAFE6
:101460008EAF9FAF23972BAD3CAD4DAD5EAD2796B4
:101470006CAD7DAD8EAD9FAD27970E94EBB7A501FA
:1014800094010E94C8B827966CAF7DAF8EAF9FAF16
:1014900027972DA13EA14FA158A5CA01B9010E94CD
:1014A000F3B320E030E040E05FE30E94F3B39B0140
:1014B000AC0160E070E080E89FE30E94EBB769ABAD
:1014C0007AAB8BAB9CAB8DA59EA5AFA5B8A9898740
:1014D0009A87AB87BC878BAD9CADADADBEAD8D871C
:1014E0009E87AF87B88B6091120270911302882794
:1014F00077FD8095982F0E9494B320910A02309135
:101500000B0240910C0250910D020E94F3B32AE0AD
:1015100037ED43E25CE30E94F3B36DAB7EAB8FAB80
:1015200098AF0E94DB384B015C0198EC890E911C4E
:10153000A11CB11C22242394312CA9E1A9A329A523
:101540003AA52216330608F041C10E9470A90E94F4
:10155000DB38681979098A099B0997FD0BC00E943D
:10156000DB384B015C01B8EC8B0E911CA11CB11C4B
:101570000E940872E9A1E150E9A3EE2309F43FC0FB
:1015800029A93AA94BA95CA96D8D7E8D8F8D98A153
:101590000E94F3B36B017C012DA13EA14FA158A580
:1015A000C301B2010E94F3B3A70196010E94ECB7F8
:1015B0006DA77BAF8C0129A93AA94BA95CA9C301EE
:1015C000B2010E94F3B36B017C012DA13EA14FA19A
:1015D00058A56D8D7E8D8F8D98A10E94F3B39B01D0
:1015E000AC01C701B6010E94EBB72B013C018DA5F0
:1015F0009BADD8018D8F9E8FAF8FB8A36CC0B1010A
:1016000080E090E00E9492B32DA13EA14FA158A589
:101610000E94F3B36B017C010E94C5B86D8F7E8F71
:101620008F8F98A3C701B6010E944DBA69A37AA310
:101630008BA39CA3A9ADBAADCD90DD90ED90FC90AD
:101640001397F7FAF094F7F8F09414968D919D9112
:101650000D90BC91A02D8DA79EA7AFA7B8AB2D8DE7
:101660003E8D4F8D58A1C701B6010E94F3B32B01E7
:101670003C0129A13AA14BA15CA16DA57EA58FA536
:1016800098A90E94F3B39B01AC01C301B2010E946F
:10169000ECB72B013C0129A13AA14BA15CA1C701E8
:1016A000B6010E94F3B36B017C012D8D3E8D4F8DF1
:1016B00058A16DA57EA58FA598A90E94F3B39B01A3
:1016C000AC01C701B6010E94EBB76D8F7E8F8F8F83
:1016D00098A3B9E1B9A3A30192012F966CAD7DAD9A
:1016E0008EAD9FAD2F970E94ECB769837A838B8371
:1016F0009C832D8D3E8D4F8D58A163966CAD7DAD35
:101700008EAD9FAD63970E94ECB76D837E838F8310
:10171000988723962CAD3DAD4EAD5FAD239769857F
:101720007A858B859C850E94ECB769877A878B8741
:101730009C8727962CAD3DAD4EAD5FAD27976D854F
:101740007E858F8598890E94ECB76D877E878F870D
:10175000988BCE0101960E947936C0901B04898136
:101760009A81AB81BC81898B9A8BAB8BBC8B8D8131
:101770009E81AF81B8858D8B9E8BAF8BB88F89850D
:101780009A85AB85BC85898F9A8FAB8FBC8FAE0154
:10179000475E5F4FBE016B5E7F4FCE0141960E9458
:1017A000EF2EEDA8FEA80FA918AD9E01235F3F4FB5
:1017B000AE01475E5F4FBE016B5E7F4FCE0141962B
:1017C0000E94BA61EFEF2E1A3E0AB9CEC0901B04F8
:1017D0008091460390914703A0914803B09149033B
:1017E000898B9A8BAB8BBC8B80914A0390914B0376
:1017F000A0914C03B0914D038D8B9E8BAF8BB88F16
:1018000080914E0390914F03A0915003B0915103EA
:10181000898F9A8FAB8FBC8FAE01475E5F4FBE0141
:101820006B5E7F4FCE0141960E94EF2EEDA8FEA881
:101830000FA918AD22E533E0AE01475E5F4FBE0150
:101840006B5E7F4FCE0141960E94BA610E94CE36F8
:10185000CE5ADF4F0FB6F894DEBF0FBECDBFDF917B
:10186000CF911F910F91FF90EF90DF90CF90BF909D
:10187000AF909F908F907F906F905F904F903F9030
:101880002F9008954F925F926F927F929F92AF92A6
:10189000BF92CF92DF92EF92FF920F931F93CF935D
:1018A000DF93982EC82FDD27C7FDD095FE01EF5797
:1018B000F84E1491811104C061E080E79EE006C0FB
:1018C00081E0981205C061E08BEF9DE00E94AE764A
:1018D000FE01EE0FFF1FEE0FFF1FEB58F84E459075
:1018E000559065907490612F772767FD7095872FCD
:1018F000972F0E9494B36B017C0120E030E040EC14
:101900005FE3C301B2010E94F3B3A70196010E94F5
:10191000F3B3AB01BC0100E010E09801892D36DB88
:10192000FE01EE0FFF1FEE0FFF1FE759F84E259146
:10193000359145915491C701B6010E94F3B36B01F3
:101940007C0120E030E0A9010E948EB35E01AA0C68
:10195000BB1CAA0CBB1C882309F447C000E010E0A4
:101960009801B701A6017058892D10DBFE01EA59D4
:10197000F84E6491611119C0E9EBFCE084918F018C
:101980000F5F1F4F882321F00E94FD34F801F6CF2E
:10199000E4E4F7E184918F010F5F1F4F882321F06A
:1019A0000E94FD34F801F6CF6AE0F501EC5CF84ED8
:1019B000459055906590749070E080E090E00E94B2
:1019C00094B39B01AC01C301B2010E94C8B82B01C2
:1019D0003C01A7019601C701B6010E94ECB7AB011B
:1019E000BC0193018201892DD1DAFE01E85FFB4F32
:1019F00081E08083FE01E651FA4F8083F501E85DC6
:101A0000F84F1082118212821382892D0E94D836DB
:101A1000F501E656F94F6591759185919491CC0F3A
:101A2000DD1FCC0FDD1F8E0106501A4FFE01E05165
:101A3000FC4F20813181428153810E94ECB7F80133
:101A400060837183828393830E941B61CA5BDC4F36
:101A5000F80180819181A281B38188839983AA83CF
:101A6000BB83911004C060E080E79EE006C0F1E017
:101A70009F1214C060E08BEF9DE0DF91CF911F912A
:101A80000F91FF90EF90DF90CF90BF90AF909F901D
:101A90007F906F905F904F900C94AE76DF91CF91D6
:101AA0001F910F91FF90EF90DF90CF90BF90AF907C
:101AB0009F907F906F905F904F9008952F923F92EC
:101AC0004F925F926F927F928F929F92AF92BF924E
:101AD000CF92DF92EF92FF920F931F93CF93DF93FA
:101AE000CDB7DEB7C150D1400FB6F894DEBF0FBE00
:101AF000CDBF0E94FF4F81110C94E39BFE013196F4
:101B00008CE3DF011D928A95E9F7C090EF03C6527E
:101B1000DF4FC882CA5DD0408AE40E9442378823E2
:101B200021F00E9488A60C94E39B86E50E94CC37A6
:101B3000882349F00E94D335CC52DF4F79836883E4
:101B4000C45DD04006C0CC52DF4F19821882C45DFC
:101B5000D040CC52DF4F28813981C45DD040253040
:101B6000310570F0ECE0F7E184918F010F5F1F4FBA
:101B7000882311F40C94E39B0E94FD34F801F4CF08
:101B800084E40E944237882341F00E94F435C15218
:101B9000DF4F8883CF5DD04005C0C152DF4F188230
:101BA000CF5DD040CC52DF4F48815981C45DD040D9
:101BB000433051056CF484E50E944237882379F064
:101BC0000E94F435C352DF4F8883CD5DD0400CC0F6
:101BD00051E0C352DF4F5883CD5DD04005C0C352A2
:101BE000DF4F1882CD5DD04088E50E94CC37882336
:101BF00021F00E94D335162F01C012E089E50E9422
:101C0000CC37882321F00E94D335062F01C002E093
